:020000040800F2
:10000000005000201DA30008BDA30008158E0008A5
:10001000BDA30008BDA30008BDA3000800000000A8
:10002000000000000000000000000000BDA3000868
:10003000BDA3000800000000BDA30008413D00086A
:10004000BDA30008BDA30008BDA30008BDA3000810
:10005000BDA30008BDA30008BDA30008BDA3000800
:10006000BDA30008BDA30008BDA30008BDA30008F0
:10007000BDA30008BDA300084D7C0008BDA3000877
:10008000BDA30008BDA30008BDA30008BDA30008D0
:10009000BDA30008BDA30008BDA30008BDA30008C0
:1000A000BDA30008817A0008BDA30008917A00086A
:1000B000757A0008657A0008557A0008E120000882
:1000C000E5200008DB200008DF200008BDA30008B1
:1000D000BDA30008457C00083D7C0008BDA30008C6
:1000E000513D0008BDA30008BDA3000800000000AA
:1000F0000000000000000000000000000000000000
:0C01000000000000000000005FF808F1A3
:10010C002DE9F04F664B674C97B02360002363607A
:10011C0007F09EFA18B907F0BDFA05F027F805F0BC
:10012C00EFF8614A614D1378614F43F0010313708E
:10013C00002309930A930B934FF4E0130C932B6851
:10014C00B87B43F480332B60AB6943F01003AB6195
:10015C002B6803F400330A93099B013309930A9B20
:10016C001BB9099BB3F5A06FF2D12B684F4913F45F
:10017C00003301D0022315E00A6842F001020A6044
:10018C0009932B6803F002030A93099B013309932B
:10019C000A9B1BB9099BB3F5A06FF2D12B689B0787
:1001AC0034D501230B93434B43491A683F4E42F01D
:1001BC0010021A601A6822F003021A601A6842F0E0
:1001CC0002021A606B686B606B686B606B6843F45F
:1001DC0080636B60394B1A68043B22F070425A60A2
:1001EC00374A1160696821F47C116960596841F0E3
:1001FC0000415960D96821F40041D9604FF4E011F5
:10020C000C910B990293012901D118E0FEE7022908
:10021C0019D168B10C9BB3F5801F02D14FF4A01318
:10022C0005E00C9BB3F5E01F02D14FF400130C93C7
:10023C000C996B680B4343F480336B6003E0736879
:10024C0043F4601373602B6843F080732B60296850
:10025C00164B8E01FBD5596821F003015960596882
:10026C0041F0020159606B68104903F00C03082B34
:10027C00F9D14B68DFF8509003F00C03042B03D03A
:10028C00082B03D00C4B27E0136825E04B6848681B
:10029C00C3F38343C00303F1020317D4094A1AE0E2
:1002AC00C94A0008B00300200417002000100240C7
:1002BC00000A00200020024000127A0004100140C5
:1002CC002400002000093D00380000204968126815
:1002DC00890348BF52085343C9F800306B68BD4AC4
:1002EC00C3F30313D15CD9F800309046CB40C9F866
:1002FC000030029BDFF820B39B6816AE13F4004F5E
:10030C00B54B14BF022201221A70B44B4FF0000AF5
:10031C00CBF80C30AB69B24843F00103AB616B6AAC
:10032C00A3606B6A43F080736B62AB6943F01C0390
:10033C00AB614FF6FF7326F8183D31468DF842A09D
:10034C0001F096F9A748314601F092F93146A648DA
:10035C0001F08EF9A54A3046536843F000735360A0
:10036C0005F0C0FC109BA24AB646B3FBF2F3A14ABF
:10037C00DFF8A8C21360A04B4FF47A72C3F800A048
:10038C00D9F80030DFF89892B3FBF2F39B4A013BAB
:10039C005360F0238BF823300723C2F808A01360B6
:1003AC00BB68C9F80030BCE80F00AEE80F009CE851
:1003BC000300AB698EE8030043F01003AB61AB693B
:1003CC00029A43F01003AB61AB6943F01003AB61CD
:1003DC004FF480431361029A4FF400531361029A55
:1003EC004FF4004313610AF1040156F80A0031443A
:1003FC000AF1080A01F03CF9BAF1180FF3D1D9F857
:10040C0000301B0712D597F82231012B0ED8A268A9
:10041C007B4B12F0805B93F8233100F0768605E07D
:10042C00774B002283F8232105F0F2F8642003F0C7
:10043C0032FCA022734800210CF061FAEB69002217
:10044C0043F00703EB61AB6943F4006343F00C0327
:10045C00AB616D4D002305F10C01535401320E2A92
:10046C00F7D1FF22AA76EA762A776A77DFF8B4B159
:10047C00664ADFF8B4A1C2F800B0654A02211170D7
:10048C0050461946182203930CF039FA0122039BAB
:10049C008AF80C2097F805A0ABF5B3722A623046A7
:1004AC001946142285F81EA00CF029FABAF10E0F89
:1004BC0004D00AF0EF0ABAF1080F02D101238DF82B
:1004CC004A30012003F018F918B14088003018BFE9
:1004DC000120D9F8003000F00100C3F340028DF880
:1004EC004620C3F380128DF84820C3F340328DF8B8
:1004FC004020C3F3C0328DF8432013F400628DF812
:10050C00450004D097F81621561E72427241B7F876
:10051C00D8508DF84420ADF84E50C3F30042DD04A2
:10052C00C3F3804003F001018DF84920C3F3C002EE
:10053C0048BF334B8DF8470048BFB3F8E030B7F8ED
:10054C00E40048BFADF84E30B0F5FA7F84BF00230D
:10055C00ADF84E3097F86631ADF84C002D4884F864
:10056C002430002384F8253043709DF84A308DF8F0
:10057C004110002B8DF842200CBF0023022301B93F
:10058C0002B1013308EB8308D8F828304FF000088B
:10059C00A3F1020A1A3303934FF6FF723AF8023FA3
:1005AC00934200F00A81D9B2DFF880909DF84500A3
:1005BC000F011B0A09EB07054A4618B1023901293C
:1005CC0040F2F780022B33D19DF84020002A71D1E4
:1005DC00EFE000BF9CD40008141700200005FA05BA
:1005EC0000080140000C01400010014000000140D7
:1005FC0040420F00680700206C07002010E000E06C
:10060C00000A002018110020B0030020140700205D
:10061C00F0070020D503002000ED00E0ACD400086A
:10062C00E80F00207A0B0020F407002054E50008A6
:10063C00012B3FD19DF84130002B00F0BA80FF23F5
:10064C0084F86C3084F86D30D3195A7B586803F1F8
:10065C00080B1B890026ADF834300DA9022384F851
:10066C007060E5678DF837308DF8362084F8286097
:10067C00E66226636663A66684F86E6084F86F6033
:10068C0000F0F6FF9BF80210324659F8070006F00E
:10069C0005FE284605F0DEF9B74BB849C4F88030A2
:1006AC00B74BC4F88860C4F8843028460A1D07F09C
:1006BC0063FA7EE0022BDAB246D15FFA88F24FF091
:1006CC001C0909FB02F9DFF828C304EB0906012118
:1006DC0086F870100CEB070191F80DE001F108029F
:1006EC00486809894FF0000B86F87180ADF834101A
:1006FC0086F872B00DA986F87AB0F5678DF836E0F9
:10070C008DF83730CDF814C0049200F0B1FFDDF84D
:10071C0014C0049A5CF8070091785A4606F0BEFDA6
:10072C00284605F097F9974A9449C6F88020964ACE
:10073C004944C6F88420C6F888B028460A1D07F03C
:10074C001BFA08F1010834E0032A32D19DF8473036
:10075C008E4E3BB194F82670284608214FF6FF7256
:10076C0000231BE0BDF84C208949B2F5FA7FBDF897
:10077C004E3091F826700BD986492846B1FBF2F21F
:10078C00082192B200F0A6FF834B46F827000AE03E
:10079C0082492846B1FBF2F2012192B200F09AFF95
:1007AC007F4B46F82700C36094F82630013384F859
:1007BC002630039B9A457FF4EFAE7A4B04221A70D5
:1007CC000026794D794B354433441036402E0FCBEF
:1007DC0085E80F00F5D106F0EFFA754B754E1A68E7
:1007EC00039312F4802F02BF734B01221A703378DB
:1007FC00724D43F004030020337001F0FFF8B5F89C
:10080C00EC000496002840F0C684B5F9EE30002BBD
:10081C0040F0C184B5F9F030002B40F0BC8495F861
:10082C00FB3000210593664B0C221B686548B3F81E
:10083C005630B5F8F470069395F8F380B5F80C9033
:10084C0095F80FA00CF05BF85F4B002118461422B2
:10085C0007930CF054F85D490022C4F850210A703B
:10086C0001F03BFC079B8346494E1C46002800F0D8
:10087C00B284574BB7F5807F2360564B6360564B61
:10088C00E360564B2361564B01D1002216E0BB2F7F
:10089C0001D9012212E0612F01D902220EE0292F89
:1008AC0001D903220AE0132F01D9042206E0092FF3
:1008BC0001D9052202E0002FE7D006221A70494B1D
:1008CC0001221A70484A136843F00103136043462F
:1008DC0046490022092B0A7001D90023F8E740F29F
:1008EC00B2324FF0010808FA03F10A40002A40F036
:1008FC00968011F04D0F00F092800793C6F85021AE
:10090C0001F0EBFB079B002800F0898006210A46CA
:10091C000DAB682001F03AFA9DF8391001EA080293
:10092C009DF8371001EA080101FA08F343EA820145
:10093C009DF8352002EA08030B430AD05BB243450D
:10094C0001D1002302E0022B0FD1012386F8543190
:10095C0050E00DF1230368200C21424601F016FAF9
:10096C009DF8233013F00F0303D1032003F09DF9FE
:10097C0040E0042BE9D1E4E7B91200083004002070
:10098C00991300082116000891120008E8100020A5
:10099C00B003002000127A00B913000840420F0087
:1009AC00A913000878070020E4020020D4D4000822
:1009BC00E80F002004170020A8030020000A0020E4
:1009CC00EC07002034010020A0160020DC000020E1
:1009DC002D1D0008572000083120000890C1793DDA
:1009EC000C0000202C00002084070020121700208F
:1009FC0054E500085D4B5E4A1A605E4A5A6096F8F0
:100A0C005421002A0CBF6F226E221A725A4B0322F9
:100A1C005A705A4A136843F00203136002E0012B28
:100A2C003FF65BAF554B1A68984612F0020F02D096
:100A3C004E4B1B689847FFB25149BAF1000F2AD0B0
:100A4C00D8F800304FB940F2596213F0020F40F25F
:100A5C00712318BF13467D2208E09A0759BF4FF443
:100A6C007A731A464FF4FA634FF47A72994505DBA0
:100A7C00B9F57A6FA8BF4FF47A6900E09946531E16
:100A8C004B44B3FBF2F3013BDBB203FB022286F8CF
:100A9C0055310A6003E086F855A1C1F80090394B36
:100AAC001B689847059F384A00231370924617B16C
:100ABC00022F40F06B834FF0000916AB03F8249D16
:100ACC001E200A210122C6F8589101F05FF9C0B12D
:100ADC009DF83430482B40F082832C4B2C4AD9465D
:100AEC001A602C4A5A60BBF1000F00F07883224B3D
:100AFC000222DA70D8F8003043F00803C8F800304E
:100B0C0001E081466BE395F8E8300BB1224A137093
:100B1C0095F8E9300BB1214A137095F8EA300BB116
:100B2C008AF80030D8F80030DFF87C8013F0080F1A
:100B3C003CD0BDF918B04FF064099BFBF9F738466F
:100B4C0008F036FA824609FB17B000B208F030FA0A
:100B5C00134908F081FA0146504608F075F911491D
:100B6C0008F07AFAC8F8000023E000BF3401002036
:100B7C00DD190008992000082C00002084070020B3
:100B8C00D8000020A016002013170020B800002069
:100B9C00911E0008151E0008DC0000201217002012
:100BAC008988883C00002041C01100200023C8F82F
:100BBC000030049B049A1B780A2743F0020313703D
:100BCC00029A4FF400535361029A4FF4804313611D
:100BDC00029B029ADB68192083F40053D360029BBA
:100BEC00029ADB68013F83F48043D36003F053F82F
:100BFC00192003F050F817F0FF07DFF83883E7D11E
:100C0C004FF480434FF40059AC4FC8F81030C8F87B
:100C1C0010903B681B0709D5A94BC8F814901B68AA
:100C2C009847A84B0122C8F810901A70A64BDFF811
:100C3C0008831B68187B08F0BBF9A44908F00CFA70
:100C4C00A34908F001F904F0F8F88146B8F800005F
:100C5C0008F0AEF9494608F0FFF90BF0AFFF9D4BD9
:100C6C001880B8F8000008F0A3F901469A4808F07B
:100C7C00A7FA9A4908F0A4FA9449C6F85C012069CD
:100C8C0008F0EAF9964908F0E7F9964C964BFF21E3
:100C9C0018601B2220460BF032FE204600222270E8
:100CAC003A68924B012112F0020F18BF6170197053
:100CBC001FBF032119700221A170540741BF19787D
:100CCC004C1C1C70032448BF445412F00A0F0CD067
:100CDC001A7804218154511CC9B205244454D11CE6
:100CEC0002321970D2B206218154039A126891060D
:100CFC0041BF19784C1C1C70072448BF44546979B7
:100D0C00082901D00E2904D119784C1C1C700B2415
:100D1C00445419780C274754570748BF734F01F1B7
:100D2C000104E4B248BF02311C7041BF39706D49F7
:100D3C0010270F55197812274C1CE4B2475457054D
:100D4C001C7008D595F88C712FB1684F0231397031
:100D5C00644913270F55970541BF19784C1C1C701B
:100D6C00152448BF4454D40548BF1A784FF00004EA
:100D7C0041BF511C19701A238354002198225C48DE
:100D8C000BF0BDFD012002F063FEB8B3012C35D889
:100D9C004FF04C0B0BFB04F9DFF854A10AEB090CD8
:100DAC000CF1480898F8027017B10134E4B2ECE782
:100DBC0090F9003090F804E018464E4B03228DE871
:100DCC00840001213A4653F82E30CDF814C002F0BD
:100DDC0065FC029070B1DDF814C0394660465A4685
:100DEC000BF08DFD029B4AF8093001231C4488F856
:100DFC000230E4B2012002F011FEC6E73E4A3F4B3E
:100E0C00B5F8E2101A603E4BB5F8280119803D493F
:100E1C0000230B808B703C490A6081B23B4A22F85C
:100E2C0013100133122BF9D1039B1B68D9045CBF3F
:100E3C00B5F82E1111801B0740F1008195F8223175
:100E4C00062B00F2F580DFE803F004070E7994B26C
:100E5C00B20045F2F05201E042F6F8222C4B1A8017
:100E6C0004F083FEE3E042F6F822294B1A8008F0E6
:100E7C009FF8284908F0F0F8274907F0E3FF08F03D
:100E8C00D7FA0023254A42F823000133122BF9D15B
:100E9C00234A244940201160234A137002F0D8FDE4
:100EAC00002800F0C58001234FF0070C90F90000DA
:100EBC0040218DE808101D4A1D4BB3E0840700202B
:100ECC00B8000020D00000207801002035FA8E3CBC
:100EDC00DB0FC93F940100200AE81C4100401C466E
:100EEC00BD37863591070020740100209007002043
:100EFC003C02002008D600081A0B002088060020AF
:100F0C008C060020F80F0020E40F00202C09002094
:100F1C00E4010020CDCCCC3F0000B044E40800201C
:100F2C0020000020595700081C0F0020D55900083C
:100F3C00A0860100001001401E00002042F6F8229D
:100F4C00AA4B40201A80AA4AAA4B1A60AA4B10221C
:100F5C001A7002F07DFD00286AD001234FF0000EBC
:100F6C0090F9000040218DE80840A44A4FF4E13389
:100F7C0058E042F6F8229D4B40201A80A04A9D4B27
:100F8C001A609D4B08221A7002F062FD00284FD0A7
:100F9C000123002790F9000040218DE88800994A30
:100FAC004FF4E13302F07AFBC6F860013CE042F604
:100FBC00F8218E4A062B11808F494FF00C02DFF876
:100FCC00B8C2DFF8B8E2904F904E914C91480A703D
:100FDC000DD000238CF800308EF800303B701B23B2
:100FEC0033700523227003704FF4E1340AE00021C2
:100FFC008CF800108EF80010397022702121864C6C
:10100C0031700370854A7B4B40201A6002F020FD42
:10101C0070B10123002690F900008DE848002346AA
:10102C007F4A402102F03AFB003018BF012028B95A
:10103C00082004F069F87B4A6E4B1A60039B1A680F
:10104C006D4B12F4804F1FBF082119707648694907
:10105C0018BF086042F20101114099B144F62060BA
:10106C0062490880910441BF082119706F48614999
:10107C0048BF0860D20741BF0C221A706C495D4A08
:10108C0048BF11601A78043A5A7002F0DDFD694BC2
:10109C0018606B79052B02BF674B4FF4C8721A802E
:1010AC00664B4FF47A721A80654A137843F0080342
:1010BC001370644A137823F002031370039B1A68AD
:1010CC0040F6020313406BB15F4A604B1A60604BF1
:1010DC0003221A705F4B01221A705F4A002313809F
:1010EC005E4A13805E4B4FF400425A61AB68039A20
:1010FC0013605C4B01221A70049B049A1B7863F0FA
:10110C007F03137017B0BDE8F08F013B092B3FF63E
:10111C008DA9029A4FF400535361534ADFF860A132
:10112C001068314630605046039300F0A1FA082253
:10113C00CAF810203C2002F0AEFD029B1A46039B1D
:10114C00136197F823319B45BFF66AA9029B4FF4B4
:10115C0080411961029B4FF4004205911A610823EA
:10116C0004927820CAF81430039302F089FD029B94
:10117C000599049A5961029B78205A61039B0BF1E3
:10118C00010BCAF8103002F07BFDDAE7012F7FF675
:10119C00BAAC1F4687E4354B00221A7000B207F038
:1011AC0007FF334907F058FF0D90B5F9EE0007F033
:1011BC00FFFE2F4907F050FF0E90B5F9F00007F035
:1011CC00F7FE2B4907F048FF2A490F900DA803F0B2
:1011DC00A7FEFFF724BB012002F067FDE9E4012F15
:1011EC007FF691AC00278AF8009064E4E4010020BB
:1011FC0045570008200000201C0F0020295900082A
:10120C002D570008DD5800088C0900208E0900209D
:10121C00710800208F09002090D003005956000857
:10122C0009580008B957000889570008A957000841
:10123C0099570008C40100209A06002010170020BE
:10124C008E060020161700200C0B00204C0F0020DF
:10125C0000170020340000201C0200201E02002079
:10126C0000100140A803002014D50008280000201D
:10127C0035FA8E3C280F0020720800208D090020C2
:10128C000008014010F80A3C0133DBB20A2B84BF82
:10129C0010F8131C044A00F80A3C82BF002322F801
:1012AC00113000F80A3C704750090020334A70B5E1
:1012BC00136C9068194440F68C23081A984291607C
:1012CC00D060516013463BD9127893F94510104603
:1012DC008A420BD1111F082908D893F846101829F7
:1012EC0001D8013103E083F8442002E0002183F8A7
:1012FC00461093F944402149A24219D191F8474034
:10130C00B4B10C310024944206DA51F8046F1C4D30
:10131C0025F814600134F6E70C2805D01849002490
:10132C0021F810400130F7E71648017801310170BF
:10133C0083F84520002201211A7083F8471070BDF4
:10134C0092F84710C9B140F2DA51A0F2EF248C4266
:10135C0008D811780B2905D80B1D0131117042F8F2
:10136C00230070BD002283F84720074B03F13002A5
:10137C00002143F8041F9342FAD170BDD80300201A
:10138C0050090020AD000020E4030020024A136C39
:10139C000133194411647047D8030020024B53F8F1
:1013AC0020301B6819807047E8100020074BA1F50E
:1013BC007A7153F820301A681B8959434FF47A73A9
:1013CC0091FBF3F189B21180704700BFE810002047
:1013DC008F4A70B51368988A80B2C1B2CE072ED5E9
:1013EC00198821F400610904090C1980198889B243
:1013FC0041F48061198000211171517999B1917971
:10140C0011B9D179FF290ED101219171117A0229DB
:10141C0001BF198889B241F400611980517A41F0F9
:10142C0001011982DFE0517A01F0FE011982D379B2
:10143C00FF2B00F0D880764BFF211971D3E08D077C
:10144C003AD5BFF35F8F107AC0B2012813D151790E
:10145C0089B1917979B1198821F480610904090C59
:10146C001980BFF35F8F198B1988907289B241F480
:10147C00007119801BE0198BBFF35F8F107A6449E0
:10148C0002280AD1487940B1897931B1198821F4FF
:10149C0080610904090C19809FE0107A5C490328CB
:1014AC0005D1487918B18979002940F0968099883E
:1014BC0089B241F4806195E04C0754D501219172B9
:1014CC005179002936D09179002933D0117A1888B6
:1014DC00022911791CD920F480600004000C1880BA
:1014EC001C8AD568C8B2E4B249B26C54198889B266
:1014FC0041F400711980811C1171198A0130C9B233
:10150C0040B22954998889B241F48061998026E0CF
:10151C0080B240F4007018801C8AD568C8B2E4B25E
:10152C0049B26C541C8A411C49B2E4B203306C546D
:10153C00107114E09179364809B9017C41B11988D0
:10154C0089B241F40071198011790131117106E0F1
:10155C00198889B241F4807119800121817119882F
:10156C00C905FCD43FE001F0400101F0FF04E1B1FA
:10157C0010791E8AD568C4B2611C40B2F6B22E54E2
:10158C00C9B2157A117149B2C81C854201BF98883D
:10159C0020F480600004000C08BF9880137A8B4202
:1015AC0021D11B4B02341C711DE006061BD5117991
:1015BC0048B2451C0AD054690131205CC9B218826A
:1015CC00107A117149B288420DD106E0D1791471AB
:1015DC001982517909B9117A29B9998821F4806154
:1015EC000904090C9980117A92F90400013188429E
:1015FC00074B0CD100219971997A31B119688B88FC
:10160C0023F440731B041B0C8B800023137670BDDA
:10161C001405002038B510F80E2C044650F8043C84
:10162C005AB9012200F80E2C20F80C1C997A186873
:10163C000222BDE8384005F031BE30F80C2C20F801
:10164C000A1C891A89B220F8081C084A10F80F0CD9
:10165C00002522F8101004F80E5C1868997A2A46B6
:10166C0005F01CFE04F8065C38BD00BF50090020D4
:10167C00F0B5B1F800E000234EFA03F2D50725D5FA
:10168C008E784FEAD30CF40648BFCC7806F00F02E4
:10169C0003F0070748BF2243BF0050F82C500F241B
:1016AC00BC4025EA0404BA402243282E40F82C20E2
:1016BC0005D1C46801229A4024EA020205E0482EB2
:1016CC0004D1C46801229A402243C2600133102B1A
:1016DC00D2D1F0BD2DE9F7438E460546DFF898923E
:1016EC00114699F819400068164698467246631CD4
:1016FC0089F8193006F0CEF92B8901A9ADF8043020
:10170C0018238DF80630686802238DF80730FFF730
:10171C00AFFFAB7A09F11C07240127442A6849461C
:10172C000C2B00F2F680DFE813F00D00F400F4004F
:10173C00F4005100F400F400F4008A00F400F4000A
:10174C00F400C200138CDFF834C223F001031B0435
:10175C001B0C1384138CB2F804E0108B624520F040
:10176C0073004FEA00404FEA10409BB21FFA8EFE06
:10177C0040F0700014D00CF5006C624510D00CF5E4
:10178C00406C62450CD00CF5806C624508D00CF5B1
:10179C00806C624504D023F0020343F0030307E09E
:1017AC0023F00E032EF4407E43F003034EF4807EB0
:1017BC00A2F804E01083A2F834801384138B23F076
:1017CC0008031B041B0C43F0080336E0138CDFF8F2
:1017DC00ACC123F010031B041B0C1384138CB2F844
:1017EC0004E0108B624520F4E6404FEA00404FEADB
:1017FC0010409BB21FFA8EFE40F4E04008D00CF56E
:10180C00006C624504D023F0200343F0300307E062
:10181C0023F0E0032EF4406E43F030034EF4806E60
:10182C00A2F804E01083A2F838801384138B23F4FD
:10183C0000631B041B0C43F40063138369E0138CDB
:10184C00DFF838C123F480731B041B0C1384138C36
:10185C00B2F804E0908B624520F073004FEA004030
:10186C004FEA10409BB21FFA8EFE40F0700008D079
:10187C000CF5006C624504D023F4007343F4407300
:10188C0007E023F460632EF4405E43F440734EF49F
:10189C00805EA2F804E09083A2F83C801384938BC2
:1018AC0023F008031B041B0C43F0080330E0138CDB
:1018BC00DFF8C8C023F480531B041B0C1384108C5A
:1018CC00B2F804E0938B20F4005023F4E6431B049D
:1018DC0000041B0C000C62451FFA8EFE43F4E0431F
:1018EC0040F4405003D00CF5006C624503D12EF44B
:1018FC00804E4EF4804EA2F804E09383A2F8408010
:10190C001084938B23F400631B041B0C43F40063BF
:10191C0093832B7B43B1B2F844306FEA43436FEAB5
:10192C0053439BB2A2F8443013889BB243F001039B
:10193C001380AB7A0C2B18D8DFE803F007171717B6
:10194C000B1717170F17171713000B1902F1340089
:10195C000AE00B1902F1380006E00B1902F13C0009
:10196C0002E00B1902F14000D86138460C44A68401
:10197C00226203B0BDE8F08314050020002C014066
:10198C00104B13B593F8DC201C46CAB90E4B1B68E0
:10199C00B3B11A681AB10D49886902438A619A88F1
:1019AC009868ADF8042002228DF8072004220DEB74
:1019BC0002018DF80620FFF75BFE012384F8DC3072
:1019CC0002B010BD140500200005002000100240DC
:1019DC0008B5FFF7D5FF074B1B7813B1012B03D0CC
:1019EC0008BD4FF4006201E04FF48052024B1A80A4
:1019FC0008BD00BF040500201E000020012828BFE0
:101A0C0001202DE9F04F0646142000FB06F3704F21
:101A1C0089B0F918FC586F4B0A691C6083F8DD60BB
:101A2C006D4BB1F80880DD69B1F80AA02A43DA6180
:101A3C00A2884D6822F440721204120C4AEA08097A
:101A4C00A28003A9C5F8109002228DF80E0028463A
:101A5C000193ADF80C908DF80F20FFF709FE019B58
:101A6C0000971F464FF0080BAA6818EA020F03D123
:101A7C000A2002F005F9F7E70A20C5F8148002F0F5
:101A8C00FFF8C5F810800A2002F0FAF8BBF1010B40
:101A9C00EAD1C5F814A00A2002F0F2F8C5F81480B7
:101AAC000A2002F0EDF8C5F810800A2002F0E8F8E0
:101ABC000222C5F810A0284603A98DF80F201C227D
:101ACC008DF80E20ADF80C90FFF7D2FD434A03A819
:101ADC0094423A690BBF42F4001242F480023A611C
:101AEC003A610BBF3A693A6922F4001222F480027F
:101AFC003A61A38823F440731B041B0CA380238836
:101B0C009BB243F001032380A58804F0EBF8059900
:101B1C00334B25F03F05B1FBF3F32D042D0C1D4386
:101B2C00ADB2A5802288002522F001021204120C0D
:101B3C0022802C4A03A8B1FBF2F100298AB208BF1B
:101B4C00012242F400414FF4967253434FF47A72DF
:101B5C0093FBF2F301339BB22384A1832388009A75
:101B6C009BB243F001032380238823F4816323F089
:101B7C0002031B041B0C23804FF48043238114238A
:101B8C0003FB0626737B01248DF80C308DF80D5069
:101B9C008DF80E508DF80F4003F03EFF337B9DF80F
:101BAC000F208DF80C308DF80D508DF80E501AB1A9
:101BBC0003A803F031FF08E05A0903F01F039C400F
:101BCC0002F12003084A42F8234009B0BDE8F08F27
:101BDC0040D50008140500200010024000540040BD
:101BEC0040420F00804F120000E100E010B5214C84
:101BFC002368998A89B211F4706F1CBF012284F892
:101C0C00DE2011F4E06F2BD01A8B9A88890522F410
:101C1C0080624FEA02424FEA12429A8020D41A881C
:101C2C0092051DD41A88D0050FD51A88D105FCD47D
:101C3C001A8892B242F400721A801A889205FCD467
:101C4C0094F8DD00FFF7DAFE0AE01A8892B242F44B
:101C5C0000721A809A8822F440721204120C9A8034
:101C6C002268938A23F470631B041B0C9382002359
:101C7C00237610BD14050020064A08B513880133DD
:101C8C009BB21380044B93F8DD00FFF7B7FE0020E6
:101C9C0008BD00BF820700201405002013B51F4BA0
:101CAC004000C0B2587202AC1868D97104F8012D0A
:101CBC00002101221A745C615971DC601A721A7667
:101CCC0083F8DE1040B38288920515D40288D405BF
:101CDC000DD447F230520188890502D5013AFAD168
:101CEC0012E08AB1028892B242F480720280828839
:101CFC0092B242F44072828047F23052197E11B196
:101D0C00013AFBD100E012B9FFF7B6FF04E0034B38
:101D1C0093F8DE0080F0010002B010BD1405002025
:101D2C0008B5FFF72DFE6B2180226820FFF7B6FF68
:101D3C00642001F0B0FF6B2103226820FFF7AEFF97
:101D4C000F2001F0A8FF0F4B19211A786820FFF71C
:101D5C00A5FF0F2001F09FFF0B4B1A211A7868206A
:101D6C00FFF79CFF1B2118226820FFF797FF1C210F
:101D7C0010226820FFF792FFBDE808406820372149
:101D8C0000228BE7050500200C00002010B5400058
:101D9C001C4CC0B26072E171012000212174607191
:101DAC00227220762068E360636184F8DE1040B311
:101DBC0083889B0515D40388D9050DD447F230537D
:101DCC000288920502D5013BFAD112E08BB103884F
:101DDC009BB243F48073038083889BB243F44073BB
:101DEC00838047F23053227E12B1013BFBD100E0DD
:101DFC0013B9BDE810403FE7024B93F8DE0080F0CA
:101E0C00010010BD1405002037B5044603211E2027
:101E1C0006226B46FFF7BAFF78BB9DF801309DF8A0
:101E2C000000174D43EA002000B207F0C1F8296802
:101E3C0007F012F907F0D6FA9DF8033020809DF8D0
:101E4C00020043EA002000B207F0B2F8A96807F0DC
:101E5C0003F907F0C7FA9DF80530A0809DF804003F
:101E6C0043EA002000B207F0A3F8696807F0F4F821
:101E7C0007F0B8FA6080012000E0002003B030BD0C
:101E8C00100000202DE9FF41604B1B689BB11A68C4
:101E9C001AB15F49886902438A619A889868ADF8DB
:101EAC00042002228DF8072004220DEB02018DF88C
:101EBC000620FFF7DDFB322001F0EDFE00211122A0
:101ECC001E20FFF7EBFE012160221E20FFF7E6FE2D
:101EDC00642001F0E0FE002402A8FFF795FF2746DE
:101EEC0026460A25022101221E20FFF7D7FE3220AA
:101EFC0001F0D1FE02A8FFF787FFBDF90820BDF95C
:101F0C000A1014448A42A8BF0A46BDF90C300F448B
:101F1C0093421E44A8BF134613F5805F09DD3D4A6A
:101F2C00013DD36883F40053D360DBD14FF001083B
:101F3C0001E04FF000081E2000211222FFF7AEFE38
:101F4C000A25022101221E20FFF7A8FE322001F0F3
:101F5C00A2FE02A8FFF758FFBDF90820BDF90A1030
:101F6C00A41A8A42A8BF0A46BDF90C307F1A9342C4
:101F7C00A6EB0306A8BF134613F5805F07DD254AC1
:101F8C00013DD36883F40053D360DAD101E04FF004
:101F9C000008204607F00CF801461F4807F010F91E
:101FAC001E4D20F000402860384607F001F801462D
:101FBC00194807F005F920F000406860304606F03B
:101FCC00F7FF0146164807F0FBF820F00040A86028
:101FDC00002170221E20FFF761FE012120221E200D
:101FEC00FFF75CFE1E2002210022FFF757FE642043
:101FFC0001F051FEB8F1000F04D14FF07E532B606D
:10200C006B60AB6004B0BDE8F08100BF0805002038
:10201C00001002400010014000406F4610000020EC
:10202C0001C05E4613B501220DF107033A210446A7
:10203C006820FFF7ABFE052001F022FE9DF807306B
:10204C0003B10123237002B010BD13B50622044660
:10205C00432168206B46FFF799FEA8B19DF800203C
:10206C009DF80130012043EA022323809DF80220D1
:10207C009DF8033043EA022363809DF804209DF809
:10208C00053043EA0223A38002B010BD13B506222B
:10209C0004463B2168206B46FFF778FEA8B19DF8FB
:1020AC0000209DF80130012043EA022323809DF893
:1020BC0002209DF8033043EA022363809DF804203C
:1020CC009DF8053043EA0223A38002B010BDFFF750
:1020DC007FB98BE5FFF77CB988E507B5232001F0C4
:1020EC00DAFD6820752101220DF10703FFF74EFE82
:1020FC0028B19DF80700A0F168035842584103B07D
:10210C005DF804FB7C492DE9F04F0C687B4A04F523
:10211C009C43203313607A4B89B01868059110F4F6
:10212C00804F9046019307D104F082F820B998F8BB
:10213C000430013388F80430724B1E78BEB1724AF9
:10214C001268944240F2F680013E1E70F2E03B6849
:10215C00072C98BF195D6D4B88BF21461B686C48D6
:10216C009847032C0AD908EB4404E0800136684BED
:10217C00F4B21D78674FA542E9D81FE03A6804F124
:10218C000E0302EB83039988DA880028EBD04FF416
:10219C007A73401A5843531A90FBF3F040F6C90374
:1021AC0000F57A70984205DC40F2EE239842B8BFF5
:1021BC00184601E040F6CA0080B2D4E798F80460F3
:1021CC000324B6FBF4F40F2388F82A3098F82C304B
:1021DC0004EB440403933B68341B029398F82BA044
:1021EC00E3B2DFF84CB104930024AC4251DA4A4B11
:1021FC00670033F81490BAF1000F09D104F018F805
:10220C0028B1039B002B08BF4FF0000900E0D1461A
:10221C00029B988A484502D8D88A48450ED2E0B22B
:10222C0003F0B4FF032C8146DFBF98F82AE00120AD
:10223C00A0402EEA0000D8BF88F82A0003F0F8FF6F
:10224C0018B1364827F800901FE0049B98F87600E8
:10225C002BF8139028B9022E14D9284B012083F89F
:10226C007600BBF80000BBF802300344BBF8040056
:10227C0003442B489BB23B521BB2032093FBF0F35D
:10228C009BB200E04B4625483B5201340BF1060B48
:10229C00ABE798F82A202348A2F10F077A427A413B
:1022AC0088F89020204B6AB1204A1268560109D454
:1022BC000268D9689A60521AC82A3BD9012283F85D
:1022CC00212037E002689868DA605B68121A9A423B
:1022DC0088BF154B4FF0000188F82B1088BF83F88E
:1022EC0021100024AC4225DAE0B203F04FFF0B4B77
:1022FC0023F814000134F5E70C170020F405002036
:10230C00E80F0020F00F0020EC0F00202000002030
:10231C001C0F0020E40F0020FA0500202C090020DF
:10232C006C060020F40F0020F80F00208C07002012
:10233C0022060020019B1B68DC0405D5884B1B681A
:10234C00D80701D406F052FD864B1A68937AFBB17C
:10235C008549013B31F81300137B1BB1C0F53B6081
:10236C00083080B200B2A0F57A70B0F57A7FA8BFC1
:10237C004FF47A7020EAE07006F01AFE7B4906F002
:10238C001FFF7B4906F068FE07F052F8794B188066
:10239C00019B794C1B6813F4807F00F00281059B34
:1023AC00DFF8DCA11A68754B9A4205D99AF802300D
:1023BC0013B901238AF802309AF80230002B00F08E
:1023CC00F0806F4B267893F82150654B691E4D4277
:1023DC004D411F68002DC6F38006C7F3806702933A
:1023EC0014BF4FF000094FF003099AF82030052B69
:1023FC0000F2D180DFE803F0034B5073829F002E74
:10240C0039D0D8F89400B8F8981001F0AFFB012837
:10241C0009D15C4A5C4B12681B68D288642101FBB1
:10242C000233CAF810306FB1564B1B681B794BB195
:10243C0006F0C2F803238AF820304FF47A73CAF8F6
:10244C001C30D2E7002D40F0A6804F4BDFF830B1A6
:10245C001A68DAF810309A4209D906F0ADF803235D
:10246C008BF8203040F6B833CBF81C30BDE7012395
:10247C008BF82030B9E74FF4806017B102F034FECE
:10248C0001E002F020FE0023CAF8103083E0002D9A
:10249C0046D106F091F8A8E725B105238AF820303B
:1024AC00012100E0294666B1D8F894304FF00209BA
:1024BC00DA892D4B1A805A809A80324A12685288D7
:1024CC00DA80314B1A68DAF814309A4201D8002EAF
:1024DC005ED147F23053CAF81C30032321E0237835
:1024EC0043F00203237006F081FC274BDAF81C2022
:1024FC001B681344CAF81830042312E0224B9DB118
:10250C001A68DAF818309A4245D9204B1B781BB957
:10251C00029B1B68DA073ED4237823F00203237056
:10252C0005238AF8203060E71B68DAF81C20134476
:10253C00CAF818302FE0134A134B12681B68D28864
:10254C00642101FB02334FF48060CAF81030002381
:10255C008AF820308AF8033002F0B5FD45E700BF59
:10256C008C070020E40F00202C09002000007A4486
:10257C0000C07F44E007002016170020404B4C00A1
:10258C00F80F0020D8160020F40F00201C000020AB
:10259C0000297FF42AAFB9F1000F02D0484601F0B0
:1025AC0011FB9E4D05F58D70B5F8E21001F0DEFAC9
:1025BC00AA46814668B905F0F1FF994B0022C3F891
:1025CC000090C3F80490C3F80890964B1A605A60B8
:1025DC009A6023785B073AD5019B1B68DF0636D5DA
:1025EC0098F89A30904DDE0631D4904B1B7843B35B
:1025FC009AF87231B9F1000F11D15BB18C4B1A689A
:10260C00D5F89C309B1A002B04DA06F0EFFB85F80A
:10261C00A0901CE0102001F0D5FA01230EE03BB194
:10262C00834A4FF47A71126801FB0323C5F89C307E
:10263C0098F8A0305BB101F0B3FA002388F8A03011
:10264C0005E0B9F1000FE5D095F8A030F2E70022D3
:10265C0016469AF870719AF87111BAF82A51BAF8AC
:10266C002CE1744BB60833F912000293A842C4BF94
:10267C0066F07F03DEB201327045B8BF46F040060B
:10268C00042AEED198F8A1206748B24205D190F8FF
:10269C00A220F92A04D8013200E0002280F8A220FE
:1026AC00624A88F8A16092F800B0634D0392BBF1C6
:1026BC00000F1CD12A68D00708D5B9F1000F16D12C
:1026CC002278D10713D506F05BFB10E02278520775
:1026DC000DD5554A92F82B204AB1584AD27832B9C6
:1026EC0011B106F083FB02E0B9F1000FF9D098F8B4
:1026FC00A220DFF85891142A63D1003718BF0127A4
:10270C00BBF1000F13D05F2E02D087B17D2E0ED1FE
:10271C00227802F0040202F0FF0B12B106F066FB05
:10272C0005E00B2001F04EFA3F4B83F8A2B0227863
:10273C0002F0040202F0FF01002A42D1572E0BD105
:10274C003F4B4FF47A721A803E4B1B6813F0080310
:10275C0037D13D4A138034E0019B1A68530718D5D2
:10276C005A2E16D198F8A3302F4A2BB1012382F898
:10277C00A31082F8A43024E092F8A53083F0010372
:10278C0082F8A5300BB10C2000E00D2001F01AFAF4
:10279C0017E05D2E00F0F6835B2E00F0F5835E2EC5
:1027AC0001D10320F1E3562E01D102F031FF039B3E
:1027BC001A78002A00F0F9836F2E40F0F28306F0AD
:1027CC00DFFA019B1B68580751D598F8A530164ABB
:1027DC0093B1237859070FD5029BB3F90610BAF8B9
:1027EC002A31994208DD2B6813F0010302BF322114
:1027FC00A2F8A81082F8A5302B68DA0328D598F82F
:10280C00AA20094B2AB993F8A32012B93222A3F8B3
:10281C00A820012388F8AA3029E000BF000A002074
:10282C0050100020CC100020F40500201C000020CB
:10283C00F40F00202C0900208C070020F80F00203A
:10284C001017002084070020DA070020EC07002076
:10285C0098F8A330A54A53B1237803F0040303F08E
:10286C00FF0123B9012382F8A31082F8A430D9F810
:10287C00006000232B6006F17B0406F1CB07227865
:10288C00637814F8010C9A420BD2214601F04AF9F4
:10289C0038B114F8022C012303FA02F22B6813430B
:1028AC002B600434BC42EAD1914B1B7843B1914C60
:1028BC00914E2368914D13F0020F40F0F682EDE239
:1028CC0006F1CA0406F589762278637814F8010CAF
:1028DC009A4223D2214601F025F9F8B1A378884A0F
:1028EC00013B03EB4303257913440C2202FB0582C5
:1028FC00D2F8B01094F803E099427C480ED0C2F89C
:10290C00B0300023C2F8B43082F8ACE0012390F868
:10291C00DC20AB4022EA030380F8DC300634B442FE
:10292C00D2D1784A784B12681C68029298F82B2006
:10293C00764F0392002604933A68002A00F0A7828F
:10294C001578002D00F0A3827B680299CB1A002B1E
:10295C000ADB01F5FA737B6098F8DC100123B340B5
:10296C0021EA030388F8DC30039B002B00F08F82F4
:10297C0017F8043C51780433DBB2002940F04C8248
:10298C00634931F91310BAF8283103F1C8008142B8
:10299C0002DD92F802B014E0C83B994204DA92F8D6
:1029AC0002B0CBF1000B0CE098F8DC200123B34013
:1029BC0022EA030388F8DC30029B03F5FA737B6090
:1029CC0065E298F8DC303341DB0700F16082BBF143
:1029DC00000FCCBF0220012001F01AF96B1E434AF4
:1029EC00132B00F24D82DFE813F0140020002F00AF
:1029FC00400057005E00D3002F018B01B701E301AB
:102A0C004B0240004B005E00D3002F01A6000201D8
:102A1C005E0123789B44BBF1FA0FA8BF4FF0FA0B71
:102A2C002BEAEB7B84F800B00AE063789B44BBF1A3
:102A3C00640FA8BF4FF0640B2BEAEB7B84F801B05A
:102A4C00204601F055F81BE2E37820469B44BBF18D
:102A5C00640FA8BF4FF0640B2BEAEB7B84F803B038
:102A6C00D2F8E01000F0FCFF0AE263795B44642BBF
:102A7C00A8BF642323EAE3730D2D637100F0008279
:102A8C0023799B44BBF1640FA8BF4FF0640B2BEA76
:102A9C00EB7B84F804B0F3E1A3799B448BF3080B34
:102AAC0084F806B0ECE1D2F8E49099F80020022A00
:102ABC0034D1584606F07CFA164906F081FBD9F859
:102ACC00241006F0C1F90021059006F063FC40B912
:102ADC00059A1149104606F07BFC059A10B10E4A76
:102AEC0000E00022C9F8242022E000BFF4050020F9
:102AFC00151700208C070020840700208807002071
:102B0C0068D50008F40F0020E8070020A406002078
:102B1C002C090020000020410000C84299F8022036
:102B2C005A44C82AA8BFC82222EAE27289F80220B5
:102B3C000F2D00F0A581B44BD3F8E4502B78022B69
:102B4C001AD1584606F034FAB04906F039FB296A16
:102B5C0006F07AF90021834606F01CFC38B9584679
:102B6C00AB4906F035FC20B1DFF8A4B201E04FF020
:102B7C00000BC5F820B083E16B789B44BBF1C80F08
:102B8C00A8BF4FF0C80B2BEAEB7B85F801B077E1BF
:102B9C00D2F8E49099F80020022A1BD1584606F08E
:102BAC0007FA9B4906F00CFBD9F8301006F04CF9EB
:102BBC000021059006F0EEFB40B9059A94491046A9
:102BCC0006F006FC059A10B1914A00E00022C9F803
:102BDC00302009E099F80C205A44C82AA8BFC82212
:102BEC0022EAE27289F80C20102D00F04981864B04
:102BFC00D3F8E4502B78022B1AD1584606F0D8F9AA
:102C0C00834906F0DDFAE96A06F01EF900218346D5
:102C1C0006F0C0FB38B958467D4906F0D9FB20B107
:102C2C00DFF8ECB101E04FF0000BC5F82CB027E158
:102C3C00EB7A9B44BBF1C80FA8BF4FF0C80B2BEA33
:102C4C00EB7B85F80BB01BE1D2F8E49099F80020EF
:102C5C00022A1BD1584606F0ABF96E4906F0B0FAC1
:102C6C00D9F83C1006F0F0F80021059006F092FB24
:102C7C0040B9059A6649104606F0AAFB059A10B1B0
:102C8C00634A00E00022C9F83C2009E099F81620BC
:102C9C005A44C82AA8BFC82222EAE27289F8162030
:102CAC00112D00F0ED80584BD3F8E4502B78022B0B
:102CBC001AD1584606F07CF9564906F081FAA96BF0
:102CCC0006F0C2F80021834606F064FB38B958467A
:102CDC004F4906F07DFB20B1DFF834B101E04FF035
:102CEC00000BC5F838B0CBE06B7D9B44BBF1C80F33
:102CFC00A8BF4FF0C80B2BEAEB7B85F815B0BFE0F3
:102D0C00D2F8E4502B78022B1AD1584606F050F921
:102D1C003E4906F055FAA96A06F096F8002183465A
:102D2C0006F038FB38B95846394906F051FB20B14A
:102D3C00DFF8DCB001E04FF0000BC5F828B09FE0E5
:102D4C00EB789B44BBF1C80FA8BF4FF0C80B2BEA24
:102D5C00EB7B85F803B093E0D2F8E4502B78022B90
:102D6C001AD1584606F024F9294906F029FA696B5C
:102D7C0006F06AF80021834606F00CFB38B9584679
:102D8C00234906F025FB20B1DFF884B001E04FF0B9
:102D9C00000BC5F834B073E06B7B9B44BBF1C80FE0
:102DAC00A8BF4FF0C80B2BEAEB7B85F80DB067E0A2
:102DBC00D2F8E4502B78022B1AD1584606F0F8F8CA
:102DCC00144906F0FDF9296C06F03EF80021834603
:102DDC0006F0E0FA38B958460D4906F0F9FA20B178
:102DEC00DFF82CB001E04FF0000BC5F840B047E025
:102DFC00EB7D9B44BBF1C80FA8BF4FF0C80B2BEA6F
:102E0C00EB7B85F817B03BE0F40500200000204177
:102E1C000000C84200007A44012931D19078844ADC
:102E2C0032F913B0BBF5617F05DB40F633039B45EC
:102E3C00A8BF9B4601E04FF4617B0C2D20D14FF4D1
:102E4C00966393FBF0F0ABF5617B9BFBF0FB794A4F
:102E5C005FFA8BFB13785B4512D0BBF1040F34BFC8
:102E6C005B46022305FB03A51370049B05F2F24598
:102E7C001D6002F021FA0BF10100C0B200F0C8FE97
:102E8C0098F8DC200123B340134388F8DC3001367A
:102E9C00042E07F10C077FF44FAD08E5019B1B686E
:102EAC00D8050FD5644BDB7863B13368990709D526
:102EBC002B8813F001070AD105F070FB012002F0FA
:102ECC0013F904E0012002F0FEF8012300E00023D6
:102EDC00226852070CD55BB1012002F0F4F82B8864
:102EEC009B0708D405F05AFB022002F0FDF802E023
:102EFC00022002F0E8F82B88504A13F0030F4FF42D
:102F0C00005114BF51611161326812F00A0F23D0C5
:102F1C002268D70609D55E070AD4042002F0E4F82B
:102F2C00474B1B88A8F8E83002E0042002F0CBF8ED
:102F3C002368980606D52B88590606D4402002F043
:102F4C00D3F802E0402002F0BEF823685A0642BFD4
:102F5C003B4B1B88A8F8EA3023684FF480701B05A4
:102F6C0002D502F0C1F801E002F0ADF89AF8053094
:102F7C00082B01D00E2B58D1402009B0BDE8F04FE2
:102F8C0002F0A1B8012000E00220C7B27B1E8AF833
:102F9C00F03402F0EBF802F0B3F9384600F038FEEA
:102FAC000FE417B17E2E3FF40AAC972E04D14FF4E8
:102FBC00C873A8F8A63004E4A72E07D198F89A3065
:102FCC0043F0040388F89A30FFF7FBBB0022BB2EBA
:102FDC00079201D1022303E0B72E04D14FF6FE7302
:102FEC00ADF81E300AE0BE2E01D1022304E0BD2E46
:102FFC007FF4E7AB4FF6FE73ADF81C30D9F8003018
:10300C00BDF81C10B3F858200A44A3F85820BDF89A
:10301C001E10B3F85A200A44A3F85A2002F0F8FA0A
:10302C00002388F8A230FFF7CCBB09B0BDE8F08FC5
:10303C002C090020DC160020F80F002000100140A5
:10304C00DA07002070472DE9F047054609F09BFC94
:10305C00314E0446D6F8088090B9304805F002FC91
:10306C002F4B53F8241049B10123A34013EA080F46
:10307C0002D02C4801F0D2FD0134F1E72A4822E0BD
:10308C0028462A49224609F087FC58B9284805F0F9
:10309C00E9FB284C54F8041F0029EFD0214801F01B
:1030AC00BDFDF7E72B784FF000092D2B03BF013541
:1030BC0004F1FF344FF0010A4FF0000A184B53F89B
:1030CC00297027B91C48BDE8F04705F0CBBB284652
:1030DC003946224609F060FCD8B9012000FA09F003
:1030EC00020601D51548EEE78305FBD4BAF1000FB3
:1030FC0003D002F009F8124803E040EA0800B0607F
:10310C00104805F0AFFB3946BDE8F0470E4801F01A
:10311C0085BD09F10109D1E7000A002034E6000859
:10312C00A4D500083EE6000879EB000842E600084A
:10313C0047E60008A0D5000853E6000862E6000840
:10314C0070E6000879E60008D6E7000810B50848D4
:10315C0005F088FB074B00241C701C63064B1C708D
:10316C0003F02AFE05F0D4FD044B1C6010BD00BF1B
:10317C0081E60008E006002015170020FC16002050
:10318C0070B5064600240B4BE518AA8816420AD0E7
:10319C00E158094801F042FD2846002105F0FBFAF0
:1031AC00064805F05FFB40F6C82314349C42EAD174
:1031BC0070BD00BFCCD80008ADE6000879EB000864
:1031CC00F8B504460E46174600252046202109F086
:1031DC00CCFB0446D0B10134204609F029FCB0F5F3
:1031EC00617F05DB40F634039842A8BF184601E026
:1031FC004FF46170A0F56170192390FBF3F00DB9D9
:10320C00307000E070703B7801333B700DB90125D4
:10321C00DBE72046F8BD7FB504780646E4B9364BAB
:10322C001921186800EB840090F87B5090F87920F5
:10323C004D4305F5617590F87A30009590F87C0057
:10324C00414301F5617101912C482146013401F093
:10325C00E5FC142CE3D14CE009F0EAFB13280546FD
:10326C0041DC254B701C1C68202100238DF80F308D
:10327C0009F07BFB1E35064670B10136304609F06D
:10328C00D7FB1A289FBF04EB850358709DF80F30AD
:10329C00013398BF8DF80F303046202109F065FBC3
:1032AC00064670B10136304609F0C2FB0D289FBFAF
:1032BC0004EB850398709DF80F30013398BF8DF89F
:1032CC000F3004EB85043046E11C0DF10F02FFF7C3
:1032DC0077FF9DF80F30042B0BD0601C00210422CB
:1032EC0009F00DFB05E0064806490022132301F006
:1032FC0095FC04B070BD00BFEC070020B7E60008D9
:10330C00CCE60008EBE60008014805F0ABBA00BFBC
:10331C00F1E600082DE9F041047806467CB9334DFE
:10332C002146B5F85621B5F858313148013401F031
:10333C0075FC042C05F10405F2D1BDE8F0812D4992
:10334C0009F0E6FAB0B9294B4FF47A714FF4FA62EE
:10335C00A3F85611A3F85821A3F85A11A3F85C212D
:10336C00A3F85E11A3F86021A3F86211A3F86421FD
:10337C00BDE8F081304609F05BFB032805462CD8EC
:10338C003046202109F0F1FA044630B101342046D0
:10339C0009F04EFB0126074600E006462046202198
:1033AC0009F0E3FA10B9BDE8F041ADE7013009F0DE
:1033BC003FFB012EF7D140F2DC53A7F2EE229A42EA
:1033CC00F1D8A0F2EE229A42EDD8084B543503EB1B
:1033DC008503DF801881BDE8F0810748074900228A
:1033EC000323BDE8F04101F019BC00BF000A002026
:1033FC00FFE6000812E70008CCE600086AEE0008B9
:10340C00F0B5047887B0064614BB514B19201968E7
:10341C00062303FB041191F8CA5091F8CE204543C2
:10342C0005F5617591F8C930009591F8CB50C8310C
:10343C00684300F56170019008790290497945481C
:10344C0003912146013401F0E9FB0C2CDDD17DE028
:10345C0009F0EEFA0B28044672DC3D4B701C1D681B
:10346C00202100238DF8173009F07FFA064680B131
:10347C000136304609F0DCFA03289FBF062303FB14
:10348C00045383F8CE009DF817309CBF01338DF8A0
:10349C0017303046202109F068FA074680B1013711
:1034AC00384609F0C5FA0D289FBF062303FB0453C9
:1034BC0083F8C9009DF817309CBF01338DF8173085
:1034CC0006266643A9193846CA310DF11702FFF7D3
:1034DC0077FE202109F049FA074670B101373846CA
:1034EC0009F0A6FA14289FBF9DF8173076190133FE
:1034FC0086F8CC0098BF8DF817303846202109F09B
:10350C0034FA78B1013009F093FA0D289FBF0623E5
:10351C0003FB045383F8CD009DF817309CBF013397
:10352C008DF817309DF81730062B0FD0062202FBB2
:10353C0004500021C93009F0E2F9FFF7E5FE05E07F
:10354C000548064900220B2301F068FB07B0F0BDCB
:10355C00EC07002018E70008CCE60008EBE60008B2
:10356C002DE9F347047807464CB9204601A902F02F
:10357C00EBFA0134FFF7F4FF122CF6D17EE009F0E0
:10358C0057FAC5B2112D73D83E4C05F1980604EBD1
:10359C004603781C202193F8028009F0E6F93A4F93
:1035AC00034630B9A8F10202D2F1000848EB020838
:1035BC0048E007F1580800F1010A5978404609F033
:1035CC00D4F968B1032D8CBF03230023C8EB000092
:1035DC00C0B23B44184490F85C90B9F1030F02D18F
:1035EC00FFF792FE4AE0A9F10203D3F1000850461E
:1035FC004FF0200148EB030809F0B7F9D8B1B8F146
:10360C00000FEDD0013009F013FA40F2ED2380B237
:10361C00984205DD40F6CA039842A8BF184601E05F
:10362C0040F2EE20A0F2EE20192290FBF2F004EB17
:10363C004603D87002E0B8F1000FD1D104EB460379
:10364C0083F8029004EB4604A3781F4497F85820A3
:10365C00B8F1000F07D0E17819234B430B482946EA
:10366C0003F2EE2308E02946094801F0D7FA05E0F9
:10367C00084809490022112301F0D0FA02B0BDE834
:10368C00F08700BF000A0020A4D5000838E7000826
:10369C004AE70008CCE600086AEE0008F7B50546D4
:1036AC00124C0E4694F900001146A8421A469DF899
:1036BC0024709DF8203004D094F90C00A84211D14C
:1036CC000C34207A70B925B1012D0CD10097084823
:1036DC0001E00848009703F0ADFC20B1057126729B
:1036EC00606000E0002003B0F0BD00BFF4070020D4
:1036FC000044004000380140074B5B6B93F90220FB
:10370C00824201D1981C704793F90A2082420CBF67
:10371C0003F10A0000207047E0060020F0B50278A3
:10372C0087B08AB94B4C04F110064B4B94F97C11C1
:10373C0093F900208A426DD093F90C308B4269D0FA
:10374C000834B442F1D183E0002204920592451C66
:10375C0009F06EF9C4B260B2FFF7CEFF074618B19C
:10376C008DF81040012400E004462846202109F081
:10377C00FCF8054638B10135284609F059F90134F1
:10378C00ADF81200E4B200262846202109F0EDF82D
:10379C00A8B3451C284609F04BF900222F49D3B297
:1037AC0051F82210814203D00132082AF6D10023AD
:1037BC002B4A02EB8302526E824220D1022E0FD092
:1037CC00032E12D05A1E012ED2B204D0042A13D8C2
:1037DC008DF814300EE0042A0ED88DF8153009E05F
:1037EC00052B09D88DF8173004E09A1E052A03D84A
:1037FC008DF816300134E4B20136042EC4D1052CF8
:10380C0003D807B0BDE8F0407EE504AB03CB3860CD
:10381C0079601DE094F88101114B94F8805103EB11
:10382C008000406EB4F87E21009094F8830103EB85
:10383C00850503EB8000406E019094F8820103EB48
:10384C0080035B6E074802936B6E01F0E7F977E734
:10385C0007B0F0BD000A0020F407002008D60008CD
:10386C00A4D5000859E700082DE9FF415149044649
:10387C0009F04EF85049002820460CBF01260726B7
:10388C0009F046F84D490028204608BF022609F0E9
:10389C003FF8002808BF0426F10752D5484804F029
:1038AC00E1FF002004F0A7FE464804F0DBFF464F82
:1038BC00464804F0D7FF464804F0D4FF454CD7F8EF
:1038CC00088054F8041F19B1434801F0A7F9F8E730
:1038DC000D46424B53F8254054B10123AB4013EA3B
:1038EC00080F03D03E48214601F098F90135F0E766
:1038FC003C4804F0B7FF21467B1893F81A3104AA10
:10390C001344394A8A5C0131082903F8102CF3D18D
:10391C000023694635488DF8083001F07FF93448AA
:10392C0004F0A0FF3348FFF7F9FE334801F076F9B5
:10393C004020FFF725FC314804F094FF2D48FFF799
:10394C000FFEB20720D52E4804F08CFF2D4804F052
:10395C0089FF284804F090FE2B4804F083FF25488B
:10396C00FFF759FC294804F07DFF2248FFF748FD7A
:10397C00274801F053F91F48FFF7CCFC1E4801F013
:10398C004DF98020FFF7FCFB73070FD5214804F09D
:10399C0069FF214804F066FF164804F047FE1648FC
:1039AC0001F03CF94FF48070FFF7EAFB04B0BDE87E
:1039BC00F08100BF78E700082DED00087FE70008D4
:1039CC0085E7000893E70008000A0020A5E7000837
:1039DC00B1E70008A0D50008C1E70008A4D500088D
:1039EC00CFE70008DCE7000870EA0008E8E7000809
:1039FC00F1E7000818E5000879EB000800E800087A
:103A0C000DE8000820E800082EE8000838E8000857
:103A1C0047E8000855E8000866E800080B4B30B58D
:103A2C001A465C6B93F8381001290BD80B464D1CC9
:103A3C0004EBC303E9B29D882842F5D082F8381014
:103A4C00981C30BD82F83810002030BDE0060020F4
:103A5C00024B002283F83820E0E700BFE00600208C
:103A6C002DE9F047877890F803C0BBB2C7F1640E1C
:103A7C0003EB83065C42C3F178001C4D5FFA8EFEAB
:103A8C007600CCF16408A4B280B2A3B20FFA83F929
:103A9C00B9F1000F04DC002B14BF3B46012300E0FE
:103AAC00734609FB09F25B4302FB0CF292FBF3F346
:103ABC00434403FB09F30A2293FBF2F333449BB216
:103ACC0025F8023FB1F800904A880A34C9EB020A83
:103ADC001AB202FB0AF24FF47A7392FBF3F3A4B21C
:103AEC004B4484422B80D0D1BDE8F08718070020CE
:103AFC0010B544780078002240F6C41102FB02F3A2
:103B0C00193B634303F6C4135343434393FBF1F351
:103B1C00034921F812300132072AEDD110BD00BF44
:103B2C0032070020104B043033F91000B0F5617FE0
:103B3C0005DB40F633039842A8BF184601E04FF46A
:103B4C0061700A7819235A4302F28332824208DAEE
:103B5C004A78534303F283338342B4BF00200120DD
:103B6C0070470020704700BF2C0900200A4B1B68CF
:103B7C0013F4805F094BB3F9063005D0C089421AA3
:103B8C00934207DD084400E0008A8342B4BF002062
:103B9C000120704701207047E80F00202C090020FD
:103BAC0010B5064B00241C7002F04EFB044B83F83E
:103BBC0060405C66A3F86840DC6610BD1C100020F9
:103BCC00E006002030B510B9BDE83040E8E700232E
:103BDC000D4CD90004F1840212F83350854203D005
:103BEC000133102BF4D130BD084B0A44D86E28B1E8
:103BFC00214491F8854041788C4204D2DA66002247
:103C0C00A3F868205A6630BDA4D50008E006002051
:103C1C0010B540001428A8BF142000230949022421
:103C2C0001F170029C5423441A441424834202F878
:103C3C00014CF3DB0B44FF2283F870200F20BDE80E
:103C4C001040BFE7E006002010B50A4A0A4B116885
:103C5C009B6800BF12689142F7D1084A4FF47A7002
:103C6C00D2F8884000FB04F2D31AB3FBF4F300FB48
:103C7C00013010BDF40F002010E000E0E006002041
:103C8C0038B50446FFF7E0FF0546FFF7DDFF401BA4
:103C9C00A042FAD338BD10B504462CB14FF47A705B
:103CAC00FFF7EEFF013CF8E710BD2DE9F843814624
:103CBC000B26013E32D01C4C4FF4005363614FF481
:103CCC008043236109F101074FF032080525E368B1
:103CDC00404683F40053E360E36883F48043E3607D
:103CEC00FFF7D9FFE368404683F40053E360E368D1
:103CFC0083F48043E360FFF7CEFF45B1013DE6D18D
:103D0C004FF4FA70FFF7C7FF4FF0FA08DFE7013FF7
:103D1C00DDD14FF47A70FFF7BEFFCAE7034A044BBC
:103D2C00DA60BDE8F88300BF001001400400FA051A
:103D3C0000ED00E0024A136801331360704700BFC6
:103D4C00F40F0020024BD3F88C3003B118477047A6
:103D5C00E006002003681B69184703681B681847B6
:103D6C0008B50E4B1B6813F4805F0D4B14BFD3F8D2
:103D7C009020D3F8942093F8981092880023D8B20E
:103D8C00884204D2074820F813200133F7E702F0E9
:103D9C00BDFFBDE8084032207DE700BFE80F0020E2
:103DAC00E0060020BE07002010B5044680B204F0E7
:103DBC00E9FC200CBDE8104004F0E4BC38B5044626
:103DCC000D46242004F0CCFC4D2004F0C9FC002C42
:103DDC00094C14BF21203E2004F0C2FC23680022B1
:103DEC0028469A7104F0BCFC236893F84900BDE89E
:103DFC00384004F0B5BC00BF7C0700200146002011
:103E0C00DCE746282DE9F047044600F0918500F2E6
:103E1C0091802C2800F0DD844BD8052800F02681F9
:103E2C0029D8022800F009810ED8012840F09A8583
:103E3C000320FFF7E3FF002004F092FC204604F07F
:103E4C008FFC0D2000F012BD032800F00581042822
:103E5C0040F088850620FFF7D1FF432004F080FC5A
:103E6C004A2004F07DFC4D2004F07AFC312004F053
:103E7C0077FC00F05EBC262800F07A840CD822284F
:103E8C0000F07983242840F06D850420FFF7B6FFFD
:103E9C00D84B986800F061BD282800F087842A2848
:103EAC0040F060850120FFF7A9FFD24B587900F054
:103EBC00DDBC3A2800F006821AD8342800F07D8345
:103ECC000AD8322840F04E850120FFF797FFC94BE6
:103EDC0093F8240100F0CABC362800F00E8538286F
:103EEC0040F040850420FFF789FFC24C00F04FBC26
:103EFC00402800F0BE8411D83B2800F035833D28C3
:103F0C0040F03085BB4C0220FFF778FF94F872012B
:103F1C0004F026FC94F8710100F0A8BC422800F0D3
:103F2C00CB84452840F01E851320FFF767FF002443
:103F3C0000F008BD6E2800F0C98142D8652800F059
:103F4C00B28022D84B2800F0638408D8492840F06E
:103F5C0009850220FFF752FFA64B9889EAE34D280A
:103F6C0000F06584642840F0FD840720FFF746FFCD
:103F7C00E72004F0F5FB9F4B587904F0F1FB00208F
:103F8C0004F0EEFB042000F0E8BC692800F0788116
:103F9C000AD8662800F04281682840F0E38410209B
:103FAC00FFF72CFF002463E16C2800F07C816D2866
:103FBC0040F0D8840620FFF721FF0020FFF7F4FE25
:103FCC00B7E3752800F0C48215D8722800F06F830F
:103FDC0007D86F2800F0A681702800F0CD8100F082
:103FEC00C1BC732800F09A83742840F0BB844FF056
:103FFC00000801260EE3A02800F0AC830AD877282D
:10400C0000F035837B2840F0AD843C20FFF7F6FEB2
:10401C00002433E2F02800F09083FE2840F0A284C4
:10402C000820FFF7EBFE002004F0ACFB002004F0AE
:10403C00A9FB002004F0A6FB7BE30420FFF7DEFEC7
:10404C00432004F08DFB4C2004F08AFB462004F046
:10405C0087FB4C2000F00ABCFFF7D0FE012004F0D7
:10406C007FFB0A2004F07CFB0020FFE31A20FFF703
:10407C00C5FE0024604B185D013404F071FB0B2C61
:10408C00F8D100245D4B185D013404F069FB082C59
:10409C00F8D100245A4B185D013404F061FB072C55
:1040AC00F8D100F05CBC574C0B20FFF7A7FEA088A2
:1040BC0004F068FBE08880B204F064FBA368C3F3EF
:1040CC00C000C3F38002800040EA4200C3F3400208
:1040DC001043C3F3401240EAC20003F0100318432C
:1040EC0004F050FBA289236902F0080103F447593C
:1040FC0049EA010903F4804149EA010903F400414A
:10410C0049EA010903F4803149EA010903F4003159
:10411C0049EA010903F4802149EA010903F4002169
:10412C0049EA010903F4801149EA010903F000731B
:10413C0049EA0303DFF8D49012F0010F99F80090CC
:10414C0018BF4FF00208C9F3800908BF4FF00008F0
:10415C0043EA090312F0020F43EA080314BF4FF0BD
:10416C00040C4FF0000C12F0040F43EA0C0C14BFBB
:10417C004FF0100E4FF0000E12F0400F14BF20271E
:10418C0000274CEA0E0E12F0100F14BF4FF40076FD
:10419C0000264EEA070712F0200F14BF4FF480657B
:1041AC0000253E4312F4807F14BF4FF400600020C2
:1041BC00354312F4007F14BF4FF400110021284343
:1041CC0012F4806F41EA000114BF4FF080630023AA
:1041DC00002019430346247DA34219D20A4A9D5C50
:1041EC00012202FA05F50D421CBF9A40104301331F
:1041FC00F2E700BF000A002047E9000853E9000875
:10420C005CE900087C0700209107002016170020AD
:10421C00FFF7CAFDBB4B93F8F00427E31220FFF71E
:10422C00EDFDB94B00251B88B3F5806F8CBF0826BC
:10423C000126B64C04F1300333F91500013590FB1F
:10424C00F6F080B204F09EFA032DF2D1E08E04F069
:10425C0099FA208F04F096FA608F04F093FAA08FED
:10426C0004F090FAE08F04F08DFAB4F8400061E2AB
:10427C00A74B185D013404F073FA102CF8D16EE3DF
:10428C00A44D00242878400000F0FE00FFF7B6FD96
:10429C002B789C4280F063839F4B33F8140004F01E
:1042AC0071FA0134F4E7994C0620FFF7A7FDB4F836
:1042BC005A0004F067FAB4F85C0004F063FAB4F83E
:1042CC005E0037E20420FFF799FD45E34FF6FF75DA
:1042DC000720FFF793FD914B8C4C1888FF28A8BF43
:1042EC00FF20C0B204F03CFA206EA842A8BF2846BA
:1042FC0020EAE07080B204F045FAB4F8640004F0EF
:10430C0041FA804BA06E93F817313BB10A23584306
:10431C00A842A8BF284620EAE07001E000F30F0095
:10432C0080B207E2794C0B20FFF768FDE36E25465F
:10433C00187804F015FAE36E0026587804F010FA99
:10434C00EB6E724C33441879013604F009FA032EE3
:10435C00F6D1E36ED87904F003FAE36E987804F0A2
:10436C00FFF9E36ED87804F0FBF9E36E588904F09A
:10437C0009FAE36E187A79E2644C1E20FFF73EFDD1
:10438C00236F00251B78022B65D1236F05F10802E2
:10439C0053F82200624904F05FFE08F00FFC80F332
:1043AC000800C0B204F0DCF9236F5E4903EB85030F
:1043BC00D86A04F051FE08F001FC80F30800C0B28A
:1043CC0004F0CEF9236F05F10E0253F82200564982
:1043DC0004F042FE08F0F2FB80F30800C0B2013595
:1043EC0004F0BEF9032DD0D1072D236F21D1586CC9
:1043FC004B4904F031FE08F0E1FB80F30800C0B239
:10440C0004F0AEF9236F4649986C04F025FE08F0D1
:10441C00D5FB80F30800C0B204F0A2F9236F93F827
:10442C004C0004F0C1FD08F0C9FB80F30800C0B2D9
:10443C000BE02B44587804F093F9236F2B44D87A73
:10444C0004F08EF9236F2B44587D013504F088F964
:10445C000A2DC9D183E2236F2B44587804F080F9DC
:10446C00236F2B44D87A04F07BF9236F2B44587DAF
:10447C00013504F075F90A2DEDD170E2234D04F1EC
:10448C0008022B6F284953F8220004F0E5FD08F0D0
:10449C0095FB80B204F076F92B6F234903EB840370
:1044AC00D86A04F0D9FD08F089FB80B204F06AF9EF
:1044BC002B6F04F10E0253F822001B4904F0CCFDC3
:1044CC0008F07CFB013480B204F05CF9032CD5D1EC
:1044DC00072C2B6F2AD1586C134904F0BDFD08F042
:1044EC006DFB80B204F04EF92B6F0F49986C04F001
:1044FC00B3FD08F063FB80B204F044F92B6F93F822
:10450C004C001FE0000A00201E0000207C07002049
:10451C00BE0700201C0F00202C090020E00F0020FB
:10452C00000020410000C84200007A44234458781F
:10453C0004F028F92B6F2344D87A04F023F92B6F5D
:10454C002344587D013404F01DF90A2CC0D106E235
:10455C002F20FFF753FCCE4C14F8010F002800F06D
:10456C00FE8104F0FDF8F7E70120FFF747FCC94B8B
:10457C001B6F18787AE15020FFF740FC0025C54BE3
:10458C000C211C6FC44B04EB850494F87920013585
:10459C0001FB023393F8380004F0E2F894F87A0047
:1045AC0004F0DEF894F87B0004F0DAF894F87C0060
:1045BC0004F0D6F8142DE2D1D1E14820FFF71EFC0F
:1045CC000025B44B1C6F062303FB054494F8CE0066
:1045DC0004F0C6F894F8C90004F0C2F894F8CA00C4
:1045EC0004F0BEF894F8CB0004F0BAF894F8CC00C0
:1045FC0004F0B6F8013594F8CD0004F0B1F80C2DA8
:10460C00DFD1ACE1002E00F0AA815FFA88F0FFF751
:10461C00F5FB002600279F4B1A7D9742F2DA1533E3
:10462C00FA5C00240C2363439B4D05F13001595C6B
:10463C00914207D12B44586B08F0A5F982462EB94C
:10464C00B14605E001341C2CECD10EE080440CE0AA
:10465C00D1450ADA0C2303FB04535B6B13F80900F6
:10466C0004F07EF809F10109F2E70137D3E7894D2F
:10467C000024287DFFF7C2FB2B7D9C4280F06F81CC
:10468C00864B0021E65C0C2202FB01F3824800F110
:10469C003007DA5DB24205D1034493F8380004F0D8
:1046AC005FF802E001311C29EDD10134E4E77C4CC8
:1046BC001620FFF7A3FBB4F8280104F063F8B4F854
:1046CC00D40004F05FF8B4F8D60004F05BF8B4F84A
:1046DC00D80004F057F8B4F86A0104F053F800203D
:1046EC0004F03EF8002004F03BF8002004F038F809
:1046FC0094F8170104F034F894F8240104F030F81D
:10470C00002004F02DF8634B0A201B6FB3F95630D0
:10471C0093FBF0F080B204F035F838E00820FFF796
:10472C006DFB0124E0B2013404F01AF8092CF9D124
:10473C0015E1002004F026F811E1564C0420FFF797
:10474C005DFB236FB3F85A0004F01CF8236FB3F829
:10475C005800EFE70C20FFF751FB524B1868FFF79E
:10476C0023FB514B1868FFF71FFB504B1868F4E004
:10477C004B4C0620FFF742FBB4F8EC0004F002F8B7
:10478C00B4F8EE0003F0FEFFB4F8F000D2E794F8B2
:10479C000C0103F0E5FF94F8100103F0E1FF94F82D
:1047AC000F0103F0DDFF94F811015FE03C4C072092
:1047BC00FFF724FBB4F8120103F0E4FFB4F8140182
:1047CC0003F0E0FF94F8160103F0CAFFB4F81801E7
:1047DC00B0E7334C0C20FFF711FB94F8220103F0E7
:1047EC00BFFFB4F82C0103F0CDFFB4F8280103F09F
:1047FC00C9FFB4F82A0103F0C5FF94F8230103F0B4
:10480C00AFFFB4F82E0103F0BDFFB4F8300191E70F
:10481C00234C0420FFF7F2FA94F8680103F0A0FF90
:10482C0094F8690103F09CFFB4F86A0182E7204C0C
:10483C00204D2078002600EB4000C0B2FFF7DEFAD6
:10484C00237802359E4280F08A8015F8020C03F022
:10485C0087FF15F8010C013600EB800000EB80009F
:10486C0000F2EE2080B203F08DFFE9E703F078FF51
:10487C0075E00820FFF7C2FA0024094B234493F893
:10488C001A01013403F06CFF082CF6D167E000BF6D
:10489C0003D700087C07002004D7000891070020EC
:1048AC00000A0020E8F7FF1FECF7FF1FF0F7FF1FCF
:1048BC001C0F0020320B0020374C1020FFF79EFA03
:1048CC00607903F04DFFA068FFF76EFA94F82201AF
:1048DC0003F046FFB4F8EC0003F054FFB4F8EE001C
:1048EC0003F050FFB4F8F00003F04CFFB4F81201E1
:1048FC0003F048FFB4F814011CE7284D264C95F83A
:10490C00740004F11006C0EBC000C0B2FFF776FAD9
:10491C0094F87C0195F9782043B29A4225D01F4A2D
:10492C0092F984209A4220D00834B44217D0EFE791
:10493C000D20FFF763FA002003F012FF0020FFF7B1
:10494C0033FA06E0164B185D013403F009FF0B2C0B
:10495C00F8D10020FFF728FA0020FFF725FA0120F4
:10496C00BDE8F0870020BDE8F08703F0F9FEB4F84D
:10497C007E0103F007FF94F8800103F0F1FE94F838
:10498C00810103F0EDFE94F8830103F0E9FE94F845
:10499C00820103F0E5FEC7E7000A00207C07002037
:1049AC0047E90008034B1A68D379591C1344D17199
:1049BC00187A70477C07002010B5FFF7F3FF84B21C
:1049CC00FFF7F0FF04EB002080B210BDF0B501241E
:1049DC00B0FBF4F58D4201D34C43F9E70026D4B17A
:1049EC00B0FBF4F504FB1500B4FBF1F41EB9002D7B
:1049FC0001DC002CF3D1092D03F1010EEFB204DD23
:104A0C00002A14BF3725572500E030253D441D7082
:104A1C0001367346E3E71C70F0BDF0B50124B0FB22
:104A2C00F4F58D4201D34C43F9E70026D4B1B0FB29
:104A3C00F4F504FB1500B4FBF1F41EB9002D01DCF8
:104A4C00002CF3D1092D03F1010EEFB204DD002A85
:104A5C0014BF3725572500E030253D441D70013625
:104A6C007346E3E71C70F0BD2DE9F843089E002B5C
:104A7C00074688461446334614BF4FF030094FF0B2
:104A8C00200913F8012B0AB9254603E0002CFBDDA5
:104A9C00013CF6E7002D04DD38464946C047013D90
:104AAC00F8E7354624EAE474A01B284415F8011BEA
:104ABC0011B13846C047F7E7BDE8F883014B1868D9
:104ACC00FFF74BB9D4020020F8B507460C464868EE
:104ADC00002115461E4604F053FC58B1284604F03C
:104AEC0067FA104904F0B8FA01464FF07E5004F012
:104AFC0067FB60606168304604F0A6F901463046F9
:104B0C0004F05EFB256806462946384604F09AF9FF
:104B1C000146304604F0A0FA0146284604F094F908
:104B2C002060F8BDDB0FC94030B5054687B00C4698
:104B3C0003A800210C2207F0E2FE2846002104F015
:104B4C0047FC20B12846284904F07EF903E02846AA
:104B5C00254904F077F9254904F07EFA04F042FC6B
:104B6C00054680EAE0706946A0EBE57000F0ECFFCA
:104B7C00002DACBF20232D2368468DF80C3007F098
:104B8C0002FF012807D130238DF80D308DF80E303F
:104B9C008DF80F300CE0022805D130238DF80D3044
:104BAC008DF80E3004E0032804BF30238DF80D304F
:104BBC00694603A807F0CAFE03A807F0E4FE033811
:104BCC00C5B22A4603A9204607F008FF0023635507
:104BDC002046074907F0BAFE03AB2046591907F0E7
:104BEC00B5FE204607B030BD6F12033A00007A4480
:104BFC0049EA000870B50646B6FBF2F408461546BD
:104C0C0014B12046FFF7F6FF05FB1464024B1B5D45
:104C1C0000F8013B70BD00BF4BEA00080FB42DE952
:104C2C00F04F7B4B89B012ACD3F80080794B54F821
:104C3C00046BD3F80090049400253178002900F01F
:104C4C008580252902D00136404673E072784FF0FA
:104C5C00000A302A0CBFB278B71CA2F1300312BF85
:104C6C004FF0000BF71C4FF0010B092B19D8A2F1D8
:104C7C003003D9B2092905D80A2202FB0A3A17F8DF
:104C8C00012BF4E7A2F16103052B02D8A2F1570323
:104C9C0005E0A2F14103052B03D8A2F137030A2B3F
:104CAC00EADD6C2A2FD13A787E1C642A00F08880C9
:104CBC000AD8252A3CD002D8002A47D0BDE7582A6A
:104CCC000CD0632A19D0B8E7732A22D002D86E2AE6
:104CDC0037D0B2E7752A62D0782AAED1271D20686A
:104CEC00A2F1580462424FF0100162415BE02CD9F2
:104CFC00582A38D0632A34D13E4640462178271DA5
:104D0C00C84701350FE0642A69D00ED9732A14D133
:104D1C003E46236840460093494652460023FFF71F
:104D2C00A3FE271D05443C4687E7252ADFD13E46D6
:104D3C0040462521C84701357FE70ED86E2A10D191
:104D4C003E46236804341D6077E752B9324B18682D
:104D5C00FFF700F80028F9D053E0752A28D0782AFC
:104D6C0001D03E4669E7A2F1580304F1040C5A4203
:104D7C002068CDF80CC04FF010015A4105ABFFF77D
:104D8C0025FEDDF80CC03E46644605AB009340465C
:104D9C00494652465B46FFF767FE05444DE72068DF
:104DAC00271D0A21002205ABFFF737FE3C46ECE736
:104DBC0004F1040CCDF80CC020680A210022DDE7B8
:104DCC002068271D002808DA2D238DF81430404266
:104DDC000DF115030A210022E6E705ABFAE720687E
:104DEC0004F1040C00280ADA2D238DF8143040420B
:104DFC000DF11503CDF80CC00A210022BFE705AB5D
:104E0C00F8E7284609B0BDE8F04F04B0704700BF82
:104E1C00B4030020B0030020D402002080EAE07329
:104E2C00A3EBE0738B4206DB002801DD401A7047D0
:104E3C0002D0084470470020704770B5044604F057
:104E4C00D1FA2030402857D820462C4904F0C0FA1B
:104E5C0028B120462A4903F0F5FF0446F4E7204622
:104E6C00284904F097FA28B12046254903F0ECFFB5
:104E7C000446F4E72046244904F0AAFA30B122494A
:104E8C00204603F0DFFF01461F480AE020461F4979
:104E9C0004F080FA40B11C49204603F0D5FF0146CE
:104EAC001A4803F0CFFF04462146204604F0D4F8FC
:104EBC0005462046294604F0CFF8154906462846F3
:104ECC0004F0CAF8134903F0BDFF0146284604F06C
:104EDC00C3F8114903F0B8FF0146284604F0BCF8AA
:104EEC000E4903F0AFFF0146304604F0B5F8014619
:104EFC00204603F0A9FF70BD002070BDDB0F4940B8
:104F0C00DB0FC940DB0F49C0DB0FC93FDB0FC9BF4B
:104F1C009A7C2E36FAAF4F393587083CA4AA2A3E24
:104F2C002DE9F04F056885B00C4681463B49284673
:104F3C0003F08AFFFFF781FF80462846FFF77DFFCD
:104F4C00D9F8045006463549284603F07DFFFFF793
:104F5C0074FF07462846FFF770FFD9F808900546FE
:104F6C002E49484603F070FFFFF767FF824648461C
:104F7C00FFF763FF41468146504604F06DF8414609
:104F8C008346484604F068F851460190304604F0D8
:104F9C0063F849460290304604F05EF839460390B7
:104FAC00504604F059F84946206007F1004004F0DF
:104FBC0053F829466060A560029804F04DF801464C
:104FCC00019803F041FF2946E060039804F044F88F
:104FDC000146584603F036FF3946206106F1004081
:104FEC0004F03AF829466061584604F035F8014659
:104FFC00039803F027FF2946A061019804F02CF8D0
:10500C000146029803F020FF4146E061384604F067
:10501C0023F8206205B0BDE8F08F00BFDB0FC93F5D
:10502C002DE9F04107688AB0466885680446084651
:10503C0001A9FFF775FF0199384604F00DF80499A2
:10504C008046304604F008F80146404603F0FCFE6A
:10505C0007998046284603F0FFFF0146404603F0BF
:10506C00F3FE02992060384603F0F6FF059980465E
:10507C00304603F0F1FF0146404603F0E5FE089987
:10508C008046284603F0E8FF0146404603F0DCFE6C
:10509C0003996060384603F0DFFF069907463046F7
:1050AC0003F0DAFF0146384603F0CEFE09990646B6
:1050BC00284603F0D1FF0146304603F0C5FEA06040
:1050CC000AB0BDE8F081074B10B51A881C4622EADD
:1050DC0000009042188002D00120FEF799FD208834
:1050EC0010BD00BF88070020064B10B51A881C465F
:1050FC0010439042188002D00120FEF789FD2088D1
:10510C0010BD00BF88070020024A936823EA000004
:10511C0090607047000A002008B5104B1A780023E5
:10512C00D9B2914207D20E49002051F82310013315
:10513C0009680880F4E73220FEF7ADFD094B1B68C7
:10514C005A0309D5084B9B685B0305D4BDE808409E
:10515C0040F2DC50FEF79FBD08BD00BF7807002071
:10516C00E8100020E80F0020000A00202DE9F34190
:10517C0001F048F84B4A692313704FF4A363538032
:10518C00BE231371EF2382F81635002319461646F9
:10519C0082F81735F25C0133B3F5A36F81EA020193
:1051AC00F8D1404B404A83F81715404B04275A60FE
:1051BC0002F188325A600020013F17F0FF075ED0E1
:1051CC003A4B34223A4CDA6004F17848A8F5784826
:1051DC00C8F3090353B100234FF4005056F808806C
:1051EC00019300F0C9FD0428E6D11CE04FF43020F7
:1051FC0000F0C2FD0428DFD12C4D4FF430202B6978
:10520C0043F002032B616C612B6943F040032B616B
:10521C0000F0B2FD41F6FD732A69042803EA02038B
:10522C002B61D8D0C8E7214D4FF400502B6943F0C7
:10523C0001032B611FFA88F3238000F09DFD0428E5
:10524C0013D1A31C0193019B4FEA1848A3F80080CB
:10525C004FF4005000F090FD41F6FE732A690428CB
:10526C0003EA02032B6106D0A6E741F6FE732A6916
:10527C0013402B61A0E70F4B04349C42A4D10B4A82
:10528C000428136943F08003136102D102F0E0F9A2
:10529C0010B90520FEF709FD00F0A0FF02B0BDE833
:1052AC00F08100BF000A0020230167450020024066
:1052BC0000F8000818FD000810B50E4C2068FEF729
:1052CC0017FC20680022047A02FB02F3193B6343AB
:1052DC0003F6C4135343192193FBF1F3064921F848
:1052EC0012300132072AEFD1BDE810400349FEF716
:1052FC00B7BB00BFE807002004020020D40A00203E
:10530C002DE9F04102F0A4F910B90420FEF7CDFC10
:10531C00A34C00F077FFA3494FF4A362204607F09B
:10532C00E3FA94F8F0344FF48E71022B84BF00230F
:10533C0084F8F03494F8F0249B4D01FB02F3E01850
:10534C0000F5CE702344286093F8F00101FB024273
:10535C00022803F5F47384BF0020187292F8F03120
:10536C00924A13700C2202FB0343914A03F2F2435C
:10537C00136046F20902A3681A401AB9884A43F42A
:10538C0000539360A368D80703D54FF40050FFF780
:10539C00BBFEA368590409D50820FFF7B5FE4FF4EE
:1053AC000050FFF7B1FE0120FFF7AEFEA3681A070D
:1053BC0006D54FF40050FFF7A7FE0120FFF7A4FE1F
:1053CC00A3689B0413D54FF40040FFF79DFE744B6C
:1053DC0093F81631012B03D14FF40060FFF794FEC4
:1053EC004FF48030FFF790FE4020FFF78DFE94F8CD
:1053FC0070216B4B2AB193F8742112B1002283F8FF
:10540C0074214FF0000C67466A4E6B4B1E6004EB28
:10541C000C03B3F87EE14FEA5E0101F077314FEAFD
:10542C009E0303F03333C1EB0E00C11A4FEADE03C7
:10543C0003F01133CB1A03EB231303F00F32FF23CA
:10544C0092FBF3F31EF00108C3EB032318BF0137E3
:10545C00A2EB030318BFFFB2012B0ADD022B40F0B5
:10546C009C80B8F1000F00F098801EF0BC0F00F08B
:10547C0094800CF1080CBCF1100FC8D1013F012F26
:10548C0000F28B80FFF718FF002130224B4807F009
:10549C0036FADFF878814A4B2F68C3F80080494B05
:1054AC0007F179001F6000F023FB474B80F00100EF
:1054BC001870464B08F126021A60387801F00EFD80
:1054CC00434B94F8681108F194021A6064224A4321
:1054DC00404BC8325A6000229A60DA601A615A61F5
:1054EC009A61DA6183F8202083F821203A4B08F185
:1054FC002C021A60394B08F108021A60384B394FEC
:10550C00C3F80080384B08F1A0021A6008F1A4031C
:10551C003B60364BB4F8F6001E6003F045FDB860F6
:10552C00B4F8F80003F040FD2D683A1D95F85C3096
:10553C00F8603B7195F87830286E7B7194F8733174
:10554C007D613B742A4B2B491A602B4B05F164028D
:10555C001A6003F081FD01464FF07C5003F030FEE1
:10556C00B5F81641254B1860204603F021FD014685
:10557C00234803F025FE234903F06EFD224BBD6149
:10558C00186005F1680305F21115FB613D62C7F85F
:10559C002480BDE8F04100F021BE00F087FA71E7ED
:1055AC00000A002000F80008EC070020DC160020A0
:1055BC00E80700201A0B0020E40F0020A0060020B2
:1055CC00D4060020D80600201C000020E00000209B
:1055DC00D8160020F80F002048010020700700208A
:1055EC00740700200C080020E0020020A403002017
:1055FC0078010020DB0F4940B0010020AC010020F5
:10560C00000061444C3D0F44DC020020D40A002011
:10561C0008B5FFF7ABFDFFF773FEBDE808400120AE
:10562C00FEF7F6BA084BDA68D10709D4DA685207E4
:10563C0008D4DB6813F0100F14BF0320042070474C
:10564C0001207047022070470020024003788B42F3
:10565C0086BF024B33F81100002070473808002039
:10566C000022134670B5234914180C44247E83EA97
:10567C000423082413F4004F4FEA430318BF83F4A8
:10568C00815304F1FF3418BF83F0010314F0FF04BD
:10569C009BB2EFD10132192AE5D100F1190200F1C8
:1056AC001A050A440D44167E2A7E02EB062292B29B
:1056BC009A421ED10F4B93F83950E2B2AA4215D23E
:1056CC00431C03EB4203DBB2CA1801330B44127EBA
:1056DC001B7E03EB02239BB24FF4AF6253431B13AD
:1056EC0003F5487321F814300134E6E7012381F8FF
:1056FC003A3070BD3808002003788B420BD9074B29
:10570C00890093F83B201944C86B02B1400800F59E
:10571C00777080B270470020704700BF38080020B7
:10572C0007299DBF034B03EB8101B1F86C000020EE
:10573C00704700BF38080020034B03EB4101B1F860
:10574C008C00C008704700BF3808002008B5084B13
:10575C0003EB8101D1F8AC0003F026FC054903F002
:10576C007BFC054903F070FB03F062FE80B208BDC0
:10577C00380800200000203F00005C44024B03EB83
:10578C004101B1F8F400704738080020024B03EBDC
:10579C004101B1F81801704738080020024B03EBA7
:1057AC004101B1F8180170473808002000207047FB
:1057BC0010B50446FEF748FA41F288310E4BE4B2BC
:1057CC00D3F83021C3F83001821A8A42C3F834214D
:1057DC0084BF002283F8382193F8382106490F2A18
:1057EC00134418BF013283F8394112BF81F83821B4
:1057FC00012381F8493110BD3808002070B50546E9
:10580C00FEF722FA314CD4F84C31C4F84C01C31ACF
:10581C00B3F5FA5FC4F8503182BF002384F85431D9
:10582C0084F8553194F854312BB9A12D02BF274A75
:10583C00012182F8551194F85511244A29B1D11837
:10584C00EDB201330D7682F8543194F8545194F83A
:10585C005631AB4239D11D4B93F85731052B02D041
:10586C00062B03D02CE00020FFF7FAFE637E1E2BE4
:10587C0026D100200246C1B26B1E994219DA21448E
:10588C000B7E0821DBB283EA0206F60744BF83F0E5
:10589C001803C3F3460301F1FF3154BF5B0843F017
:1058AC00800311F0FF01C2F34702ECD101301A461C
:1058BC00E1E723441B7E9A4202D10320FFF7D0FE7E
:1058CC00002384F8553184F8543170BD3808002019
:1058DC0010B50446FEF7B8F941F288310E4BD3F8F7
:1058EC005821C3F85801821A8A42C3F85C2184BF3C
:1058FC00002283F8602193F860210749142A13448D
:10590C0018BF013283F8614112BF81F86021012375
:10591C0081F8763110BD00BF3808002038B5044638
:10592C00FEF792F9274A2749D2F87831C2F8780164
:10593C00C31AB3F57A6F84BF002382F87C3192F8D6
:10594C007C3133B9A82C3BD181F87D31A1F87E3163
:10595C0006E0022B02D181F8804101E0242B02D811
:10596C00D11881F8814192F8801101330231DBB2F8
:10597C0049008B42134D82F87C3118DAB5F87E3130
:10598C00E0B283EA0020082310F4004F4FEA4000F5
:10599C0018BF80F4815003F1FF3318BF80F0010071
:1059AC0013F0FF0380B2EFD1A2F87E0138BD0131B4
:1059BC008B4201BF002385F87C31012385F87D31B2
:1059CC0038BD00BF3808002010B50446FEF73CF97E
:1059DC0040F6AC510F4AD2F8A831C31A8B42C4BF5F
:1059EC00002382F8AC3192F8AC31D11881F8AD417A
:1059FC0023B90F2C0DD10749C1F8A8010133DBB233
:105A0C00192B044982F8AC310CBF0123002381F817
:105A1C00C63110BD380800200C4B0D49DA684378AC
:105A2C00D243C2F30222C2F10402934002781B015A
:105A3C00DBB20A4482F8003303780122580903F0E0
:105A4C001F0302FA03F341F82030704700ED00E029
:105A5C0000E100E073B5054600210068012202F068
:105A6C0019F82A680124138800269BB243F001031D
:105A7C001380EB7A01A88DF804308DF805408DF871
:105A8C0006608DF80740FFF7C7FFEB7A1B2B0BD195
:105A9C00192301A88DF804308DF805408DF80660A7
:105AAC008DF80740FFF7B8FF02B070BD10B50F4C72
:105ABC000021122204F2423006F021FF05230421BA
:105ACC0084F8483384F84A3384F8503384F85233DA
:105ADC005223012284F8491384F8511384F8423379
:105AEC0084F84C23A4F8462310BD00BF38080020CE
:105AFC0000F1500302781AB98178C278914204D32C
:105B0C0004309842F6D1002070470120704770B5E0
:105B1C000646441E14F8011F89B1094D284606F0AB
:105B2C0024FF0028F6D005F1080398423FBF054B2F
:105B3C00401BC018A31B38BF80F8E232EAE770BDE7
:105B4C0070EA000838080020031EB8BF2D2210B5DB
:105B5C00B8BF58420C46B8BF01F8012B0A22FFF718
:105B6C0049F800230370204610BD07B51B4B03F208
:105B7C00E462C3F8E02693F8EA225AB1012A14D160
:105B8C00032183F8E616072183F83B2083F8E716F8
:105B9C000C2208E0022183F8E616032183F83B204F
:105BAC0083F8E716072283F8E4260D4A0D4B4020B4
:105BBC001A60FDF74DFF70B10122002390F900002F
:105BCC0040218DE80C00084A4FF4E133FDF766FDE7
:105BDC00003018BF012003B05DF804FB380800202A
:105BEC000557000820000020BD57000801200021A7
:105BFC00FEF7E4B84FF6FE7302681340036000230F
:105C0C00036043608360C360284B984201D1284AEB
:105C1C0027E0284B984201D1254A2AE0264B98428E
:105C2C0001D1234A2DE0254B984201D1204A30E086
:105C3C00234B984201D11E4A33E0224B984204D1A7
:105C4C001B4A536843F470032EE01F4B984204D157
:105C5C00174A536843F0706326E01C4B984204D1FA
:105C6C001B4A536843F00F031EE01A4B984204D1B1
:105C7C00174A536843F0F00316E0174B984204D1CF
:105C8C00134A536843F470630EE0144B984204D1EA
:105C9C000F4A536843F4704306E0114B984204D109
:105CAC000B4A536843F4702353607047080002405A
:105CBC00000002401C000240300002404400024040
:105CCC00580002406C000240800002400804024070
:105CDC00000402401C040240300402404404024010
:105CEC00580402401F4A10B5536803F00C03042BF0
:105CFC0003D0082B04D01C4B14E01C4B5B6811E048
:105D0C0053685168C3F38343C90303F1020301D4FD
:105D1C00174906E0516811F4003F1449496818BF4F
:105D2C0049084B43036053681249C3F30313CC5C1B
:105D3C000368E34043605468C4F302240C5D23FA07
:105D4C0004F484605468C4F3C2240C5DE340C36063
:105D5C005268C2F381320A44127CB3FBF2F3036142
:105D6C0010BD00BF0010024000127A00200000207D
:105D7C0000093D0090D8000810B50446FFF752FC0E
:105D8C00012806D11CB1FFF74DFC013CF8E70520BA
:105D9C0010BD002C08BF052010BD0F4B1A6842F037
:105DAC0001021A6059680D4A0A405A601A6822F0BA
:105DBC00847222F480321A601A6822F480221A60EB
:105DCC005A6822F4FE025A604FF41F029A60044B88
:105DDC004FF000629A607047001002400000FFF81C
:105DEC0000ED00E02DE9F8435B4C0368013AC4F880
:105DFC00E83683880D46A4F8EC36072A42D8DFE84B
:105E0C0002F0040A101822292F35B4F8E8360B805A
:105E1C00B4F8EA3613E0B4F8EA360B80B4F8E83696
:105E2C0005E0B4F8E8365B420B80B4F8EA365B4226
:105E3C0005E0B4F8EA365B420B80B4F8E8366B80C8
:105E4C00B4F8EC361DE0B4F8E8365B420B80B4F8DD
:105E5C00EA3612E0B4F8EA360B80B4F8E8360CE017
:105E6C00B4F8E8360B80B4F8EA3605E0B4F8EA3654
:105E7C005B420B80B4F8E8365B426B80B4F8EC36CE
:105E8C005B42AB80354B1B7A002B62D1B5F900001D
:105E9C0003F08EF88046B5F9020003F089F8074646
:105EAC00B5F9040003F084F8D4F8F0160646404621
:105EBC0003F0D2F8D4F8FC168146384603F0CCF83F
:105ECC000146484602F0C0FFD4F808178146304618
:105EDC0003F0C2F80146484602F0B6FF06F06EFE2B
:105EEC00D4F8F4162880404603F0B6F8D4F800171E
:105EFC008146384603F0B0F80146484602F0A4FF4C
:105F0C00D4F80C178146304603F0A6F801464846F3
:105F1C0002F09AFF06F052FED4F8F816688040465C
:105F2C0003F09AF8D4F804178046384603F094F836
:105F3C000146404602F088FFD4F810170746304659
:105F4C0003F08AF80146384602F07EFF06F036FE72
:105F5C00A880BDE8F88300BF38080020200000208E
:105F6C0044F6FB71084BD3F81427137803EB431357
:105F7C0000FB03135078C0EB0030B3FBF0F39078C8
:105F8C00B3FBF0F080B27047380800202DE9F84FD1
:105F9C00774C0023B4F92227A4F818370A2A18BF23
:105FAC0084F8203794F82067714B002E66D1714A23
:105FBC0003F5E465C3F82427C3F82C274FF07E5271
:105FCC00C3F830276C4AA846C3F834276B4A6C498F
:105FDC00C3F8382740F2DC52C3F874271022A3F818
:105FEC0072271822C3F82817A3F8702708EB0607A6
:105FFC004FF09741386903F02FF80021814603F0E8
:10600C00C9F928B148464FF07C5102F01BFF04E05F
:10601C0048464FF07C5102F017FF03F045FAC5E9F2
:10602C000E0178684FF0974103F016F800210746EF
:10603C0003F0B0F928B138464FF07C5102F002FF62
:10604C0004E038464FF07C5102F0FEFE03F02CFACF
:10605C0004360C2EC5E9080105F10805C6D10A2342
:10606C00A4F82237474BC4F89037C4F89C37C4F8CF
:10607C009437C4F8A037012384F82037DFF808C11F
:10608C00D4F87487B4F97257DCF82430C8F10006E0
:10609C00AE407343DCF820704FEAE67BD4F890E70F
:1060AC0007FB0B33C4F89067A7FB0667D4F89C2753
:1060BC001F44DCF84430DCF840A053434FEAE27B49
:1060CC00D4F8A0070AFB0B39C4F8A027AAFB0223BB
:1060DC004B44B61A67EB0307DCF82C30DCF82820AD
:1060EC000EFB03F34FEAEE7B02FB0B39A2FB0E23F4
:1060FC00B6184B445F41DCF84C30DCF84820434385
:10610C004FEAE07B02FB0B39A2FB0023D4F8941777
:10611C00B21ADCF83460C4F8A40701FB06F6DCF80C
:10612C0030004B4467EB0303CF17C4F8981700FB00
:10613C000766A0FB010180183144C4F894E759416B
:10614C00B4F9702702F06CFE6A1E01239340C4F868
:10615C009C07C01841EBE3712A4602F061FE10EB7C
:10616C00080080B2FFF7FCFEA4F8A807BDE8F88F82
:10617C003808002056157D396350FABF0CE0743F87
:10618C005615FD39000024FA580F002070B512493D
:10619C004300D1F8AC270E46D418257E15B1022D3C
:1061AC0010D00BE0022805D9032807D1D1F8B0375D
:1061BC00DB0401D5D08970BD908A70BD3344B3F82F
:1061CC00F40070BD607E00EB800000EB800000F2FC
:1061DC00EE2080B270BD00BF3808002008B5FDF776
:1061EC0033FD074B022283F8B827D3F8BC27C3F83A
:1061FC00B407C3F8C827012283F8E12708BD00BF04
:10620C003808002008B5FDF71FFD084B022283F863
:10621C00B827D3F8C82700F5B71000F5587002F26C
:10622C00DC52C3F8B407C3F8C82708BD38080020EF
:10623C0042F20102034BD3F8B0371A420CBF0120D3
:10624C000020704738080020104B10B593F8E42755
:10625C001C46012A0DD007D3022A0ED10C4AD36852
:10626C0083F48043D36008E0094B4FF480421A61F9
:10627C0003E0074B4FF480425A61FDF7E5FC00F553
:10628C00F42000F59070C4F8E80710BD3808002021
:10629C00001001402DE9F04F87B00393904B074657
:1062AC001B8893469B0736D540F2E632109B8D48EF
:1062BC00DC89B0F900301B1B03F2F315954203D8AF
:1062CC00002BB8BF5B4201E04FF4FA73B0F9022027
:1062DC0040F2E630121B02F2F314844203D8002A77
:1062EC00B8BF524201E04FF4FA729342B8BF134662
:1062FC000522C3F5FA7393FBF2F30A22643B534372
:10630C003A7FD2105343642293FBF2F3134423EAF3
:10631C00E373DBB200E06423B8460093CB1C02931A
:10632C000025029B022D13F8010F4FEA450A029338
:10633C006D4B06D1B3F9046000F11B047443621178
:10634C002EE033F91510CBF100024C00944203DB24
:10635C005C452246A8BF5A46644C34F90A40121BCD
:10636C00039C34F9156016445D4AB2F800E01EF047
:10637C00010F12D100F11B044C431EF0020F4FEA27
:10638C0024120DD0BC7C9DF900007443444364215D
:10639C0094FBF1F102EB211202E03A7A72431211F2
:1063AC005349042431F90A1098F801C091FBF4F414
:1063BC004D4E141B0CFB04FC06F10802AA5C97F86A
:1063CC00519002FB0CFC019264229CFBF2FC4FEA04
:1063DC00EC1CB9F1000F20D0022D10D160460493B3
:1063EC0002F0E6FD5FEA5901049B04D049450A46D8
:1063FC00A8BF4A4600E001223E495B6A08E06046BD
:10640C0002F0D6FD4A4606F10C01736A01EBC50198
:10641C00FEF75AFB02F0E6FF8446374B98F80B6008
:10642C001988314B01FB04F203F1280E5EF82500AC
:10643C00D21206FB0206314AB6F5001FA8BF4FF474
:10644C000016964203F13400B8BF164650F82520CA
:10645C0040F825404FF6FF700909B0FBF1F1A21A84
:10646C004A4303F1400103F14C044EF8256051F806
:10647C0025E054F8250044F825E097F85040921197
:10648C0070447613104441F825208CB1CDF810C01F
:10649C00059302F08DFD059B224603F1580101EB9B
:1064AC00C5015B6AFEF710FB02F09CFFDDF810C023
:1064BC0098F8153066445843019B4FF0640C4343E5
:1064CC0093FBFCF001350E4B06EB2020032D23F83B
:1064DC000A0008F101087FF424AF07B0BDE8F08F83
:1064EC00880700202C09002028100020D607002047
:1064FC00B207002044100020800700200000E0FFBD
:10650C00981000202DE9F04F89B00593B74B002669
:10651C00B3F90290B3F90030B9F1000FB8BFC9F16B
:10652C000009002BB8BF5B429945B8BF9946074696
:10653C00B2463446B9F5FA7F04910392A8BF4FF4E2
:10654C00FA79019000960296A94B188810F0030571
:10655C003AD0A64B610033F91420039B52005B42E6
:10656C009A4203DB039B9342A8BF1346A14A6FF0E8
:10657C00040A895E059A5B1A32F9141064221944D4
:10658C003B7A4B4393FBF2F33A7F0AFB02FA5345F7
:10659C0004DB02EB820A9A45A8BF9A46964A52F847
:1065AC002430194442F210739942A8BF1946934BF8
:1065BC009942B8BF1946BB7C42F824105943012DAF
:1065CC004FEA2133029338D08849A60031F91430B0
:1065DC0028310093019B51F824E093F801C0884BBB
:1065EC0033F9145085EAE573A3EBE573B3F5206F2B
:1065FC0016DC009A50235A4392FBFCF3042295FBC1
:10660C00F2F55D1BAE44BEF57A5F7E4BA8BF4FF42E
:10661C007A5E9E45ACBF41F824E041F8243002E09C
:10662C00002341F824308B597D2693FBF6F6019B11
:10663C00DB7A7343402693FBF6F6820712D5009A59
:10664C0009FB06F509FB02F80298C9F5FA7303FB7E
:10665C000A8803FB00534FF4FA7198FBF1F293FB99
:10666C00F1F505E0C30755BF35465246009A029D29
:10667C00634B4FF0040833F914304FEA440B93FB8F
:10668C00F8F85A4B03F18001615C01FB08F86FF0DC
:10669C004F0198FBF1F8904497F8512082B1404695
:1066AC000793069202F084FC079B069A03F10C01F7
:1066BC0001EBC4015B6AFEF707FA02F093FE804619
:1066CC004F4B3BF80300494B02B203F184013BF9F9
:1066DC0001E02BF80100CEEB02024FF0040E92FB0E
:1066EC00FEF203F1880103F1900E51F824C05EF81C
:1066FC00240041F824206044104497F850204EF8B0
:10670C0024C072B10793069202F052FC079B069AC2
:10671C0003F1580101EBC4015B6AFEF7D5F902F0F5
:10672C0061FE324A454402F1980111F8048002F1ED
:10673C00700308FB00F04FF0200890FBF8F02D1AC6
:10674C002BF80350019B013301930CB90124FBE698
:10675C00049BB2F904109B7904200F335B004B436C
:10676C0027495B11B1F90410002B91FBF0F0A3EB5E
:10677C000000B8BF5B42322B146B797B0BDC01FB46
:10678C000041214B8B42A8BF0B4620498B42ACBF2A
:10679C001363116301E000231363F97801FB00F329
:1067AC001B499B11097803290CD9B7F84E10B1F588
:1067BC00FA7F07D24842834203DB8B42A8BF0B46C9
:1067CC0000E00346116B6FF0FF0041F34F31B1F560
:1067DC00807FA8BF4FF480718142ACBF5B181B183F
:1067EC00A2F8743009B0BDE8F08F00BF281000206B
:1067FC0088070020D6070020A0100020F0D8FFFF4B
:10680C00B207002080C1FFFFFEFFFF0F020000F067
:10681C00780700202DE9F04F054690F850008DB018
:10682C000A9107920B9318B13228A8BF322000E0CE
:10683C00012002F0BDFB01469B4802F0C1FC9B4BC2
:10684C0004461888002808BF012002F0B1FB9849C3
:10685C00089002F001FC01900199204602F0F4FA34
:10686C000146019802F0ACFC924B09901B889807EA
:10687C0024D59149B1F90030B1F9020083EAE372F1
:10688C0080EAE071A2EBE372A1EBE07191420C465D
:10689C00B8BF1446B4F5E17F12DA914203DD00284B
:1068AC00D8BF404203E0002BCCBF1846584202F040
:1068BC007FFB824902F084FC064603E0002601E0DF
:1068CC004FF07E564FF0000904950024CDF8089047
:1068DC00630006937A4B33F814800FFA88F002F0B9
:1068EC0067FB784902F0B8FB02F07CFD02F060FB1C
:1068FC00754902F0B1FB704B039033F9140002F0B0
:10690C0057FB6C4B07461B889907059362D00146D1
:10691C0002F09AFA02F066FD079B5B42984203DB99
:10692C00079B8342A8BF03460699684A885E0B9A68
:10693C001B1A32F91400184402F03AFB8246287FE5
:10694C0002F032FB624902F087FB8346287A02F0A0
:10695C002BFB0146504602F07FFB5E4902F07CFBAC
:10696C0002F040FD81460BF1004002F03BFD8145F9
:10697C0005DB584602F036FD4845A8BF484602F0F4
:10698C0017FBDFF8749102900199504602F064FBFA
:10699C0059F8241002F058FA4F494FEA840B8246FA
:1069AC0002F0F8FC38B950464C4902F011FD20B108
:1069BC00DFF828A101E0DFF820A149F80BA0A87CA2
:1069CC0002F0F2FA0146504602F046FB444902F04E
:1069DC0043FB8146059BDA0700F190800FFA88F89B
:1069EC00B8F1000FB8BFC8F10008B8F5206FDFF898
:1069FC0000A14FEA840803DD00234AF8243028E084
:106A0C003849384602F028FB049B8346587802F03C
:106A1C00CBFA0146584602F0D3FB039902F012FA66
:106A2C00019902F019FB5AF8241002F00DFA2E49C4
:106A3C00824602F0AFFC38B950462C4902F0C8FC33
:106A4C0020B1DFF8A8A001E0DFF89CA0284B43F8A8
:106A5C0008A0049BD87A02F0A7FA254B53F824100F
:106A6C0002F0FAFA234902F0F7FA059B80469B07DD
:106A7C0046D53846029902F0E5F90146304602F057
:106A8C00EBFA0146029802F0DFF949460746404608
:106A9C0002F0D8F90146304602F0DEFA01464846CB
:106AAC0002F0D2F980462BE083F9223E80070020C9
:106ABC00BD37863588070020281000200000E143F0
:106ACC00B20700200000A03ECDCC4C40D6070020E1
:106ADC000000A0406F12033C0000F0C10000F04128
:106AEC000AD7A33D0000A043000040C30000404370
:106AFC00CC1000200AD7233CC4100020C846029FAB
:106B0C00DFF8E8A10AF18003185D02F051FA0146A2
:106B1C00039802F0A1FA744902F09EFA0146384635
:106B2C0002F090F995F85120834642B10AF10C011C
:106B3C0001EBC401DAF82430FDF7C6FF83466B4F36
:106B4C00039807F1B00A5AF8241002F07BF9019966
:106B5C0002F036FB039B4AF8243007F1B80353F8D4
:106B6C0024A00393514602F06DF90146099802F0F6
:106B7C0073FA0146504602F067F9039B414643F80D
:106B8C0024008246584602F05FF907F198038046CC
:106B9C00185D02F00DFA0146504602F05DFA5449B8
:106BAC0002F05AFA0146404602F04CF906F006F89B
:106BBC00069A07F170039852049B013304930CB9A5
:106BCC00012485E60A9AB7F90430947964002834D4
:106BDC005C43484B6411B3F9040002F0E9F94FF03F
:106BEC007A5102F039FA05F0E9FF201A02F0E0F9C7
:106BFC00002CB8BF6442322C064602DD00233B63F6
:106C0C0024E0089802F0EEFB20F0030002F0D0F92B
:106C1C008046687B02F0C8F90146304602F01CFA47
:106C2C0035490446404602F0CBFA0146204602F0B4
:106C3C0013FA02F0D7FB3B6B1844304B9842A8BFB9
:106C4C0018462F4B9842ACBF38633B633B6B6FF0DD
:106C5C00FF005B13B3F5807FA8BF4FF4807398429D
:106C6C00B8BF184602F0A4F90446304602F0BAFB4D
:106C7C00EB785843801102F09BF9224A03461278B4
:106C8C00032A11D9B5F84E60B6F5FA7F0CD202F092
:106C9C00A9FB7342984203DBB0420346A8BF3346BC
:106CAC00184602F085F9034695F8512062B1510857
:106CBC0003D08A42A8BF0A4600E0012218461249B6
:106CCC007B6AFDF701FF03461846214602F0BCF82B
:106CDC0002F088FB00B202F06BF905F06FFFA7F829
:106CEC0074000DB0BDE8F08FA69B443B281000202B
:106CFC00F7CC9238B207002000803B45FEFFFF0F17
:106D0C00020000F078070020441000202DE9F84321
:106D1C000024254BE0B21E78B0420ED2234B33F840
:106D2C001010234B03EB8003D3F8C0301BB10B289E
:106D3C0001D8DB6898470134EBE71E4B1B685B03FB
:106D4C002FD500242346E2B2B2422AD2DFF860905B
:106D5C004FEA840809F1C00757F8242055689D4272
:106D6C0017D0284600F0EAFEEFF31283502282F38C
:106D7C0012882821AA8C01FB009092B20132C0F833
:106D8C001421AA8ADBB292B242F00102AA8283F3E6
:106D9C00118857F8083000221B6801341A802B46E2
:106DAC00D1E7BDE8F88300BF78070020BE070020BC
:106DBC0028100020E80F00200A4B30B51A680A4B47
:106DCC0002F480521C68094B1D6800230AB1A1888B
:106DDC0000E0A988064820F8131001330C2BF5D1DC
:106DEC0030BD00BFE80F00207007002074070020A2
:106DFC00DE1600202DE9F74F334C0546D4F8907180
:106E0C003249384602F020F8FEF717F806463846A5
:106E1C00FEF713F8D4F8947181462C49384602F0E9
:106E2C0013F8FEF70AF801903846FEF706F8D5F885
:106E3C0004A007463146504602F00EF9D5F80880FA
:106E4C0083464946404602F007F90146584601F090
:106E5C00F9FF019B29688346184602F0FDF8494664
:106E6C000546504602F0F8F8394602F0F5F80146AE
:106E7C00284601F0E9FF39460546404602F0ECF899
:106E8C00314602F0E9F80146284601F0DDFF0146E3
:106E9C00584605F01FFF0E4902F0DEF80D4902F0CE
:106EAC008FF9D4F8981101F0CFFF0B4902F088F953
:106EBC0005F084FE83B21A0444BF00F5B47083B2AB
:106ECC0018B203B0BDE8F08F28100020DB0FC93FCB
:106EDC000000E144DB0F49400000204101380A4B1F
:106EEC00042804D8DFE800F00507090B0D00074A59
:106EFC0008E0074A06E0074A04E0074A02E0074AAE
:106F0C0000E0074A1A60704730000020417F0008FB
:106F1C00A1620008F1810008817C0008116500085D
:106F2C0021680008F0B5046D8279A389467923F4B1
:106F3C00005312F0020F4FEA03434FEA13430CBF06
:106F4C0000214FF4005112F0040FA38114BF4FF431
:106F5C00806E4FF0000E16F0010F8768054614BFC7
:106F6C0004200020B307238A48BF40F008029BB2DC
:106F7C0023F4405343EA01032382A18948BF90B212
:106F8C0089B221F4B05121F00C014EEA010140EA22
:106F9C000102A281A38A87B023F440731B041B0C4B
:106FAC00A38201A8FEF79EFE049E039B204A9442F6
:106FBC0018BF1E46A389192272431BB2002BB4BF03
:106FCC007E00BE00B2FBF6F66427B6FBF7F00001BC
:106FDC00010907FB1163A28912B2002AADBF1A0185
:106FEC00D90032313232ABBFB2FBF7F3B1FBF7F25F
:106FFC0003F00F0302F00702B4BF104318432A6DCD
:10700C00AB7980B2208113F0080F938A0BBF23F069
:10701C0008039BB21B0443F0080308BF1B0C9382AC
:10702C0093899BB243F40053938107B0F0BD00BF2A
:10703C00003801402DE9F3411D468C4B884698429F
:10704C0017469DF8206051D1894B8A4A8A491A60AB
:10705C008A4A59635A6102F580729A614FF48072C0
:10706C00DA601A61864A9F601A63A2F54842543A64
:10707C00DA649A641865834B31079A6942F480424A
:10708C009A615A6942F001025A614FF002038DF87D
:10709C0003304FF40073ADF8003001D51C230FE022
:1070AC00AA0706D51823784869468DF80230FAF7F6
:1070BC00DFFAEB070AD54FF48063ADF800304823B4
:1070CC00714869468DF80230FAF7D2FA0E238DF822
:1070DC0004300022012301A88DF805308DF806201C
:1070EC008DF80730624CFEF797FC4DE0674B9842E9
:1070FC0040F0B880664B5F4A9F601A604FF4807214
:10710C00DA601A61634A18655A6102F580729A61F5
:10711C00614A34079A64DA645A4BDA6942F40032F1
:10712C00DA615A6942F001025A614FF002038DF89C
:10713C0003304FF00403ADF8003001D51C230EE0F2
:10714C00A80706D51823504869468DF80230FAF77F
:10715C008FFAE90709D50823ADF8003048234A48CF
:10716C0069468DF80230FAF783FA26238DF804303D
:10717C000022012301A88DF805308DF806208DF82A
:10718C000730FEF749FC424C012384F844300023BD
:10719C002362E361A3626362C4F82C806571A7600B
:1071AC00A6712046FFF7BEFEEA072AD5206B00B376
:1071BC00E76CD4F80C806669FEF71CFD236B216D1F
:1071CC001A6822F4FF4222F0700242F485521A60CF
:1071DC00C3F804809F60DE601A6842F001021A60F6
:1071EC008A8A92B242F040028A825B689BB2236424
:1071FC0007E04FF6DF72236D1A80DA6842F0200246
:10720C00DA60AB0726D5606BF8B1A56C2669FEF782
:10721C00F1FC636B1A6822F4FF4222F0700242F414
:10722C00845242F010021A6000225E609D60DA60A7
:10723C00196841F0020119605A605A60226D938AF4
:10724C009BB243F08003938204E0226DD36843F039
:10725C008003D360226D204693899BB243F4005384
:10726C00938100E0002002B0BDE8F08100380140BD
:10727C0018160020A4D8000844000240C4110020B5
:10728C005800024000100240000801400044004039
:10729C00C4150020C4130020044400407B4B10B5DF
:1072AC001B78012B14BF00240324038C91BB23F007
:1072BC0001031B041B0C0384018B038C89B221F08A
:1072CC00F30141F0010141EA0411714C9BB2A0425F
:1072DC0012D004F50064A0420ED0B0F1804F0BD058
:1072EC00A4F59834A04207D004F58064A04203D0E2
:1072FC0004F58064A04202D123F0020301E023F0E4
:10730C000A0343F001031A4301830284038B23F025
:10731C000C0339E004293ED123F010031B041B0C91
:10732C000384038B018C23F440731B051B0D43F466
:10733C00807343EA0434564B89B2984212D003F559
:10734C00006398420ED0B0F1804F0BD0A3F5983368
:10735C00984207D003F58063984203D003F580630D
:10736C00984207D121F0200141F0100141EA0212AC
:10737C0092B204E021F0A00141F010010A43048311
:10738C000284038B23F440631B041B0C0383038BC9
:10739C009BB2038310BD082937D123F480731B04DF
:1073AC001B0C0384818B038C89B221F0F30141F017
:1073BC00010141EA0411364C9BB2A04212D004F5F3
:1073CC000064A0420ED0B0F1804F0BD0A4F59834DD
:1073DC00A04207D004F58064A04203D004F5806479
:1073EC00A04207D123F4007343F4807343EA0222D2
:1073FC0092B204E023F4206343F480731A43818334
:10740C000284838B23F00C0338E023F480531B0499
:10741C001B0C0384818B038C21F440710905090D2D
:10742C0041F4807141EA0431194C9BB2A04212D054
:10743C0004F50064A0420ED0B0F1804F0BD0A4F53F
:10744C009834A04207D004F58064A04203D004F520
:10745C008064A04207D123F4005343F4805343EAE1
:10746C00023292B205E047F6FF541C4044F48054BB
:10747C00224381830284838B23F440631B041B0C03
:10748C008383838B9BB2838310BD00BFD403002006
:10749C00002C0140026D70B515880446ADB2A906EA
:1074AC0013D5036B8BB9C36A1BB1908880B2984714
:1074BC000BE0E169928840694E1CD2B2E6614254FD
:1074CC00E169E268914228BFE3612B0613D5636A38
:1074DC00A26A9A42236D0AD0511CA069A162825CF7
:1074EC009A802369994206D30023A36270BDDA689F
:1074FC0022F08002DA6070BD026B0346C16810B5E1
:10750C00406942B11A6C8C1A013A08BF0A46005DF8
:10751C001A64C0B210BD1A6A805C01328A4228BF5C
:10752C000022C0B21A6210BD436B13B190F8440034
:10753C007047836A406A1B1A584258417047036B64
:10754C0013B15B68016C01E0C369016A8B423CBFFB
:10755C00C2689B18581AC0B27047836A8169426B23
:10756C001944D160416A994297BF0169CB1ACB1A71
:10757C00536096BF0023536083624FF0000380F882
:10758C004430136888BF816243F001031360704775
:10759C00436A8269D154436A02690133934228BF1A
:1075AC0000234362436B1BB11B68DB0705D4D4E794
:1075BC00026DD36843F08003D36070472DE9F0412E
:1075CC0005460E46078A83899BB21F40002F37D091
:1075DC00B7FA87F24FF00043D340DB4399B21F4018
:1075EC00A2F11B032982042BF0D8DFE803F0221F41
:1075FC001C190300746A24B1013C0023A4B2736209
:10760C0001E0AC8DA4B2D6F82080B8F1000FDDD02B
:10761C00D8F80030404621469847D8F80480F4E763
:10762C003068A98E08E07068298F05E0B068A98FD2
:10763C0002E0F068B5F84010036889B29847C5E7D6
:10764C00BDE8F0814171FFF76DBC8160FFF76ABC4A
:10765C000E4B1A78692A15D15A88B2F5A36F11D13D
:10766C001A79BE2A0ED193F816250020EF2A0BD1D9
:10767C0013F8012B5040064A9342F9D1B0FA80F02E
:10768C004009704700207047704700BF00F80008A1
:10769C0018FD00082DE9F74FDD4C00214FF4A362D3
:1076AC00204605F02CF9DB4B04F5CE721A60DA4B50
:1076BC0000221A70D94B04F2F2411960692323702D
:1076CC000323637140F20113A3604FF41673A4F803
:1076DC00F630FA23A4F8F830BC23A4F8F4304FF4B5
:1076EC00FA73A4F8FE30012384F8F23084F80E31DA
:1076FC0084F81631052384F89B3140F2DC53A4F84E
:10770C00283140F24C43A4F82A3140F26C73A4F8AF
:10771C002C3140F27533A4F82E3140F64303A4F813
:10772C0030312346202184F8FA106E2184F80C1194
:10773C000A2184F80D112B2184F80F11212184F8D2
:10774C001011232184F811114FF4C871A4F81211EF
:10775C00032ACCBF0121002102F1010283F832116E
:10776C0014BF1E217521122A83F8331103F1020371
:10777C00EED14FF4FA63A4F85831A4F85C31A4F8B4
:10778C006031A4F86431052384F87231C823A4F85D
:10779C00763140F27E43A4F8D43040F23A73A4F828
:1077AC00D63040F27E53A4F8DC3040F2EA53A4F811
:1077BC00DE3040F2B45340F2DC5001264FF47A77BD
:1077CC004FF0320A4FF01E094FF0190BA4F8E030BD
:1077DC004FF47A5384F8259184F873B1A4F8DA0045
:1077EC000190A4F8E2A0A4F8E430A4F8E6A0A4F870
:1077FC005671A4F85A71A4F85E71A4F8627184F8F9
:10780C00716184F8746184F8756184F87861A4F806
:10781C00D870FEF74BF97F4A002513684FF00F0E16
:10782C002674E673A573A58183F805E04FF0220E4C
:10783C0083F806E04FF00E0E83F810E04FF0350E93
:10784C00172183F81AE04FF0210E5975997583F8BA
:10785C0011E055214FF0530E4FF02808D97083F8E2
:10786C0007B02D2183F81BE000924FF05A0E6422D2
:10787C004FF00A0B4FF0780C83F80B9083F80C90B8
:10788C00597383F804A083F808E01A7783F80AC0C8
:10789C001D7083F8018083F80280DD759D731D7661
:1078AC00DD735D7683F812B083F8098019754FF497
:1078BC00FA71A3F84E103C2183F85110112183F872
:1078CC0050105749DFF878C19963D9635549C3F80B
:1078DC002CC099625449C3F830C0DFF868C15963B1
:1078EC004FF07F595149C3F82090C3F82490C3F846
:1078FC0048C001984FF04B0C4FF0000959649E772B
:10790C0083F85250C3F8409083F84CC084F8F2E4EA
:10791C004FF0410E84F8F3E484F8F4A4A4F8FC04CA
:10792C0084F8F55484F8F95484F8FA5484F8F6542D
:10793C0084F8F75484F8F85404201966152183F858
:10794C005C00A3F85850A3F85A50A3F8565083F88B
:10795C00648083F86810364983F86580D9663549A8
:10796C0083F878601967344934485967FEF7CFF8C3
:10797C00009A4FF44873D2F800A0AAF81631C82325
:10798C008AF811518AF812518AF813818AF8146115
:10799C008AF8185184F86931642384F868B1A4F822
:1079AC006A7184F86C51A4F86E31194C2B1910358E
:1079BC00C02DC3F81490F8D1514604F52E704FF435
:1079CC008E7204F091FF04F5757051464FF48E726F
:1079DC0004F08AFF114B1B681A68C4F8FE245A681D
:1079EC00C4F802259A68C4F806251A68C4F80A2552
:1079FC005A68C4F80E259A68012384F80C330223C4
:107A0C00C4F8122584F8283403B0BDE8F08F00BF09
:107A1C00000A0020EC070020DC160020E8070020FC
:107A2C008FC2F53C000060406666663F0000A040D7
:107A3C009A99193FF6287C3F3D0A773F85EA000862
:107A4C00CDCCCC3E0000404001480249B6E500BF19
:107A5C00000800409011002001480249AEE500BF2B
:107A6C0000040040681100204FF080400049A5E55B
:107A7C004011002001480249A0E500BF002C014044
:107A8C00181100200148024998E500BF002C014064
:107A9C0018110020254B10B55A43254B254C1B685B
:107AAC000139B3FBF2F20388013AA04289B292B2D7
:107ABC009BB212D004F50064A0420ED0B0F1804FFE
:107ACC000BD0A4F59834A04207D004F58064A042F2
:107ADC0003D004F58064A04202D123F070039BB262
:107AEC00154CA04206D004F58064A0421CBF23F4C0
:107AFC0040739BB203800F4B8185984202850FD057
:107B0C0003F5006398420BD003F54063984207D00D
:107B1C0003F58063984203D003F58063984201D14A
:107B2C00002303860123838210BD00BF40420F0057
:107B3C0038000020002C0140001000400C4B800A43
:107B4C0098420CD004D8B0F5801F0CD1012070479E
:107B5C00084B984205D04933984206D003E00220E6
:107B6C00704703207047FE2070470020704700BF0D
:107B7C0001001000020010002DE9F84304680746CC
:107B8C00204688469146FFF7D9FF03284BD8BA7A8E
:107B9C009108B8F1000F06D1A589AEB202258D402F
:107BAC0026EA0505A5810A2303FB00131F4A42F8A8
:107BBC002380043342F82390B8F1000F07D0BD7A2C
:107BCC00A189AD080223AB400B439BB2A3812823B0
:107BDC00434303F120011144EFF31286502585F342
:107BEC00128803F10C051C331544134455F8047F1B
:107BFC0017B10F60296804319D42F7D100230B6047
:107C0C00F3B283F31188282303FB0020036A23B10A
:107C1C00A3899BB243F0010304E0A38923F0010381
:107C2C001B041B0CA381BDE8F88300BF18110020B6
:107C3C0000482FE4C415002000482BE4181600203F
:107C4C000A4B4FF400525A604FF6FE730848D0F8B6
:107C5C00882011680B401360826FC36F9A4201D069
:107C6C0054307AE4012380F89830704700000240C9
:107C7C00C41500202DE9F04F85B002939B4B804634
:107C8C001C88019104F00204A4B2009294B1984BA8
:107C9C00B3F90240B3F90030002CB8BF6442002B9A
:107CAC00B8BF5B429C42B8BF1C46B4F5007FA8BF6E
:107CBC004FF40074C34600278D4B4FF0040E33F97C
:107CCC0017208C4B8C4933F917304FEA470A002B9D
:107CDC0093FBFEFEB8BF5B42B3F5206F4FEA420246
:107CEC004FEA870951F827000FDCCEEB020303445F
:107CFC00B3F57A5F8148A8BF4FF47A538342ACBF87
:107D0C0041F8273041F8270002E0002341F82730E2
:107D1C0051F809509BF80B309BF80160ED11734939
:107D2C005D4356430988AD1189074FEAA6133BD032
:107D3C00009949428A4203DB00999142A8BF11463F
:107D4C0042F210766E4A6F483AF90220891A029A6A
:107D5C0032F91720114459F800200A44B242A8BF46
:107D6C003246694EB242B8BF324649F8002098F804
:107D7C000800414398F81C00C91100EB8000C0F1C9
:107D8C00000C614503DB8142A8BF01468C4698F884
:107D9C001210CCEB03064A431213AD1A654366432B
:107DAC0002EB65250CEB6623584AD65D98F85120FA
:107DBC0006FB0EF6A3EBA61672B13046039201F049
:107DCC00F7F85349534B01EBC701039A1B68FCF7B7
:107DDC007BFE01F007FB064646494F4B3AF8010083
:107DEC003AF903E002B2CEEB02024FF0040E92FB22
:107DFC00FEF22AF803009E440C3359F80EC059F8D1
:107E0C00030049F80E206044104498F8502049F8BB
:107E1C0003C0894662B1039201F0CAF83F493D4B59
:107E2C0001EBC701039A1B68FCF74EFE01F0DAFA6E
:107E3C003B4B3C4ADB5D35445843A5EB60102AF8BC
:107E4C0002000BF1010B0FB9012735E7284B042475
:107E5C00B3F90410019B28489B7985680F335B00AC
:107E6C004B43B9F904105B1191FBF4F4002BA3EB19
:107E7C000404B8BF5B42322B98F80D100BDC01FBED
:107E8C000451294B8B42A8BF0B4628498B42ACBFEF
:107E9C008360816001E00023836098F8031001FB8C
:107EAC0004F323499B11097803290CD9B8F84E1017
:107EBC00B1F5FA7F07D24C42A34203DB8B42A8BF39
:107ECC000B4600E0234681686FF0FF0041F34F3111
:107EDC00B1F5807FA8BF4FF480718142ACBF5B18B5
:107EEC001B18938005B0BDE8F08F00BF88070020F9
:107EFC0028100020B20700205010002080C1FFFF86
:107F0C00D6070020A0100020F0D8FFFFA8100020FA
:107F1C00341000204C1000206C1600208010002023
:107F2C00C010002098100020FEFFFF0F020000F090
:107F3C00780700202DE9F04F87B00493994B4FF050
:107F4C00000BB3F90270B3F90030002FB8BF7F42B9
:107F5C00002BB8BF5B429F42B8BF1F468246D94632
:107F6C00D8465C46B7F5FA7F0392A8BF4FF4FA7770
:107F7C000190CDF808B08C4B198811F0030040D05B
:107F8C00022C3ED0874B650033F91420039B520022
:107F9C005B429A4203DB039B9342A8BF1346834A7E
:107FAC006FF00408AD5E049A5B1B32F91450642226
:107FBC001D449AF808306B4393FBF2F39AF81C209B
:107FCC0008FB02F8434504DB02EB82089845A8BF86
:107FDC009846774A52F824302B4442F21075AB4243
:107FEC00A8BF2B46734DAB42B8BF2B4642F824308A
:107FFC009AF81220012802FB03F34FEA2333029371
:10800C0041D0684B6C4D33F91490019BA00093F850
:10801C0001C06A4B55F824E033F9146086EAE67324
:10802C00A3EBE673B3F5206F1DDC022C15D05023A7
:10803C0003FB09F292FBFCF3042296FBF2F69E1B67
:10804C00B644BEF57A5F5E4BA8BF4FF47A5E9E4590
:10805C00ACBF45F800E02B5007E089EAE973A3EBCD
:10806C00E973642BE3DD00232B50534B4FF07D0C55
:10807C00C35893FBFCFC019BDB7A03FB0CF34FF026
:10808C00400C93FBFCFB8A0713D5022C11D007FB89
:10809C000BF607FB09F30299C7F5FA7202FB0833DA
:1080AC0002FB01624FF4FA7593FBF5F392FBF5F6C4
:1080BC0008E0CB0704D5022C02D0029E434601E017
:1080CC005E464B46620000923C4A042532F914206D
:1080DC0092FBF5F53B4AA25C55436FF04F0295FBC2
:1080EC00F2F59AF851201D44E2B1022C0592284673
:1080FC000BD100F05DFF059A530803D09A42A8BF3C
:10810C001A4600E00122304905E000F051FF2F49EA
:10811C00059A01EBC4012E4B1B68FCF7D5FC01F052
:10812C0061F90546254B009A0098D15A294B0AB2A1
:10813C00C05E121A042092FBF0F20098C15203F1B7
:10814C000801143351F824E053F8240041F824209A
:10815C00704410449AF8502043F824E062B1059220
:10816C0000F026FF1C491A4B01EBC401059A1B6851
:10817C00FCF7AAFC01F036F9184B35441B5D2026A0
:10818C00584390FBF6F0164B009A281AD052019BDC
:10819C0001340133032C01937FF4EDAE07B0BDE83D
:1081AC00F08F00BF2810002088070020D607002081
:1081BC00A0100020F0D8FFFF50100020B2070020C4
:1081CC0080C1FFFFA81000204410002034100020B4
:1081DC004C1000208016002080100020C0100020C1
:1081EC00981000202DE9F04F89B00593934B07466A
:1081FC001B880C469B0702924DD540F2E631129B30
:10820C008F4AD889B2F900301B1A03F2F3158D424C
:10821C0003D8002BB8BF5B4201E04FF4FA73B2F9FC
:10822C000220101A40F2E63200F2F311914203D808
:10823C000028B8BF404201E04FF4FA7097F84C5058
:10824C003DB39842B8BF1846C0F5FA7000F0B0FEC6
:10825C007C4900F0B5FF4FF07E5100F0F3FD06466F
:10826C00642090FBF5F000F0A3FE0146304600F0D0
:10827C00F3FE4FF07E5100F0E7FD0021064601F0C1
:10828C0089F830B930464FF07E5101F0A1F820B199
:10829C0001E0002601E04FF07E56E31C04930097AA
:1082AC000024049B620013F8015F022C04930392D8
:1082BC00654B09D1B3F904000A35684300F078FE28
:1082CC00624900F07DFF5DE033F91490484600F000
:1082DC006FFE8046029800F067FE5A4900F070FF6E
:1082EC000146404600F0B8FE029B8046584200F022
:1082FC005FFE82464046514601F04CF848B9029860
:10830C0000F056FE82464046514601F061F800B935
:10831C00C246039A4E4B985E00F04AFE0146504608
:10832C0000F090FD059B804633F9140000F040FEF0
:10833C000146404600F088FD464900F041FF3F4BA6
:10834C008246B3F8008018F0010F03D0796C00F06E
:10835C0083FE17E005F1140009FB00F000F028FE85
:10836C003A4900F02DFF18F0020F05460BD0B96CFE
:10837C00504600F071FE314600F06EFE0146284674
:10838C0000F062FD0546039A334BDFF8EC80985EF3
:10839C0000F00EFE314B596C00F05EFE0146284693
:1083AC0000F050FD009B8246196A00F055FE2C4BE4
:1083BC000546185D00F0FCFD0146284600F04CFE19
:1083CC00284900F0FDFE97F8512081469AB1022C05
:1083DC0009D1530803D09A42A8BF1A4600E00122E3
:1083EC004846214902E0214901EBC401D8F800308C
:1083FC00FCF76AFB8146D8F80030504619460193C9
:10840C0000F02AFE009BDFF874B0D96A00F024FE5D
:10841C00104900F021FE5BF8241000F015FD144902
:10842C00A500804600F0B6FF50BB4046114900F055
:10843C00CFFF38B3DFF83C8024E000BF8807002072
:10844C002C0900200000FA432810002000004842AC
:10845C00D607002000002041B20700206C16002037
:10846C00301000200000C8424410002034100020BE
:10847C0000007AC300007A434C100020CC1000207E
:10848C00DFF810814BF80580DFF80CB1504655F839
:10849C000B1000F0D7FC45F80BA0069001994FF09B
:1084AC007E5000F08DFE069B0146184600F0D4FD70
:1084BC0082460BF10C03EA580BF1180B104655F8D9
:1084CC000B100793069200F0BFFC514600F0BCFC69
:1084DC00069A079B45F80B2097F85020014645F863
:1084EC0003A032B12349019B01EBC401FCF7ECFA68
:1084FC0001460846204900F063FE009B996B00F092
:10850C00ABFD1E4B0546185D00F052FD014628469A
:10851C0000F0A2FD1A4900F053FE1A49054600F07E
:10852C0039FF30B92846184900F052FF10B1164DEA
:10853C0000E0144D4146484600F086FC294600F008
:10854C0083FC04F03BFB114BB0F57A7FA8BF4FF4D2
:10855C007A709842B8BF1846039A0D4B0134985262
:10856C00009B032C03F1040300937FF49AAE09B033
:10857C00BDE8F08F8010002000004040301000203B
:10858C000000C842000096C30000964318FCFFFF91
:10859C009810002000007AC3B4160020044B00226F
:1085AC001A605A60034B00221A605A60704700BF71
:1085BC00A0100020C410002010B50B4C0123E37058
:1085CC004FF48060022384F82030FCF78DFD074ABD
:1085DC00074BD26E1B685278642101FB0233636136
:1085EC0023880133238010BDF80F00206C16002067
:1085FC00F40F0020704707B5064B07490093074B53
:10860C00074A01930748084BFCF708FB03B05DF8D9
:10861C0004FB00BF53E90008AEEA00085CE900085F
:10862C00B4EA00088EEA000847E9000808B50378A8
:10863C0033B90C4B0C481978BDE80840FCF7EEBA7E
:10864C0004F0F6F902280CD8064B0C221870074BD4
:10865C0002FB0030064B02301860FCF72DFE05487B
:10866C00E5E708BDDC160020BBEA0008F00E002090
:10867C00E807002018E5000808B503783BB90B4B58
:10868C000B4893F8F014BDE80840FCF7C7BA04F0A7
:10869C00CFF9022808D8054B83F8F004FCF766FDE7
:1086AC00FCF72EFE0348E8E708BD00BF000A0020D7
:1086BC00BFEA000818E5000873B5037813B9FAF798
:1086CC0023FE3FE001AA204904F0E1F90024024610
:1086DC00264625469AB134B1012C08D1104604F037
:1086EC00A7F9064603E0104604F0A2F9054601AAD4
:1086FC000020154904F0CBF901340246EAE70B2DB2
:10870C0003D9124812490C230CE0022C11D1A6F506
:10871C007A73B3F57A7F08D90C480E494FF47A7204
:10872C004FF4FA63FCF77AFA0CE00B4B03EB4503BE
:10873C005E80094B094803EB45032946B3F9022037
:10874C00FCF76CFA02B070BDECE40008CCE6000853
:10875C00EBE60008A5EC0008DC160020CCEA0008CB
:10876C0010B50446054B2146D869FBF7F6FA044BC5
:10877C001B6898796040987110BD00BFDC16002012
:10878C007C07002010B50446C0B2FFF7E9FF200AB1
:10879C00BDE81040E4E737B58288836804461006CC
:1087AC000D4641BF29494FF48E7091F8F01400FB2F
:1087BC000133D10542BF26490C20097802F03F0253
:1087CC0048BF00FB0133042A12D006D8012A0DD071
:1087DC00022A2FD193F900102DE0102A0AD0202A5A
:1087EC000AD0082A26D1B3F9001024E0197822E027
:1087FC00198820E019681EE069461868FCF794F99E
:10880C0001461448FCF70AFAF5B1E06800F0D0FB19
:10881C006946FCF789F901460F48FCF7FFF9206916
:10882C0000F0C6FB6946FCF77FF901460A48FCF7E5
:10883C00F5F909E000210948FCF7F0F925B10848E1
:10884C00E1682269FCF7EAF903B030BD000A0020A8
:10885C00DC160020B6EB0008AFEB0008DFEA0008DE
:10886C00DBEA000810B5441E14F8011F21B1034BBC
:10887C00186AFBF772FAF7E710BD00BFDC16002090
:10888C0013B5164B16491C6891F82400154B164964
:10889C001A8851F82010154B15481B7800914FF48D
:1088AC007A71B4FBF1F1FCF7B9F9124B1248196863
:1088BC00124BB1FBF3F1FCF7B1F91148FFF7D2FF02
:1088CC00104B11481A88114B92B219884FF4A363BC
:1088DC0002B0BDE81040FCF7A1B900BFF40F0020B6
:1088EC00DC160020E00F0020BCD80008340000206B
:1088FC00E2EA00083800002025EB000840420F0097
:10890C0079EB00088207002035EB00088007002077
:10891C002DE9F0410024804625460F4E4146A759CB
:10892C00384604F06DF858B139460C48FCF776F926
:10893C0030190021FFF72FFF0948FFF793FF01358E
:10894C0040F6C82314349C42E7D11DB9BDE8F04170
:10895C00044887E7BDE8F081CCD80008B1E60008F0
:10896C0079EB000853E600082DE9F04F85B0054679
:10897C0004F009F8064620B1012818D12B782A2BCF
:10898C0015D19C48FFF76EFF00249B4D9B48615905
:10899C00FCF744F928193146FFF7FDFE9848FFF71C
:1089AC0061FF40F6C82314349C42EED11EE12846E8
:1089BC003D2103F0DAFF002800F0138103461A462C
:1089CC0013F8011D2029FAD0441C531B2046019397
:1089DC0004F02EF88346204602780346202A00F144
:1089EC000100F9D0092AF7D02D2A03D10346DFF86C
:1089FC00349204E02B2A08BF03464FF07E591E46E2
:108A0C000024324616F8011BA1F13007FBB2092BEA
:108A1C000DD87C49204600F01FFB0446384600F078
:108A2C00C7FA0146204600F00FFA0446E9E72E2962
:108A3C00134617D1734F334616F8010B3038C2B2B8
:108A4C00092A0FD800F0B4FA394600F0B9FB0146F8
:108A5C00204600F0F9F96B490446384600F0FCFA60
:108A6C000746E8E71A7802F0DF02452A39D15A782E
:108A7C002D2A02D10233012704E02B2A14BF013323
:108A8C0002330027013B002613F8012F303AD1B2F4
:108A9C00092903D80A2101FB0626F5E7B6F59A7FCA
:108AAC0028BF4FF49A76B0464FF07E53B8F1070FBB
:108ABC0007D91846544900F0CFFAA8F10808034624
:108ACC00F4E706F0070636B118464E4900F0C4FA32
:108ADC00013E0346F7E719462FB1204600F070FB24
:108AEC0004E04FF07E51204600F0B6FA0346002613
:108AFC0014247443454F039307F1100854F808A04D
:108B0C00504603F040FF8446514662462846CDF855
:108B1C0008C003F041FFDDF808C0039B002858D1C2
:108B2C009DF80420624554D11946484600F094FA49
:108B3C00A0443C440546E06900F03AFA0146284658
:108B4C0000F03CFC002842D0206A00F031FA0146CB
:108B5C00284600F029FC002839D0A38A9A0658BF71
:108B6C005D46142202FB06761C0648BF2848B269F3
:108B7C0042BF90F8F0044FF48E7404FB0022D80529
:108B8C0042BF24480C24007803F03F0348BF04FB89
:108B9C000022042B29460BD004D8013B012B0CD806
:108BAC0015700AE0102B05D0202B05D0082B04D112
:108BBC00118002E0156000E0156051461648FCF784
:108BCC002DF84046002105B0BDE8F04FE3E5134811
:108BDC0003E001368A2E8BD1114805B0BDE8F04F69
:108BEC0040E6284605B0BDE8F04F91E605B0BDE87B
:108BFC00F08F00BF67EB0008CCD80008B1E6000886
:108C0C0079EB00080000204120BCBE4CBCD8000809
:108C1C00000A0020DC1600207CEB000887EB000823
:108C2C0053E60008000080BFF0B585B0044603F0A1
:108C3C00AAFE082826D1621EE01D1F4912F8013F2A
:108C4C0009681944497801F00301022908BF203B47
:108C5C0082421370F1D1254604F1080715F8016B17
:108C6C001648314603F081FE20B12846314603F008
:108C7C007CFE10B1FAF748FB1CE0BD42EED1204659
:108C8C00FCF745FF0E48FFF7EDFD00230D4A04A944
:108C9C001A4492F81A210A440849595C0133082BEA
:108CAC0002F80C1CF2D10023074801A98DF80C30F6
:108CBC00FBF7B4FF05B0F0BD3C00002070EA0008E3
:108CCC00A7EB0008000A0020D7E7000838B50024FD
:108CDC000B4D60592544FFF7C5FD696811B1094872
:108CEC00FBF79CFFA96811B10748FBF797FF0748F2
:108CFC001034FFF7B7FDB4F5A87FE9D138BD00BF3C
:108D0C0094E30008ADEB0008B3EB000879EB000826
:108D1C0010B50A48FFF7A6FD094B1C6A2046FBF765
:108D2C0019F818B90A20FAF7B6FFF7E7FBF718F8A5
:108D3C00FCF7F2F9034A044BDA6010BDB9EB0008FA
:108D4C00DC1600200400FA0500ED00E008B505482B
:108D5C00FFF788FDFEF79EFCFCF708FABDE808401B
:108D6C00D6E700BFC5EB000808B50448FFF77AFD4D
:108D7C00FCF7FCF9BDE80840CAE700BFDBEB0008D4
:108D8C0013490B7813F0010F03F004021BD0F2B956
:108D9C001048006840011AD4980714D443F0040317
:108DAC000B700D4B4FF47A711A880C4B05201A80FE
:108DBC000B4B0C4A1B6892F8722101FB02330A4AD6
:108DCC001360FAF7FFBE12B90120FAF721BF704702
:108DDC00161700208C070020DA070020DE06002082
:108DEC00F40F0020000A002090060020054A13789A
:108DFC00590705D523F0040304201370FAF7E2BEDB
:108E0C00704700BF1617002008B5044B1B7803F001
:108E1C000503052B01D1FAF7A3FFFEE70417002089
:108E2C00D0400B1C1141203A03D49C4613411843EB
:108E3C006346524293401843704700BF80F0004095
:108E4C0002E000BF81F0004142001FBF5FEA410316
:108E5C0092EA030F7FEA226C7FEA236C6AD04FEA16
:108E6C001262D2EB1363C1BFD2184140484041405B
:108E7C00B8BF5B42192B88BF704710F0004F40F40D
:108E8C00000020F07F4018BF404211F0004F41F429
:108E9C00000121F07F4118BF494292EA030F3FD0F5
:108EAC00A2F1010241FA03FC10EB0C00C3F1200308
:108EBC0001FA03F100F0004302D5494260EB400097
:108ECC00B0F5000F13D3B0F1807F06D340084FEA02
:108EDC00310102F10102FE2A51D2B1F1004F40EBF7
:108EEC00C25008BF20F0010040EA0300704749005F
:108EFC0040EB000010F4000FA2F10102EDD1B0FA2A
:108F0C0080FCACF1080CB2EB0C0200FA0CF0AABF1E
:108F1C0000EBC25052421843BCBFD04018437047BC
:108F2C0092F0000F81F4000106BF80F400000132C2
:108F3C00013BB5E74FEA41037FEA226C18BF7FEA99
:108F4C00236C21D092EA030F04D092F0000F08BFDB
:108F5C000846704790EA010F1CBF0020704712F0C2
:108F6C007F4F04D1400028BF40F00040704712F101
:108F7C0000723CBF00F50000704700F0004343F066
:108F8C00FE4040F4000070477FEA226216BF08469C
:108F9C007FEA23630146420206BF5FEA412390EA5F
:108FAC00010F40F4800070474FF0000304E000BF55
:108FBC0010F0004348BF40425FEA000C08BF704706
:108FCC0043F0964301464FF000001CE050EA0102CA
:108FDC0008BF70474FF000030AE000BF50EA0102DF
:108FEC0008BF704711F0004302D5404261EB4101CC
:108FFC005FEA010C02BF84460146002043F0B643F1
:10900C0008BFA3F18053A3F50003BCFA8CF2083A15
:10901C00A3EBC25310DB01FA02FC634400FA02FC1E
:10902C00C2F12002BCF1004F20FA02F243EB020025
:10903C0008BF20F00100704702F1200201FA02FC87
:10904C00C2F1200250EA4C0021FA02F243EB02007A
:10905C0008BF20EADC7070474FF0FF0C1CEAD052BE
:10906C001EBF1CEAD15392EA0C0F93EA0C0F6FD07F
:10907C001A4480EA010C400218BF5FEA41211ED05D
:10908C004FF0006343EA501043EA5111A0FB013149
:10909C000CF00040B1F5000F3EBF490041EAD3711E
:1090AC005B0040EA010062F17F02FD2A1DD8B3F19A
:1090BC00004F40EBC25008BF20F00100704790F009
:1090CC00000F0CF0004C08BF49024CEA502040EA5B
:1090DC0051207F3AC2BFD2F1FF0340EAC250704721
:1090EC0040F400004FF00003013A5DDC12F1190F5F
:1090FC00DCBF00F000407047C2F10002410021FAD1
:10910C0002F1C2F1200200FA02FC5FEA310040F1E8
:10911C00000053EA4C0308BF20EADC70704792F061
:10912C00000F00F0004C02BF400010F4000F013A99
:10913C00F9D040EA0C0093F0000F01F0004C02BF94
:10914C00490011F4000F013BF9D041EA0C018FE703
:10915C000CEAD15392EA0C0F18BF93EA0C0F0AD009
:10916C0030F0004C18BF31F0004CD8D180EA01002F
:10917C0000F00040704790F0000F17BF90F0004FC8
:10918C00084691F0000F91F0004F14D092EA0C0FAA
:10919C0001D142020FD193EA0C0F03D14B0218BF3D
:1091AC00084608D180EA010000F0004040F0FE4083
:1091BC0040F40000704740F0FE4040F4400070471F
:1091CC004FF0FF0C1CEAD0521EBF1CEAD15392EA9E
:1091DC000C0F93EA0C0F69D0A2EB030280EA010C8E
:1091EC0049024FEA402037D04FF0805343EA111127
:1091FC0043EA10130CF000408B4238BF5B0042F185
:10920C007D024FF4000C8B4224BF5B1A40EA0C0029
:10921C00B3EB510F24BFA3EB510340EA5C00B3EB5B
:10922C00910F24BFA3EB910340EA9C00B3EBD10F49
:10923C0024BFA3EBD10340EADC001B0118BF5FEA9B
:10924C001C1CE0D1FD2A3FF650AF8B4240EBC250C4
:10925C0008BF20F0010070470CF0004C4CEA502085
:10926C007F32C2BFD2F1FF0340EAC250704740F4D4
:10927C0000004FF00003013A37E792F0000F00F0C6
:10928C00004C02BF400010F4000F013AF9D040EA44
:10929C000C0093F0000F01F0004C02BF490011F4D8
:1092AC00000F013BF9D041EA0C0195E70CEAD153D0
:1092BC0092EA0C0F08D142027FF47DAF93EA0C0FB7
:1092CC007FF470AF084676E793EA0C0F04D14B029B
:1092DC003FF44CAF08466EE730F0004C18BF31F04D
:1092EC00004CCAD130F000427FF45CAF31F0004347
:1092FC007FF43CAF5FE700BF4FF0FF3C06E000BFE0
:10930C004FF0010C02E000BF4FF0010C4DF804CD02
:10931C004FEA40024FEA41037FEA226C18BF7FEA12
:10932C00236C11D001B052EA530C18BF90EA010F14
:10933C0058BFB2EB030088BFC81738BF6FEAE170A3
:10934C0018BF40F0010070477FEA226C02D15FEA3F
:10935C00402C05D17FEA236CE4D15FEA412CE1D0AB
:10936C005DF8040B704700BF844608466146FFE772
:10937C000FB5FFF7C9FF002848BF10F1000F0FBD54
:10938C004DF808EDFFF7F4FF0CBF012000205DF84D
:10939C0008FB00BF4DF808EDFFF7EAFF34BF0120D2
:1093AC0000205DF808FB00BF4DF808EDFFF7E0FF6B
:1093BC0094BF012000205DF808FB00BF4DF808EDBC
:1093CC00FFF7D2FF94BF012000205DF808FB00BF1F
:1093DC004DF808EDFFF7C8FF34BF012000205DF801
:1093EC0008FB00BF4FEA4002B2F1FE4F0FD34FF023
:1093FC009E03B3EB12620DD94FEA002343F00043F6
:10940C0010F0004F23FA02F018BF404270474FF0A3
:10941C000000704712F1610F01D1420205D110F02A
:10942C00004008BF6FF0004070474FF000007047DD
:10943C0042000ED2B2F1FE4F0BD34FF09E03B3EBB2
:10944C00126209D44FEA002343F0004323FA02F0DE
:10945C0070474FF00000704712F1610F01D14202CA
:10946C0002D14FF0FF3070474FF00000704700BF43
:10947C007BB972B90029BEBF00204FF0004106E055
:10948C0008BF00281CBF6FF000414FF0FF3000F008
:10949C0075B882B0EC462DE9005000F03FF8DDF8CD
:1094AC0004E002B00CBC704710B500210446FFF775
:1094BC0071FF20B92046BDE8104000F009B804F156
:1094CC00004000F005F8404261EB410110BD00BFC7
:1094DC00D0B500F0B9F900220E4B06460F4600F04D
:1094EC0007FA00F017FC044600F08CF900220A4B36
:1094FC0000F0FEF902460B463046394600F044F8BF
:10950C0000F008FC2346002242EA000210461946ED
:10951C00D0BD00BF0000F03D0000F0412DE9F0414E
:10952C00069C904606460F461D4600F013FC08FBB1
:10953C0001FCA8FB002300FB05C5B21A2B4467EB0A
:10954C0003038646C4E90023BDE8F0812DE9F84306
:10955C00089E1746804689461D4600F051FD00FBCB
:10956C0005F3A0FB074507FB0137B8EB04043D44AA
:10957C0069EB0505C6E90045BDE8F883704700BFF7
:10958C0081F0004102E000BF83F0004330B54FEAA8
:10959C0041044FEA430594EA050F08BF90EA020F15
:1095AC001FBF54EA000C55EA020C7FEA645C7FEAA8
:1095BC00655C00F0E2804FEA5454D4EB5555B8BFCB
:1095CC006D420CDD2C4480EA020281EA030382EA3C
:1095DC00000083EA010180EA020281EA0303362DCE
:1095EC0088BF30BD11F0004F4FEA01314FF4801CA1
:1095FC004CEA113102D0404261EB410113F0004FB3
:10960C004FEA03334CEA133302D0524263EB430369
:10961C0094EA050F00F0A780A4F10104D5F1200E07
:10962C000DDB02FA0EFC22FA05F2801841F1000162
:10963C0003FA0EF2801843FA05F359410EE0A5F136
:10964C0020050EF1200E012A03FA0EFC28BF4CF067
:10965C00020C43FA05F3C01851EBE37101F000451D
:10966C0007D54FF0000EDCF1000C7EEB00006EEB2A
:10967C000101B1F5801F1BD3B1F5001F0CD34908B4
:10968C005FEA30004FEA3C0C04F101044FEA44520B
:10969C0012F5800F80F09A80BCF1004F08BF5FEA92
:1096AC00500C50F1000041EB045141EA050130BD72
:1096BC005FEA4C0C404141EB010111F4801FA4F115
:1096CC000104E9D191F0000F04BF01460020B1FA6A
:1096DC0081F308BF2033A3F10B03B3F120020CDAA2
:1096EC000C3208DD02F1140CC2F10C0201FA0CF080
:1096FC0021FA02F10CE002F11402D8BFC2F1200CE5
:10970C0001FA02F120FA0CFCDCBF41EA0C0190409A
:10971C00E41AA2BF01EB0451294330BD6FEA0404E3
:10972C001F3C1CDA0C340EDC04F11404C4F12002CE
:10973C0020FA04F001FA02F340EA030021FA04F3E0
:10974C0045EA030130BDC4F10C04C4F1200220FA37
:10975C0002F001FA04F340EA0300294630BD21FA75
:10976C0004F0294630BD94F0000F83F4801306BF3B
:10977C0081F480110134013D4EE77FEA645C18BF2F
:10978C007FEA655C29D094EA050F08BF90EA020FC6
:10979C0005D054EA000C04BF1946104630BD91EABE
:1097AC00030F1EBF0021002030BD5FEA545C05D1C1
:1097BC004000494128BF41F0004130BD14F5800400
:1097CC003CBF01F5801130BD01F0004545F0FE4174
:1097DC0041F470014FF0000030BD7FEA645C1ABFA9
:1097EC00194610467FEA655C1CBF0B46024650EAE0
:1097FC00013406BF52EA033591EA030F41F400210C
:10980C0030BD00BF90F0000F04BF0021704730B591
:10981C004FF4806404F132044FF000054FF0000166
:10982C0050E700BF90F0000F04BF0021704730B527
:10983C004FF4806404F1320410F0004548BF4042FC
:10984C004FF000013EE700BF42004FEAE2014FEA51
:10985C0031014FEA02701FBF12F07F4393F07F4F2C
:10986C0081F06051704792F0000F14BF93F07F4F5E
:10987C00704730B54FF4607401F0004521F00041A1
:10988C0020E700BF50EA010208BF704730B54FF027
:10989C0000050AE050EA010208BF704730B511F02C
:1098AC00004502D5404261EB41014FF4806404F164
:1098BC0032045FEA915C3FF4DCAE4FF003025FEAE6
:1098CC00DC0C18BF03325FEADC0C18BF033202EB6E
:1098DC00DC02C2F1200300FA03FC20FA02F001FAC8
:1098EC0003FE40EA0E0021FA02F11444C1E600BF67
:1098FC0070B54FF0FF0C4CF4E06C1CEA11541DBF1A
:10990C001CEA135594EA0C0F95EA0C0F00F0DEF8E4
:10991C002C4481EA030621EA4C5123EA4C5350EAC9
:10992C00013518BF52EA033541F4801143F480131A
:10993C0038D0A0FB02CE4FF00005E1FB02E506F0AB
:10994C000042E0FB03E54FF00006E1FB03569CF000
:10995C00000F18BF4EF0010EA4F1FF04B6F5007F06
:10996C0064F5407404D25FEA4E0E6D4146EB060678
:10997C0042EAC62141EA55514FEAC52040EA5E5001
:10998C004FEACE2EB4F1FD0C88BFBCF5E06F1ED8AB
:10999C00BEF1004F08BF5FEA500E50F1000041EBE2
:1099AC00045170BD06F0004646EA010140EA02008F
:1099BC0081EA0301B4EB5C04C2BFD4EB0C0541EAB1
:1099CC00045170BD41F480114FF0000E013C00F3C6
:1099DC00AB8014F1360FDEBF002001F0004170BDEA
:1099EC00C4F10004203C35DA0C341BDC04F1140403
:1099FC00C4F1200500FA05F320FA04F001FA05F28F
:109A0C0040EA020001F0004221F0004110EBD3705B
:109A1C0021FA04F642EB06015EEA430E08BF20EA87
:109A2C00D37070BDC4F10C04C4F1200500FA04F32A
:109A3C0020FA05F001FA04F240EA020001F00041BC
:109A4C0010EBD37041F100015EEA430E08BF20EA2F
:109A5C00D37070BDC4F1200500FA05F24EEA020E77
:109A6C0020FA04F301FA05F243EA020321FA04F0A6
:109A7C0001F0004121FA04F220EA020000EBD3705D
:109A8C005EEA430E08BF20EAD37070BD94F0000F5D
:109A9C000FD101F00046400041EB010111F4801F91
:109AAC0008BF013CF7D041EA060195F0000F18BF42
:109ABC00704703F00046520043EB030313F4801F7E
:109ACC0008BF013DF7D043EA0603704794EA0C0F38
:109ADC000CEA135518BF95EA0C0F0CD050EA41064E
:109AEC0018BF52EA4306D1D181EA030101F00041CB
:109AFC004FF0000070BD50EA410606BF10461946F3
:109B0C0052EA430619D094EA0C0F02D150EA0136FE
:109B1C0013D195EA0C0F05D152EA03361CBF10463F
:109B2C0019460AD181EA030101F0004141F0FE41DE
:109B3C0041F470014FF0000070BD41F0FE4141F462
:109B4C00780170BD70B54FF0FF0C4CF4E06C1CEA62
:109B5C0011541DBF1CEA135594EA0C0F95EA0C0F17
:109B6C0000F0A7F8A4EB050481EA030E52EA0335D2
:109B7C004FEA013100F088804FEA03334FF08055F3
:109B8C0045EA131343EA12634FEA022245EA111520
:109B9C0045EA10654FEA00260EF000419D4208BFD1
:109BAC00964244F1FD0404F5407402D25B084FEA7E
:109BBC003202B61A65EB03055B084FEA32024FF42A
:109BCC0080104FF4002CB6EB020E75EB030E22BF87
:109BDC00B61A754640EA0C005B084FEA3202B6EB47
:109BEC00020E75EB030E22BFB61A754640EA5C00F6
:109BFC005B084FEA3202B6EB020E75EB030E22BF86
:109C0C00B61A754640EA9C005B084FEA3202B6EB86
:109C1C00020E75EB030E22BFB61A754640EADC0045
:109C2C0055EA060E18D04FEA051545EA16754FEAA7
:109C3C0006164FEAC30343EA52734FEAC2025FEAC5
:109C4C001C1CC0D111F4801F0BD141EA00014FF054
:109C5C0000004FF0004CB6E711F4801F04BF014325
:109C6C000020B4F1FD0C88BFBCF5E06F3FF6AFAE41
:109C7C00B5EB030C04BFB6EB020C5FEA500C50F1D1
:109C8C00000041EB045170BD0EF0004E4EEA113154
:109C9C0014EB5C04C2BFD4EB0C0541EA045170BD5B
:109CAC0041F480114FF0000E013C90E645EA060E9F
:109CBC008DE60CEA135594EA0C0F08BF95EA0C0FCD
:109CCC003FF43BAF94EA0C0F0AD150EA01347FF415
:109CDC0034AF95EA0C0F7FF425AF104619462CE7EC
:109CEC0095EA0C0F06D152EA03353FF4FDAE10464F
:109CFC00194622E750EA410618BF52EA43067FF4A0
:109D0C00C5AE50EA41047FF40DAF52EA43057FF42F
:109D1C00EBAE12E74A0011D212F5001211D20DD59A
:109D2C006FF47873B3EB62520ED44FEAC12343F055
:109D3C00004343EA505323FA02F070474FF00000FF
:109D4C00704750EA013002D14FF0FF3070474FF0AE
:109D5C000000704700292DE9F043C0F2A8800026CE
:109D6C00002BC0F29E8081468E4690469C4617463C
:109D7C0004460D46002B3DD18A4259D9B2FA82F3E2
:109D8C003BB1C3F120029D4020FA02F29F401543E3
:109D9C009C40390CB5FBF1F01FFA87FE01FB105506
:109DAC000EFB00F3220C42EA0545AB4209D9ED1932
:109DBC0000F1FF3280F00B81AB4240F20881023897
:109DCC003D44ED1AB5FBF1F301FB13550EFB03FEFD
:109DDC00A4B244EA0545AE4508D9ED1903F1FF32AA
:109DEC0080F0F780AE4540F2F480023B43EA00433A
:109DFC00002203E08B420FD900221346341C18BFFB
:109E0C00012460424FF0000565EB4501584051407C
:109E1C0000196941BDE8F083B3FA83F2002A40F0DF
:109E2C0089808B4202D3804500F2E2800123E5E772
:109E3C0012B90123B3FBF2F7B7FA87F8B8F1000FA8
:109E4C003BD1ED1B4FEA174C1FFA87FE0122B5FBE5
:109E5C00FCF00CFB10550EFB00F3210C41EA054500
:109E6C00AB4207D9ED1900F1FF3102D2AB4200F23F
:109E7C00C3800846ED1AB5FBFCF30CFB13550EFB27
:109E8C0003FEA4B244EA0545AE4507D9ED1903F12A
:109E9C00FF3102D2AE4500F2AD800B4643EA0043DF
:109EAC00ACE752426FEA060663EB43035BE74042C2
:109EBC0061EB41014FF0FF3652E707FA08F7C8F1A2
:109ECC00200225FA02F34FEA174CB3FBFCF11FFA00
:109EDC0087FE0CFB113324FA02F205FA08F50EFB8F
:109EEC0001F92A43100C40EA0343994504FA08F49B
:109EFC0007D9DB1901F1FF3078D2994576D90239AF
:109F0C003B44C9EB0303B3FBFCF00CFB10330EFB1F
:109F1C0000F592B242EA03439D4207D9DB1900F1E6
:109F2C00FF325FD29D425DD902383B445D1B40EA53
:109F3C0001428CE7C2F1200328FA03F10CFA02FC6F
:109F4C0041EA0C0C4FEA1C402EFA03F1B1FBF0F580
:109F5C001FFA8CF700FB151129FA03F30EFA02FE17
:109F6C0007FB05F943EA0E0E4FEA1E4343EA014193
:109F7C00894508FA02F808D911EB0C0105F1FF33F9
:109F8C0032D2894530D9023D6144C9EB0101B1FBA4
:109F9C00F0F300FB131107FB03F71FFA8EFE4EEADA
:109FAC00014E774508D91EEB0C0E03F1FF3117D289
:109FBC00774515D9023BE64443EA0543A3FB0889E0
:109FCC00C7EB0E0ECE4509D305D0002216E710467E
:109FDC00F7E613460AE794404445F6D2013BF4E712
:109FEC000B46E9E71046A1E71D46CEE7014688E798
:109FFC00134603E7023B51E702383D443AE700BF02
:10A00C002DE9F043002B44D18A42154604464FD922
:10A01C00B2FA82F70E464FB1C7F12003B94020FACD
:10A02C0003F602FA07F50E4300FA07F42F0CB6FB01
:10A03C00F7F01FFA85FE07FB10620EFB00F1260CF1
:10A04C0046EA0243994209D95B1900F1FF3280F0CC
:10A05C00EE80994240F2EB8002382B44591AB1FB46
:10A06C00F7F307FB13110EFB03FEA4B244EA014104
:10A07C008E4508D9491903F1FF3280F0DA808E45FC
:10A08C0040F2D780023B43EA004000263146BDE84F
:10A09C00F0838B4247D8B3FA83F6002E48D18B421B
:10A0AC0002D3824200F2CF8001203146BDE8F0831A
:10A0BC0012B90125B5FBF2F5B5FA85FCBCF1000F20
:10A0CC0078D1491B2F0C1FFA85FE0126B1FBF7F046
:10A0DC0007FB10110EFB00F2230C43EA01418A42EC
:10A0EC0007D9491900F1FF3302D28A4200F2BC8031
:10A0FC001846891AB1FBF7F307FB13110EFB03FE8D
:10A10C00A4B244EA0142964508D9521903F1FF3131
:10A11C0080F09180964540F28E80023B43EA0040ED
:10A12C003146BDE8F083002630463146BDE8F08369
:10A13C00C6F1200422FA04F5B3402B4321FA04F7AC
:10A14C004FEA1348B7FBF8FC1FFA83F908FB1C779E
:10A15C0020FA04FE01FA06F509FB0CF44EEA05059B
:10A16C004FEA154E4EEA0747BC4202FA06F204D9F2
:10A17C00FF180CF1FF3168D38C463F1BB7FBF8F48A
:10A18C0008FB147709FB04F9ADB245EA0741894590
:10A19C0004D9C91804F1FF355DD32C4644EA0C44AC
:10A1AC00A4FB0223C9EB0101994249D345D02046B7
:10A1BC0000266BE7CCF1200405FA0CF521FA04F328
:10A1CC002A0CB3FBF2F61FFA85FE02FB163820FAB6
:10A1DC0004F701FA0CF10EFB06F90F433C0C44EAB0
:10A1EC000843994500FA0CF407D95B1906F1FF31C5
:10A1FC0038D2994536D9023E2B44C9EB0303B3FB45
:10A20C00F2F002FB10330EFB00F1BFB247EA03433E
:10A21C00994207D95B1900F1FF3721D299421FD916
:10A22C0002382B441746591A40EA06464EE71046A8
:10A23C0014E7134627E70B4670E7B0409042B6D2BE
:10A24C00601E002622E7304620E7BC4294D9ACF1D0
:10A25C00020C1F4491E789459FD9023C19449DE7A4
:10A26C003846DFE70E46C8E70238294441E700BF0D
:10A27C004FEA4102B2F1E04324BFB3F5001CDCF11C
:10A28C00FE5C0DD901F0004C4FEAC0024CEA507054
:10A29C00B2F1004F40EB830008BF20F00100704783
:10A2AC0011F0804F21D113F13872BCBF01F0004086
:10A2BC00704741F480114FEA5252C2F11802C2F1B8
:10A2CC00200C10FA0CF320FA02F018BF40F0010039
:10A2DC004FEAC1234FEAD32303FA0CFC40EA0C00EB
:10A2EC0023FA02F34FEA4303CCE77FEA625307D128
:10A2FC0050EA01331EBF4FF0FE4040F4400070475F
:10A30C0001F0004040F0FE4040F40000704700BFF8
:10A31C0019481A49026800608A4217D0002103E0EC
:10A32C00174B5B58435004311648174B42189A424E
:10A33C00F6D3164A02E0002342F8043B144B9A422F
:10A34C00F9D3FBF72AFD00F035F8FEE7114E124861
:10A35C0030601248016821F07061016041020160B7
:10A36C000F4C182020600F490F4808600F48D0F898
:10A37C0000D0406800470000F04F0020EFBEADDE7B
:10A38C00E8F6000800000020A8000020A80000202B
:10A39C0018170020181002400900000004000140AA
:10A3AC00140C0140000C01404434434400F0FF1FE6
:10A3BC00FEE700002DE9804893B0F5F7A1FEAF4C05
:10A3CC00AF4D23782E6833B1AE4B1B68F31A002BBC
:10A3DC00A4BF00232370FBF72BFF10B1AA4B002264
:10A3EC001A70AA4B1F683B0740F18A81A84B1B6867
:10A3FC001B7A062B00F27881DFE813F007000700C8
:10A40C003400D400100138013801A24B1A78002A0C
:10A41C0000F06A8100221A709F4B022293F800E030
:10A42C009E4B1B6893F800C09D4B93F800809D4891
:10A43C0002F10109835C43FA0EF303F00F03634549
:10A44C000CD20B2B9FBF815C10F8090001EA0801AC
:10A45C0000EB01219CBF944840F823100232102AD3
:10A46C00E5D108E1914B1A78002A00F03D810022D9
:10A47C001A708F4B8F4A93F802C093F803E0597807
:10A48C000CF0070041EA00210EF03F00400140EAC9
:10A49C00DC001160197950605879890093F806C076
:10A4AC0041EA9E1100F0010E41EA8E21916093F871
:10A4BC0007E00CF00F01C90141EA50010EF07F00DA
:10A4CC00D1600001197A40EA1C1093F809C04900C8
:10A4DC00106141EADE110CF0030093F80AE041EA46
:10A4EC0040215161D97A0EF01F008001C90040EA69
:10A4FC009C0041EA5E1193F80DC093F80EE0D16117
:10A50C00197B90610CF0070041EA00210EF03F002E
:10A51C00400140EADC001162D97B5062187C890052
:10A52C0093F811C041EA9E1100F0010E41EA8E2110
:10A53C00916293F812E00CF00F01C90141EA50014D
:10A54C000EF07F00000140EA1C10D162D97C106330
:10A55C0093F814C0490041EADE110CF0030093F8A3
:10A56C0015E041EA402151630EF01F00997D8001F6
:10A57C00DB7D40EA9C00C90041EA5E119063D8077C
:10A58C00D1634CBF40F21471AD21116499074CBFDB
:10A59C0040F21471AD2113F0080F516414BF032362
:10A5AC000123A2E0444A1378002B00F09D80002385
:10A5BC001370424ADFF828E1107841490EEB400C49
:10A5CC00B1F800809CF803909CF8041041EA092132
:10A5DC00884540F089809EF80110012904D081291A
:10A5EC0040F08380032300E00B46102884BF102129
:10A5FC001170344992F800E00022D0B2704501F19C
:10A60C00020172D211F802CC11F8010C40EA0C20B4
:10A61C00DFF8D0C02CF812000132EEE72A4B1A7882
:10A62C00002A61D000221A70284B1A789946A82A61
:10A63C005AD1DB7C002B57D1984609EB4803D878CC
:10A64C001B7903EB0020FEF7AFFC2149FEF7B8FDA8
:10A65C002049FEF7F7FBFEF7EBFE1F4B43F82800F3
:10A66C0008F10108B8F1080FE7D104E01B4B1A7888
:10A67C00D2B300221A70012337E000BF1F0600205E
:10A68C000C170020A800002020060020E80F002056
:10A69C00E40F0020810900201E0F0020180F00205D
:10A6AC001F0F00207109002074080020FE090020F3
:10A6BC00E5090020E4080020B5090020B8090020B5
:10A6CC00B6090020BC090020AE0900209909002021
:10A6DC00CDCCCC400080BB43A408002072080020E5
:10A6EC00B9090020C40800200023DA0741BF83F019
:10A6FC0002038E4A0121C3F3400344BF117023703F
:10A70C00780406D58A4A13790BB100211171874A56
:10A71C00137044F208033B403BB1844B1B7823B1CC
:10A72C0006F5C333824AA0331360F9070CD5804B6E
:10A73C009A7959798A421FBF0122227006F5C332D9
:10A74C00A0321CBF1A609971BA0409D50023794A4A
:10A75C0032F81320002A42F01C8001330C2BF6D166
:10A76C00724B734C1B7823B9734B1B68F31A002B79
:10A77C0004DBF7F7C7FC0123E37187E0A7687B1CB8
:10A78C00A360002F7CD16D4B1B681B0778D5E36849
:10A79C00F31A002B74DB06F5C336A03663696848E0
:10A7AC00E66098476648674B01461A78FBF71AFB38
:10A7BC0065480278560713D5E368A3613B466349A5
:10A7CC0000261944A1F806615D495E5A60495E5243
:10A7DC0006315E520233062BF1D122F004020270D4
:10A7EC0094F8283083B1564B58491A88B1F80601B1
:10A7FC00121A1A80B1F808015A88B1F80A11121A03
:10A80C005A809A88521A9A80A169494A002937D0ED
:10A81C00D36802F11C005B1A4E498B4202F12201F3
:10A82C001CD84D4AD36883F48043D3600023444A38
:10A83C0030F913E032F813205E0017B2BE45C4BFE6
:10A84C00DFF80CE12EF8132031F906E00133BE4598
:10A85C00BCBF424FF253032BE9D111E00023404E11
:10A86C00936130F9137031F9132001333A44022704
:10A87C0092FBF7F2032B26F8022FF2D1FAF7C8FE5F
:10A88C00A368012BC2BF2A4B00229A60F9F7DCF9AE
:10A89C002E4B2860DB6833F47F0304D0E36AC31AC1
:10A8AC00002BFFF68CAD236B214D0344E3622D4B43
:10A8BC002D481E682D4B5B68984730B91F4B1B68A1
:10A8CC0013F0020300F00884D6E0274895F83420F2
:10A8DC000146FBF787FA264B1B88002B00F0A08063
:10A8EC00AB6B05F13C071B78483503934FF0000820
:10A8FC001F4B4FEA4809B3F800A0BAF57A7F02BFA4
:10A90C0000233B602B61184B33F918003B68034460
:10A91C003B60FEF74DFB2B690133012B2B6129D1D9
:10A92C00002368602860AB604FE000BF2006002069
:10A93C00A800002050090020F40500208407002006
:10A94C00B8070020131700208E060020000A0020F4
:10A95C00C40000207FC3C90100100140CA000020C0
:10A96C00040B0020EC070020B2070020A0160020EA
:10A97C0010170020D5F800C006936146CDF810C022
:10A98C000590FEF75FFA069B83461846FEF710FB10
:10A99C0001465846FEF714FCDDF810C0014660462F
:10A9AC00FEF752FA0346059A19466860104604935E
:10A9BC00FEF748FA01465846FEF74EFBA968FEF72B
:10A9CC0043FA049BE8602B60A860CB4ADFF82CB3F9
:10A9DC000023BAF1010F29F8023029F80B30DFF807
:10A9EC004CA328D12869012807DD0138FEF7E0FACD
:10A9FC000146E868FEF7E4FB00E0002002F06CF989
:10AA0C00039A7AB104901046FEF7D2FA049B0146E1
:10AA1C001846FEF7DDFC28B14FF47A73AAF8003023
:10AA2C0000231CE03B684FF47A7203F5FA7393FB36
:10AA3C00F2F32BF8093008F10108B8F1030F07F114
:10AA4C00040705F114057FF453AFBAF80000012890
:10AA5C0001D1F9F7B7F8BAF80030013BDEE7A649A7
:10AA6C00A64831F8132030F81300121A21F81320DD
:10AA7C000133032BF3D121E7DFF8B492D4F89030F3
:10AA8C0009F19800984709F19805002800F0E0803A
:10AA9C009B4B9C4F1A7828462946FBF7A3F93B8819
:10AAAC00B846002B41D0D9F8A0000023B8F80020FC
:10AABC009549B2F5C87F04BF002241F823204FEA24
:10AACC00830935F913C051F80920DFF864E26244B8
:10AADC0041F80920002125F8131020F81310013338
:10AAEC00032BE3D13B88012B1CD1DEF8A4304FF4AF
:10AAFC00C87CC83393FBFCF30380DEF8A820C83273
:10AB0C0092FBFCF24280DEF8AC30804AC83393FBF7
:10AB1C00FCF312889B1A8380A6F85810A6F85A10DA
:10AB2C00FAF776FD3B88013B3B80794B1B68590754
:10AB3C007AD5784F3B88BE46322B13D1D4F8A0304F
:10AB4C001A88A4F8B0205A889B88A4F8B220A4F8DC
:10AB5C00B430B6F85830A4F8B630B6F85A30A4F879
:10AB6C00B83001E0002B3FD0D4F8A0900023BEF801
:10AB7C0000206949322A04BF002241F823204FEA01
:10AB8C00830C35F9130051F80C20DFF8A481024432
:10AB9C0041F80C20002225F8132029F8132001334A
:10ABAC00032B1146E3D13B88012B1AD15B4A0C20B5
:10ABBC0011705B4A1370F9F705F8B8F8B030A9F8C2
:10ABCC000030B8F8B230A9F80230B8F8B430A9F8AF
:10ABDC000430B8F8B630A6F85830B8F8B830A6F843
:10ABEC005A303B88013B3B804E4B1A78E2B1002235
:10ABFC001A70D4F8BC30322093FBF0F3D4F8A010C8
:10AC0C000B80D4F8C03093FBF0F34B80D4F8C430F5
:10AC1C0093FBF0F33D4800881B1A8B80A6F8582054
:10AC2C00A6F85A20FAF7F4FCD4F8A020B4F898301F
:10AC3C0011885B1AA4F898305188B4F89A305B1AD2
:10AC4C00A4F89A309288B4F89C309B1AA4F89C30E3
:10AC5C00F8F7FAFFD4F8C8700546C31B18460393DF
:10AC6C00FEF7A2F9D4F8CC1004900026FEF7F4F904
:10AC7C00C4F8C8503546D4F8D0802B4F98F800B0A3
:10AC8C0005901D4A0DF1240932F91500FEF790F9D3
:10AC9C000599FEF7E1F949F82500BBF1000F4BD0FF
:10ACAC005846FEF785F901464FF07E50FEF788FABC
:10ACBC000246DFF880A011464FF07E500792FEF757
:10ACCC00C1F85AF82510FEF7C7F9AAF13C01069015
:10ACDC0031F91500FEF76CF9079A1146FEF7BCF92D
:10ACEC00DDF818C001466046FEF7AEF84AF82500BC
:10ACFC00FEF778FB788023E0B20700202C010020BF
:10AD0C00121700209A0600204C0100201E00002083
:10AD1C00E80F00209C060020640100209E06002005
:10AD2C009706002098060020AA0700201017002084
:10AD3C00A80000207C010020AD4A32F815207A8052
:10AD4C0037F9022F0135032D02FB026699D1DFF88A
:10AD5C00DCA264235E43BAF80030A6485B4396FB42
:10AD6C00F3F6493E09A9B6B2FAF75AF93B2ED8F8D0
:10AD7C00045010D9A04EB6F9EC00FEF719F9D6F82C
:10AD8C00E85001462846FEF723FB9C4B70B31A781B
:10AD9C0042F008022DE04FF07E512846FEF754F8A1
:10ADAC0001464FF07E50FEF70BFA06464FF0000BB3
:10ADBC00904B284653F82B100693FEF74DF990490B
:10ADCC00059031F91B00FEF7F3F8059A0146104681
:10ADDC00FEF73AF83146FEF73FF9069B43F82B0095
:10ADEC000BF1010BBBF1030FE2D1C3E71A7822F090
:10ADFC0008022946D4F8E4001A7001F06BFF814D6B
:10AE0C00D4F8E0302860D4F8E400D4F8E820014607
:10AE1C0003F1004B0692FEF71FF9069A05901146B6
:10AE2C001046FEF719F9059B01461846FEF70CF87B
:10AE3C0001F052FF0146584601F04CFF7249686020
:10AE4C002868FEF709F901F0B9FEDFF8E4B16E49A4
:10AE5C00ABF800006868FEF7FFF801F0AFFE6B4B33
:10AE6C00ABF802001B681A0732D5694809A9FAF732
:10AE7C00D7F8D8F808904FF07E514846FDF7E4FF1C
:10AE8C0001464FF07E50FEF79BF907464FF0000B42
:10AE9C005F4A484652F82B100692FEF7DDF85D49E2
:10AEAC00059031F91B00FEF783F8DDF814C001465C
:10AEBC006046FDF7C9FF3946FEF7CEF8069A42F810
:10AECC002B000BF1010BBBF1030FE1D1104641E05C
:10AEDC00DFF844B149465846FAF7A2F8DBF800000F
:10AEEC00DBF80830DBF80420014605930692FEF7E8
:10AEFC00B3F8069A814611461046FEF7ADF80146A6
:10AF0C004846FDF7A1FF059B814619461846FEF7FA
:10AF1C00A3F801464846FDF797FF01F0DDFE00213E
:10AF2C008146FEF72DFAA0B9DBF800004946FEF782
:10AF3C0047F94946CBF80000DBF80400FEF740F96E
:10AF4C004946CBF80400DBF80800FEF739F9CBF8DA
:10AF5C0008003148FBF74EFF304B314918800498FC
:10AF6C00FEF77AF82B68814603F100430C936B686B
:10AF7C00234D03F100430D93284BB3F90000FEF76A
:10AF8C0017F8284900F10040FEF766F80E90B5F965
:10AF9C000000FEF70DF80F90B5F90200FEF708F867
:10AFAC001090B5F90400FEF703F80CA911900FA846
:10AFBC00FAF736F898F80130012B3BD11A4B1B7875
:10AFCC005B070ED4D6F8FC00402390FBF3F3C01AB9
:10AFDC00FDF7EEFF1199FDF737FFFEF703FAC6F800
:10AFEC00FC00D6F8FC00402390FBF3F024E000BFFB
:10AFFC004001002088010020A80000208E060020BF
:10B00C00AC070020B81100204C3D0F4484070020F1
:10B01C0098010020B807002000000020DA0700206B
:10B02C00BD37863535FA8E3C161700201E000020E1
:10B03C00D6070020BAF80000FDF7BAFF01461198B8
:10B04C00FDF700FFD4F8041111904846FDF7FCFE03
:10B05C0001464846FEF7B4F8D4F800510646294696
:10B06C001198FDF7EFFE01463046FDF7F5FF01465E
:10B07C002846FDF7E9FE0646C4F800010F9801F0DA
:10B08C009DFDD4F808512978F9F7C8FED4F80C3195
:10B09C001844C4F80C01109801F090FD2978F9F7C8
:10B0AC00BDFED4F810311844C4F81001304601F03C
:10B0BC0085FD6978F9F7B2FED4F81431C24A184408
:10B0CC0003991368C4F814011944D4F818311160A9
:10B0DC000133C4F8183105E0A4F89830A4F89A307C
:10B0EC00A4F89C30F8F7B0FDB84DB94BDFF82083CD
:10B0FC001860D5F81C31C5F81C01C31A9BB2A8F80E
:10B10C0000301846FDF750FFB249FDF7A5FFB24CD1
:10B11C00B24F2368386093F85230AA46A3462BB935
:10B12C00AF4B1B7C002B00F0868027E0D5F820016C
:10B13C000021FEF725F938B1286BFDF735FFA5493D
:10B14C00FDF78AFFC5F820010026DFF8C89239F90F
:10B15C001600FDF72DFFDBF80030A24993F85220C2
:10B16C0001EBC601DAF82031F9F7AEFCFEF73AF93B
:10B17C0029F816000136032EE7D1D1E7934EB8F823
:10B18C000000FDF711FF3B6806F5A0710122B5F830
:10B19C003C91F9F799FCFEF74BF980B2B9FBF0F052
:10B1AC00EB79471CBFB2A5F8487113B3B6F94A91B5
:10B1BC000023864E8C4A06F5A67838F9131006F54E
:10B1CC00AA7E09FB01F132F813C03EF813202EF8C9
:10B1DC0013C0C2EB0C0A3AB291FBF2F2524428F8BB
:10B1EC0013200133042BE4D10023F371A6F84A0198
:10B1FC0004E0B6F84A31013BA6F84A31B5F94A01E8
:10B20C00724A00284FF0000313DDB2F94851774918
:10B21C00A1F1080232F9132031F81310424392FBCA
:10B22C00F5F28A1A704921F813200133042BEED160
:10B23C0001E0A2F84A316C4BB3F906106C4BD3F811
:10B24C0000E00493BEF80A2091420FDBB1F5FA6FCF
:10B25C009EF80750BFBF8B1A6B43A2F5FA6593FBA0
:10B26C00F5F5ACBFC5F16405643500E064255C4BB5
:10B27C002268B3F828C193F9F23005929BB21646B6
:10B28C000693002240F2E630574B4FEA420933F95D
:10B29C001280CCEB080303F2F314844203D8002B86
:10B2AC00B8BF5B4201E04FF4FA73022A03934FF0EC
:10B2BC006400059B2ED093F811412CB1039BA34243
:10B2CC00CCBF1B1B00230393039B4A4C93FBF0F74F
:10B2DC006FF0630B34F817A00BFB073B013734F905
:10B2EC0017400FFA8AF7E41B04FB0BF494FBF0F401
:10B2FC00414B544423F809400EEB02042479039B80
:10B30C0063433E4C93FBF4F364339BB26B4393FB6C
:10B31C00F0F030E093F812412CB1039BA342CCBF68
:10B32C001B1B00230393039B284C93FBF0F06FF043
:10B33C00630A0AFB003B04EB400704EB4000B7F93F
:10B34C005C71B0F95E01069BC01B00FB0BFB9BFB09
:10B35C00FAFBC7EB0B0B0BFB03FB274BA3F804B05F
:10B36C00039B9EF80600002BB8BF5B424343234867
:10B37C0093FBF0F0643073786427434393FBF7F34B
:10B38C001F4C022AA354F37A1E4C00FB03F393FBCD
:10B39C00F7F3A354737D184C00FB03F090FBF7F00C
:10B3AC00194B9854194B37D1E0459F7037DBDFF8B8
:10B3BC0030B0BBF82A215D4691423CDBB1F5FA6F07
:10B3CC00A8BF4FF4FA6137E008170020A80000204E
:10B3DC000C170020BD378635EC0700204C100020E0
:10B3EC00000A0020CC0100202C090020FC010020C8
:10B3FC00E807002032070020281000200CFEFFFF79
:10B40C00A810002012020020C010002030100020D4
:10B41C0080070020B2070020E0459D5404DA34F880
:10B42C0009305B4224F809300132032A06F1010687
:10B43C007FF428AFBBE71146891A4FF47A7359434E
:10B44C00C2F5FA62B1FBF2F1642791FBF7F2DFF877
:10B45C00B4E26FF063033EF8120003FB02110132F9
:10B46C003EF9122003B2D21A514391FBF7F3034475
:10B47C00E380944B944E1B885F063FD5934A944BC4
:10B48C0010881B88181A00B2FDF792FD9149FDF740
:10B49C00E3FD91490746FDF7D7FCF9F7CEFC804652
:10B4AC003846F9F7CAFC0746B6F90200FDF780FDED
:10B4BC008146B6F90000FDF77BFD41468246FDF75B
:10B4CC00CBFD394603904846FDF7C6FD039B01466C
:10B4DC001846FDF7B7FCFDF785FF4146308048461E
:10B4EC00FDF7BAFD394680465046FDF7B5FD0146DD
:10B4FC004046FDF7A9FCFDF775FF7080774B1B6884
:10B50C009E0772D545F20721754B764E1A68D6F810
:10B51C007031D31A8B4268DDDFF8DC81C6F87021FC
:10B52C00FAF734FD98F800306F4F032B3B8822D18B
:10B53C000A2B2CD90023282088F80030F8F7ABFB15
:10B54C00FAF724FD694B1888FAF70AFD684B1A685C
:10B55C00D37890FBF3F001300828664BA8BF082085
:10B56C001870537980B24343A6F874311379584359
:10B57C00A6F876010BE00A2B09D803235D4A88F85C
:10B58C00003000231370A6F87431A6F8763198F8C1
:10B59C000030594A012B0CD002D3022B1CD024E0D2
:10B5AC00B6F874213B889A421FDD012388F80030DD
:10B5BC0010E03988B6F876318B4202DD0223137025
:10B5CC0010E0484BB3F874310133994202DD00238B
:10B5DC0013700AE0082006E0B6F876313A88013399
:10B5EC009A42E2DC0720F8F7EDFA3C4B434E1A681E
:10B5FC0012F4006F00F0A680394B3A481968D0F865
:10B60C007831C3EB010845F20723984540F39A8043
:10B61C00DFF8DCE0B4F90670DEF800A04FF47A73C2
:10B62C009AF80AE0C0F87811BEF1010F98FBF3F814
:10B63C00BBF8E210A7F57A77DFF8CC9004D065D38D
:10B64C00BEF1020F1BD064E0D0F87C21082792FBDE
:10B65C00F7F1521AC0F87C2192FBF7F240F6E4475E
:10B66C0092B27A430021A0F88011BAF80810C1EB0D
:10B67C0012325343BAF9062093FBF2F347E03078C9
:10B68C00BAF808304007C9F8003042D51C48059379
:10B69C000392F8F76BFA039A059B18B912F0100F86
:10B6AC0018BF002707FB07F2322192FBF1F2174477
:10B6BC00BAF9062057434FF47A7297FBF2F73B44E2
:10B6CC0025E000BF8807002028100020DE0600209F
:10B6DC00DA07002035FA8E3CDB0FC93FE80F00205B
:10B6EC000C170020A8000020E00F0020500F0020B5
:10B6FC004C0F0020340000200017002016170020EB
:10B70C001A0B00201A070020E40700200023C9F8B8
:10B71C000030D9F80020984F02FB08F8D7E9000157
:10B72C004FF47A7298FBF2F810EB080241EBE873D5
:10B73C0010461946914A0023C7E90001FDF798FE0F
:10B74C008F4B1860DFF88892D9F80030DB0402D5F3
:10B75C000A20F8F737FADFF87C82D8F80020002AA4
:10B76C0045D0DFF874A28749DAF8003009689942AD
:10B77C003DD8854B854F18785168B0B901221A70A5
:10B78C003B88CB5CD3B1824B1A70FAF75DFD3B88DA
:10B79C00A3B9D8F800301B78053B012B0ED8F8F76D
:10B7AC0053FA7C4BC3F8900108E000221A703B88D6
:10B7BC00CB5C1BB1764B1A70FAF746FDD8F800300B
:10B7CC003A885B6871499B5CFE2B02D100230B808D
:10B7DC000DE0FF2B02D1F8F7E3F908E0DAF80000EE
:10B7EC000A2707FB03036748013203600A8033789A
:10B7FC005F0704D5684B4FF480425A6135E0D9F8A5
:10B80C000020D0075EBF654943F001030B70644B09
:10B81C001B7819075EBF337823F001033370D30212
:10B82C0042BF337823F0010333705E4B1A88584BB8
:10B83C001AB15D4A1268970702D45C4A128832B179
:10B84C0002221A70337823F00103337004E031784C
:10B85C00C80758BF02221A70F8F7F6F9544B1B6848
:10B86C00C01A002801DBFAF7EFFC524B1F78039348
:10B87C00002F00F0F380504B1A680493002A00F05C
:10B88C00BE85049B186803685B689847002800F025
:10B89C00B685494B494D186803689B689847092839
:10B8AC00014601D03F285BD14FF000082F68454678
:10B8BC00DFF8289137B14248D9F800103A4601F028
:10B8CC006BF810B9C84605B94D463E4B09F1100945
:10B8DC009945EFD3EDB1D5F80090D8F800A0374AD0
:10B8EC00136819F803E01AF80300704511D13449B4
:10B8FC0050B92D2B08D803F1010EC2F800E020221C
:10B90C00CA5401F80E0004E001F803E0013313609F
:10B91C00E5E72A4BDFF8A0A01A6899460AB145451D
:10B92C0012D02948FCF79EFF454509D855F8100B55
:10B93C00FCF798FFDAF800000921F8F70EFAF3E7A4
:10B94C002248FCF78FFF0027D9F800309F4298D28D
:10B95C001B4BDAF80000D95DF8F7FFF90137F3E774
:10B96C002B68002B40F02B85042840F043871448AB
:10B97C00F7F7ECFB00F043BD30020020407E0500E1
:10B98C00DC07002044070020400700204807002067
:10B99C001C100020A80000200010014016170020E9
:10B9AC008E0600209A060020840700201017002025
:10B9BC002010002015170020FC1600201007002076
:10B9CC00E0060020E4E40008E4E40008E9E40008F0
:10B9DC008C0700204C070020F40F002094E3000893
:10B9EC00059BDFF844A3186803685B68984758B355
:10B9FC00DAF8000003689B689847C84B81461B68BF
:10BA0C0093F84810002938D124286FD1012283F8EB
:10BA1C004820DFF80893D9F8003093F84820062A1C
:10BA2C00DED193F84900F8F7ECF9002800F0878094
:10BA3C00DFF8E882D8F800309879FCF791FED8F856
:10BA4C000030002283F84820B54B93F83032002B9D
:10BA5C0040F0A3844C37982F00F0D184B14AD3190D
:10BA6C0093F84A100129F5D1DFF8B082BA58C8F81A
:10BA7C000030AD4B1A600593B2E7012904D14D2873
:10BA8C0014BF00220222C2E7022904D13C2814BFB1
:10BA9C0000220322BBE703290AD140284FF0000201
:10BAAC009FBF1A71DA715871987198BF0422AEE772
:10BABC00042908D19A7983F8490080EA020983F8AD
:10BACC0006900522A3E70529A3D159791A79914249
:10BADC00997906D941409971511C19711344187206
:10BAEC0097E781420CBF0622002290E733788F49FA
:10BAFC005B078ED42328DAF8003013D10691039912
:10BB0C0001220A708A4A8B481360854AC2F82C328B
:10BB1C00FCF7A8FE8848FCF7A5FE06990B7843F0C5
:10BB2C0002030B70854B1B681B784B4501BF844A85
:10BB3C00844B1A60844A04BF844BDA6069E7D9F8F5
:10BB4C00002092F849304C2B00F09A8359D8372BAF
:10BB5C0000F0E28317D8292B00F05C8309D8252B41
:10BB6C0000F02E83272B00F03783232B40F01A860E
:10BB7C002DE2332B00F0BE83352B00F060822D2B91
:10BB8C0040F0108657E3412B00F0B98309D83C2BC9
:10BB9C0000F010813E2B00F00081392B40F0028622
:10BBAC0027E3442B00F0F0834A2B00F0FF80432B5B
:10BBBC0040F0F885F8F7F6FE0023AB60F8F7FCFED2
:10BBCC008046F8F7F9FEAB6808EB00400343AB6026
:10BBDC00F8F7E8FE85F82201F8F7EEFEA5F8EC0080
:10BBEC00F8F7EAFEA5F8EE00F8F7E6FEA5F8F00087
:10BBFC00F8F7E2FEA5F81201F8F7DEFEA5F814013D
:10BC0C00C6E3D02B00F0BA8247D8CC2B00F056827A
:10BC1C0008D8C82B77D0CA2B00F0DA804E2B40F016
:10BC2C00C1853AE3CE2B00F0BD8240F2B282F8F728
:10BC3C00C3FE6FF4AF6E00EB0E039BB2C62B98BF26
:10BC4C00A5F82801F8F7B8FEA5F8D400F8F7B4FE6B
:10BC5C00A5F8D600F8F7B0FEA5F8D800F8F7ACFEBA
:10BC6C00A5F86A01F8F79EFEF8F79CFEF8F79AFE25
:10BC7C00F8F798FE85F81701F8F794FE85F824017B
:10BC8C00F8F790FE324BD3F80080F8F795FE00EBF6
:10BC9C0080004000A8F85600ABE2D62B00F0628280
:10BCAC0008D8D32B2AD0D42B00F07283D22B12D0ED
:10BCBC0000F078BDEF2B61D005D8D82B40F0728501
:10BCCC004FF0000816E1F22B00F06283FA2B00F023
:10BCDC00738200F067BD337803F0040303F0FF08B0
:10BCEC00002B40F05583F8F75DFE022885F8F00430
:10BCFC0040F24A82174B83F8F08445E2F8F75CFE79
:10BD0C00154B188044E392F805804FEA5808B8F1B7
:10BD1C00120F23D9F9F76AFF3AE300BF7C07002022
:10BD2C00A80000203C020020F81600201617002066
:10BD3C00FC16002019E50008E9E4000814070020AF
:10BD4C00EFBEADDEF04F00200400FA0500ED00E080
:10BD5C00EC070020000A0020DC0600204FF0000950
:10BD6C00C14507D2F8F728FEC94B23F8190009F191
:10BD7C000109F5E7C74B01221A7109E3DFF81883B3
:10BD8C00D8F80090F8F718FEA9F85A00D8F80080F7
:10BD9C00F8F712FEA8F85800FAE2F8F703FE85F857
:10BDAC007201F8F7FFFD85F87101F1E2F8F704FE76
:10BDBC00A881EDE2DFF8E082D8F80090F8F7F2FD08
:10BDCC0089F80000D8F800301878FBF787F8DFE224
:10BDDC00B14B1A6898461278022A6ED14FF00008BF
:10BDEC00DFF8B49208F1080AD9F800300593F8F797
:10BDFC00D9FDFDF7D9F8A949FDF7E2F9059B43F800
:10BE0C002A00D9F800A0F8F7CDFD08F10A030AEBD7
:10BE1C00830AFDF7C9F8A249FDF7D2F9D9F8003029
:10BE2C00CAF804000593F8F7BDFDFDF7BDF89D4970
:10BE3C00FDF7C6F908F10E0A059B08F10108B8F1E7
:10BE4C00030F43F82A00CBD1B8F1070FD9F800A0A3
:10BE5C001AD1F8F7A7FDFDF7A7F89049FDF7B0F94F
:10BE6C00CAF84400D9F800A0F8F79CFDFDF79CF83F
:10BE7C008A49FDF7A5F9CAF84800D9F800A0F8F7E7
:10BE8C0091FD8AF84C0012E0F8F78CFDC2448AF858
:10BE9C000100D9F800A0F8F785FDC2448AF80B0020
:10BEAC00D9F800A0F8F77EFDC2448AF8150008F115
:10BEBC000108B8F10A0FC7D16AE24FF00009D8F8AF
:10BECC0000A0F8F76FFDCA448AF80100D8F800A06A
:10BEDC00F8F768FDCA448AF80B00D8F800A0F8F708
:10BEEC0061FDCA4409F10109B9F10A0F8AF815007C
:10BEFC00E5D14DE2DFF8A09108F1080AD9F800303D
:10BF0C000593F8F759FDFDF74FF86649FDF758F919
:10BF1C00059B43F82A00D9F800A0F8F74DFD08F16D
:10BF2C000A030AEB830AFDF73FF85E49FDF748F96F
:10BF3C00D9F80030CAF804000593F8F73DFDFDF779
:10BF4C0033F85849FDF73CF908F10E0A059B08F146
:10BF5C000108B8F1030F43F82A00CBD1B8F1070F51
:10BF6C00D9F800A01AD1F8F727FDFDF71DF84D49B7
:10BF7C00FDF726F9CAF84400D9F800A0F8F71CFD23
:10BF8C00FDF712F84749FDF71BF9CAF84800D9F834
:10BF9C0000A0F8F711FD8AF84C0012E0F8F70CFD40
:10BFAC00C2448AF80100D9F800A0F8F705FDC24494
:10BFBC008AF80B00D9F800A0F8F7FEFCC2448AF806
:10BFCC00150008F10108B8F10A0FC7D1E0E1F8F744
:10BFDC00E9FC132882463FF69DAEDFF8BC90D9F8F9
:10BFEC000080F8F7DFFC00232F490C2202FB031220
:10BFFC00117A81421FD1137808EB8A0888F87930BE
:10C00C00F8F7D0FC88F87A00F8F7CCFC88F87B00BD
:10C01C00F8F7C8FC254A264B88F87C001A60D9F83A
:10C02C000000244B18607930F9F762FD224B80F048
:10C03C0001001870ACE101331C2BD5D16AE6F8F77E
:10C04C00B1FC0B2881463FF665AE134BD3F800804C
:10C05C00F8F7A8FC03283FF65DAE062303FB09881E
:10C06C0088F8CE00F8F79EFC88F8C900F8F79AFC1F
:10C07C0088F8CA00F8F796FC88F8CB00F8F792FC21
:10C08C0088F8CC00F8F78EFC88F8CD0080E100BF72
:10C09C002C090020A8000020EC0700200000204103
:10C0AC000000C84200007A4434D70008D40A0020AB
:10C0BC00D4060020D80600201C0000205379092B40
:10C0CC007FF628AE049BD3F80080F8F76BFC049B3A
:10C0DC0088F80000D3F80080F8F764FC88F80100B9
:10C0EC00F8F760FC049B64281B68A8BF64201871D7
:10C0FC00F8F758FC049B64281B68A8BF642058718F
:10C10C00F8F750FC049BFF281B68A8BFFF20987110
:10C11C00F8F748FC049B6428D3F8008028BF6420FF
:10C12C0088F80700F8F73EFC049B88F80200D3F867
:10C13C000080F8F737FC049B88F80300D3F80080E4
:10C14C00F8F73AFCD9F80030A8F80A005B790A2B0A
:10C15C0040F21E81C84BD3F80080F8F723FC88F816
:10C16C00080015E18046F8F727FCC44B23F81800AB
:10C17C0008F10108B8F1080FF5D109E13378580737
:10C18C0000F10681FBF786FAF8F7F0FFF9F7B8F83B
:10C19C00FEE03378590700F1FB80B94B4FF4C872BD
:10C1AC001A80F5E033785A0700F1F280B54A13781B
:10C1BC0043F004031370EBE033785B07E4D5F1E252
:10C1CC00A860F8F7F9FB8046F8F7F6FBAB6808EBCC
:10C1DC0000400343AB60DBE0F8F7EEFBA5F8EC00A6
:10C1EC00F8F7EAFBA5F8EE00F8F7E6FBA5F8F00087
:10C1FC00CEE0F8F7D7FB85F80C01F8F7D3FB85F800
:10C20C001001F8F7CFFB85F80F01F8F7CBFB85F899
:10C21C001101BDE0F8F7D0FBA5F81201F8F7CCFB43
:10C22C00A5F81401F8F7BEFB85F81601F8F7C4FB66
:10C23C00A5F81801ACE0F8F7B5FB85F82201F8F782
:10C24C00BBFBA5F82C01F8F7B7FBA5F82801F8F70C
:10C25C00B3FBA5F82A01F8F7A5FBD8F8003085F850
:10C26C0023015B79DFF85492082B40F29180F8F7A8
:10C27C00A3FBA9F82E01F8F79FFBA9F8300187E082
:10C28C00F8F790FB85F86801F8F78CFB85F86901E5
:10C29C00F8F792FBA5F86A017AE092F8058003237F
:10C2AC00B8FBF3F8B8F1120F3FF634ADDFF80C928F
:10C2BC004FF0000AC2456BD2F8F774FB89F83201D3
:10C2CC00F8F77AFB40F2ED23984205DD40F6CA03FD
:10C2DC009842A8BF184601E040F2EE20A0F2EE20F2
:10C2EC00192390FBF3F00AF1010A89F8330109F1E3
:10C2FC000209DFE7F8F756FB85F8240148E0804691
:10C30C00F8F750FB05EB080308F10108B8F1080F2A
:10C31C0083F81A01F4D13BE053794FF00709B3FBD2
:10C32C00F9F9C9EBC9029B1A13F0FF0F7FF4F2ACB9
:10C33C005FFA89F909F1FF395FFA89F9B9F1FF0F51
:10C34C0026D0F8F72FFB5FFA80FA4FFA8AF0F7F74E
:10C35C00D3F9804600283FF4DDAC80F800A0F8F754
:10C36C002BFBA8F80200F8F71DFB88F80400F8F77F
:10C37C0019FB88F80500F8F715FB88F80700F8F7A3
:10C38C0011FB88F80600D5E73F4B012283F83022D9
:10C39C000020F7F733FDFFF74BBB3C4BF858F7F792
:10C3AC00D9FC18B93220F7F776FCF6E7F7F7D8FC8A
:10C3BC00F8F7B2FE364A374BDA60FFF74BBB0C2866
:10C3CC0000F01A820A2940F02082334F3348FCF7E0
:10C3DC0049FA3846232100F0C8FA08B1C01B28607E
:10C3EC002B68002B40F037822B602B480021302229
:10C3FC0000F085FA039B1B78002B40F00082284B41
:10C40C009B680BB127489847274B284D1B6813F0A6
:10C41C00080F56D0A188264A01F145039BB28A2BFE
:10C42C001288244B4CD824480088470748D51B88D1
:10C43C00D21A92B293B218B2B330BCBF02F5B47335
:10C44C009BB210481AB2B32A0078C4BFA3F5B473D8
:10C45C009BB200079BF8F22033D552B252425343A1
:10C46C002A681BB2527A53436FF01D0293FBF2F30E
:10C47C000B44A38025E000BFE8070020DE16002057
:10C48C009A0600208E060020A80000203C02002006
:10C49C000400FA0500ED00E0E006002079EB00084E
:10C4AC00A0160020DA02002084070020EC070020F0
:10C4BC00DA070020DC06002088070020000A002094
:10C4CC001A80BA4B1B7843B1B94BB3F90620BBF8B1
:10C4DC002A319A42DCBF0023A3802B68B54F93F816
:10C4EC001881B8F1000F4FD0B34B1B889B074BD072
:10C4FC00D7F8E000D7F8E43001460393FCF7ACFD25
:10C50C00039B824619461846FCF7A6FD0146504689
:10C51C00FCF79AFCD7F8E890824649464846FCF767
:10C52C009BFD01465046FCF78FFC00F0D5FB014605
:10C53C004846FCF745FEA1498146FCF735FFF8B9A2
:10C54C00484600F077FBD7F83412FCF785FD00F075
:10C55C0035FBB0F5617FA8BF4FF46170FCF728FD87
:10C56C009749FCF72DFEF8F768FC81464046FCF72E
:10C57C001FFD4946FCF770FD00F020FB80B200E087
:10C58C000020E3881844E0808E4B2868BBF8FE201E
:10C59C0000938D4B1D688D4B196800F15803A8470B
:10C5AC008B4B8C491D78032D1AD9D7F83832B3F838
:10C5BC0002E0BEF5FA7F13D2B4F90400B1F904C05D
:10C5CC0080EAE078A8EBE078CEF10002C8EB020339
:10C5DC009C4504DB0EEB08036345A8BF63468B80C8
:10C5EC00B4F806B0B1F80280B1F80090D7F8387200
:10C5FC00B1F904A0784C0023AB4204F110043DD2F5
:10C60C000FFA8BF00493FCF7D3FC54F8181CFCF7CE
:10C61C0023FD03900FFA88F0FCF7CAFC54F8101CA9
:10C62C00FCF71AFD039A01461046FCF70DFC03902B
:10C63C000FFA89F0FCF7BCFC54F8141CFCF70CFD49
:10C64C00039A01461046FCF7FFFB039097F9010093
:10C65C0040420AFB00F0FCF7ABFC54F80C1CFCF756
:10C66C00FBFC039A01461046FCF7EEFBFCF7BAFE06
:10C67C00049B5A4A22F813000133BDE7327802F0CA
:10C68C00040202F0FF03002A79D0554B012193F8E4
:10C69C000380524B1A88A94214B207D233F91120E5
:10C6AC0001319442B8BF1446A2B2F4E74D49DFF809
:10C6BC0040E10968DEF800E0488803EB4505844258
:10C6CC00C8BF101A484AC8BF80B21468384A04F46C
:10C6DC008059B2F90660374AD8BF0020D2F8FC72F4
:10C6EC00D2F838C23D4A04F01004AA423DD0138857
:10C6FC001B1A9BB222F8023B1BB2B9F1000F0CD0F3
:10C70C00B7F80EA05645C7BFBEF802A0B1F802B0EC
:10C71C00B1F804A0BEF800B006E0B1F802B0B8F170
:10C72C00000F0AD0B1F804A0534503DB5B45A8BF4A
:10C73C005B469A4622F802ACD7E7B1F800A0534505
:10C74C0003DB5B45A8BF5B469A4622F802AC3B8AEA
:10C75C009E42CADA0CB18B8804E09CF80030002BA6
:10C76C00C3D10B8822F8023CBFE7124B93F800337D
:10C77C00002B3DF424AEFAF7C9FAFDF720BEAB420C
:10C78C00F3D21A4A32F81310144A22F81310013358
:10C79C00F5E701232370074A06F5C333A033136072
:10C7AC00FDF7DEBFF9F722FAFFF742B91C000020B3
:10C7BC002C090020A8000020880700208FC2753C9F
:10C7CC00EFB6B0441A0B002030000020E807002020
:10C7DC007807002098100020EC020020BE070020F3
:10C7EC00F80F002074070020E80F0020DE16002050
:10C7FC00700700200C2804D13148FCF733F831487D
:10C80C000EE07F2913D1FFF73CB80D293FF4DDADC5
:10C81C007F2909D12C4A013B00212C482B60D15493
:10C82C00FCF720F8FFF72DB82F2B3FF62AA8A1F123
:10C83C002002D2B25E2A3FF624A813B920293FF475
:10C84C0020A85A1C2A60204AD154214B1868F7F7AB
:10C85C0084FAFFF716B85A1EB95C202901D1134689
:10C86C00BFE5194A00212B60D1541A4B1A4DD3F84D
:10C87C0000902968DFF850A00846059100F083F875
:10C88C00074605993A46504600F086F8134A28B9EF
:10C89C001AF807304B445B78590703D01035954292
:10C8AC00E7D306E0954204D2781CEB6850449847D5
:10C8BC0002E00B48FBF7D6FF0A4B00221A6094E506
:10C8CC00EEE40008E9E40008E006002015E50008A5
:10C8DC00FC1600203C00002094E30008E4E400086F
:10C8EC00F9E400081007002010B5431E0A449142D9
:10C8FC0004D011F8014B03F8014FF8E710BD0346C3
:10C90C000244934202D003F8011BFAE7704700007F
:10C91C000D4B30B51D6810F8013BEA18527802F047
:10C92C000302012A11F8012B08BF2033AC186478DC
:10C93C0004F00304012C08BF20329B1A01D1002AF9
:10C94C00E9D1184630BD00BF3C000020024610B5AE
:10C95C0013461C780132002CFAD1013B11F8012B43
:10C96C0003F8012F002AF9D110BDC9B2034610F803
:10C97C00012B1AB18A42F9D11846704700290CBF15
:10C98C00184600207047034613F8012B002AFBD1F0
:10C99C00181A0138704700000F4B70B51E680A4416
:10C9AC00914216D010F8013BF418647804F003049B
:10C9BC00012C11F8014B08BF203335196D7805F0A7
:10C9CC000305012D08BF20341B1B03D1002CE7D11C
:10C9DC0000E00023184670BD3C000020034610B553
:10C9EC0032B111F8014B013A03F8014B002CF7D18D
:10C9FC001A44934203D0002103F8011BF9E710BD40
:10CA0C0030B5037823B90B78002B18BF002030BD4C
:10CA1C0003461A7801303AB100228C5C34B19D5C2B
:10CA2C00A542F5D10132F8E7104630BD184630BDAD
:10CA3C0000210A2200F0B4B8F0B548B9106838B932
:10CA4C00F0BD17F8016B5EB1B542FAD12BB120469F
:10CA5C0004460F4614F8015BF3E714600370F0BD55
:10CA6C004DB915602846F0BD17F8016BAE4207D0E2
:10CA7C00002EF9D11C4623460F4613F8015BF3E751
:10CA8C0015B10021217000E02B461360F0BD01238D
:10CA9C00FFF7D2BF2DE9F0470F46404CD4F8009079
:10CAAC003D4615F801EB09EB0E04667806F0080418
:10CABC0004F0FF060CB12F46F2E774462D2C03D17F
:10CACC00BD1C7C78012603E02B2C04BF7C78BD1C9C
:10CADC0013B1102B0AD15AE0302C56D12C7804F01B
:10CAEC00DF04582C4CD16C7810230235002E14BF67
:10CAFC004FF000486FF00048B8FBF3FA0027BE4631
:10CB0C0003FB1A8809EB040C9CF801C01CF0040F01
:10CB1C0001D0303C0BE01CF0030C1BD0BCF1010F1E
:10CB2C000CBF4FF0370C4FF0570CCCEB04049C426D
:10CB3C0010DAB7F1FF3F0AD0D64506D801D14445EB
:10CB4C0003DC03FB0E4E012701E04FF0FF3715F815
:10CB5C00014BD7E77C1C73460AD1002E4FF0220103
:10CB6C0014BF4FF000436FF0004301602AB911E08D
:10CB7C000EB1CEF100036AB107B1691E116009E074
:10CB8C003024002BB2D10823B0E70A23AEE7302CB7
:10CB9C00ACD1A3E71846BDE8F08700BF3C000020ED
:10CBAC0030B505460C461346034A29461068224602
:10CBBC00BDE83040FFF76EBFA000002030B5C0F3D9
:10CBCC00C755A5F17F021E2A83B0014621DC501CFB
:10CBDC001CDB162A4FEAD1740ADDC1F3160343F4A9
:10CBEC000003963DAB4060424340181903B030BD82
:10CBFC000F4B53F824502846FCF726F90190019866
:10CC0C002946FCF71FF920F0004333B9002003B08C
:10CC1C0030BDFCF7E7FB03B030BDC0F31603C0F327
:10CC2C00C75043F40003C0F19600C340DBE700BFDC
:10CC3C00A4F6000870B58AB0064600F09BF8224DA9
:10CC4C00044695F90030013303D0304600F000FC67
:10CC5C0010B920460AB070BD304600F0F5FB4FF01D
:10CC6C007E51FCF7B5FB0028F3D0184901220023B4
:10CC7C003046009208930191FCF7E6FD02460B4604
:10CC8C001348CDE90423CDE9022300F0C1FA95F94C
:10CC9C000030CDE90601022B0BD0684600F0B6FA45
:10CCAC0038B1089B53B9DDE90601FDF7E1FA0AB08A
:10CCBC0070BD00F0E7FB21230360F2E700F0E2FB1C
:10CCCC00089B0360EFE700BFA4000020ACF600084F
:10CCDC00B4F6000800F0B6B970B58AB0064600F09C
:10CCEC0041FA224D044695F90030013308D0304604
:10CCFC0000F0AEFB20B130460021FCF74BFB10B925
:10CD0C0020460AB070BD1A49012200233046019119
:10CD1C0000920893FCF798FD2C78CDE90401CDE93D
:10CD2C0002017CB900220023CDE90623684600F0FD
:10CD3C006DFA88B1089BA3B9DDE90601FDF798FAF5
:10CD4C000AB070BD0020002102460B46FCF7FAFE2B
:10CD5C00022CCDE90601E9D100F094FB21230360FC
:10CD6C00E8E700F08FFB089B0360E5E7A4000020D8
:10CD7C00B8F60008F8B520F00043B3F17E5F044626
:10CD8C0010D008DCB3F17C5F11DAB3F10C5F00F367
:10CD9C0084809D48F8BD0146FCF754F80146FCF729
:10CDAC000FFAF8BD002840F3CD800020F8BD002814
:10CDBC00C0F2CA8001464FF07E50FCF743F84FF0AA
:10CDCC007C51FCF749F9044600F0CCF98F49064632
:10CDDC002046FCF741F98E49FCF736F82146FCF762
:10CDEC003BF98C49FCF72EF82146FCF735F98A49BA
:10CDFC00FCF72AF82146FCF72FF98849FCF722F8B2
:10CE0C002146FCF729F98649FCF71EF82146FCF768
:10CE1C0023F9844905462046FCF71EF98249FCF7A4
:10CE2C0011F82146FCF718F98049FCF70DF821465A
:10CE3C00FCF712F97E49FCF705F82146FCF70CF9D2
:10CE4C004FF07E51FCF700F801462846FCF7B8F984
:10CE5C003146FCF701F926F47F6525F00F050746EE
:10CE6C0029462846FCF7F8F801462046FBF7EAFF6E
:10CE7C00294604463046FBF7E7FF01462046FCF7FF
:10CE8C009FF901463846FBF7DFFF01462846FBF7C2
:10CE9C00DBFF0146FBF7D8FFF8BD0146FCF7DCF8D9
:10CEAC0005465A49FCF7D8F85949FBF7CDFF2946F6
:10CEBC00FCF7D2F85749FBF7C5FF2946FCF7CCF82D
:10CECC005549FBF7C1FF2946FCF7C6F85349FBF758
:10CEDC00B9FF2946FCF7C0F85149FBF7B5FF2946C5
:10CEEC00FCF7BAF84F4906462846FCF7B5F84E4908
:10CEFC00FBF7A8FF2946FCF7AFF84C49FBF7A4FF5A
:10CF0C002946FCF7A9F84A49FBF79CFF2946FCF790
:10CF1C00A3F84FF07E51FBF797FF01463046FCF724
:10CF2C004FF901462046FCF797F801464148FBF7BC
:10CF3C0089FF01462046FBF785FF01463E48FBF77B
:10CF4C0081FFF8BD3D48F8BD4FF07E51FBF77CFFEB
:10CF5C004FF07C51FCF780F804462C49FCF77CF828
:10CF6C002B49FBF771FF2146FCF776F82949FBF7B3
:10CF7C0069FF2146FCF770F82749FBF765FF21464E
:10CF8C00FCF76AF82549FBF75DFF2146FCF764F8CE
:10CF9C002349FBF759FF2146FCF75EF8064620466D
:10CFAC0000F0E0F81F4905462046FCF755F81E49ED
:10CFBC00FBF748FF2146FCF74FF81C49FBF744FFF1
:10CFCC002146FCF749F81A49FBF73CFF2146FCF7D0
:10CFDC0043F84FF07E51FBF737FF01463046FCF724
:10CFEC00EFF82946FCF738F81249FBF72BFF0146FE
:10CFFC002846FBF729FF0146FBF726FF01461048A0
:10D00C00FBF720FFF8BD00BFDB0FC93F08EF11385D
:10D01C00047F4F3A4611243DA80A4E3E90B0A63EDE
:10D02C00ABAA2A3E2EC69D3D6133303F2D570140A1
:10D03C0039D119406821A233DA0FC93FDB0F4940BF
:10D04C00DA0F4940F8B521F00044B4F1FF4F034624
:10D05C0014DC20F00046B6F1FF4F07460EDCB1F1B0
:10D06C007E5F3AD08D1705F0020545EAD07556B9AA
:10D07C00022D30D0032D2BD13148F8BD084619466E
:10D08C00FBF7E2FEF8BDFCB1B4F1FF4F29D0B6F1CD
:10D09C00FF4F19D0341BE4153C2C1ADC002938DB6B
:10D0AC001846FCF78DF800F0CFF900F0B7F8012D19
:10D0BC002CD0022D22D0002D2FD02249FBF7C4FEFC
:10D0CC002149FBF7BFFEF8BD002F15DB1F48F8BD4B
:10D0DC00F8BD1E48EBE71C48F8BDBDE8F84000F071
:10D0EC009DB8B6F1FF4F19D0022DF4D0032DC3D04B
:10D0FC00012D1BD00020F8BD1548F8BD1149FBF7D8
:10D10C00A3FE01461048FBF79DFEF8BD00F1004060
:10D11C00F8BD3C34C4DA0020C9E7F8BD022D0CD0B0
:10D12C00032D08D0012D04D00A48F8BD4FF0004063
:10D13C00F8BD0948F8BD0948F8BD0948F8BD00BF5D
:10D14C00DB0F49C02EBDBB33DB0F4940DB0FC93FA2
:10D15C00DB0FC9BFDB0F493FDB0F49BFE4CB16C068
:10D16C00E4CB164020F00042B2F1FF4F70B50346FD
:10D17C0004462DD25AB300283DDBB2F5000F4FEA1E
:10D18C00E0502CD3002631467F38C3F31603C20778
:10D19C0043F4000348BF5B0040105B0019244FF0C0
:10D1AC0080728D189D4202DC5B1BA9181644013C51
:10D1BC004FEA43034FEA5202F3D113B106F00103D5
:10D1CC001E44761006F17C5606EBC05070BD70BD47
:10D1DC000146FBF741FF2146FBF736FE70BD14F408
:10D1EC0000020FD15B00190202F10102FAD5C2F163
:10D1FC0001021044C6E70146FBF724FE0146FBF78B
:10D20C00DFFF70BD01221044BCE700BF0020704757
:10D21C0000200149704700BF0000F87F2DE9F04164
:10D22C0020F00045B5F1A14F0446064608DBB5F1E8
:10D23C00FF4F6FDC002840F3A0806F48BDE8F08101
:10D24C006E4B9D4277DCB5F1445F68DB4FF0FF37E6
:10D25C0021462046FBF700FF01468046FBF7FCFE0B
:10D26C0005466749FBF7F8FE6649FBF7EDFD2946D5
:10D27C00FBF7F2FE6449FBF7E7FD2946FBF7ECFEF2
:10D28C006249FBF7E1FD2946FBF7E6FE6049FBF737
:10D29C00DBFD2946FBF7E0FE5E49FBF7D5FD414679
:10D2AC00FBF7DAFE5C4980462846FBF7D5FE5B4966
:10D2BC00FBF7C8FD2946FBF7CFFE5949FBF7C2FD2A
:10D2CC002946FBF7C9FE5749FBF7BCFD2946FBF77E
:10D2DC00C3FE5549FBF7B6FD2946FBF7BDFE7B1C8B
:10D2EC00014640464CD0FBF7AFFD2146FBF7B4FEA0
:10D2FC004E4B4F4D53F82710FBF7A4FD2146FBF77F
:10D30C00A1FD014655F82700FBF79CFD002E30DBF4
:10D31C00BDE8F0810146FBF797FDBDE8F08145497A
:10D32C00FBF792FD4FF07E51FCF752F800288DD0A0
:10D33C002046BDE8F08100F087F83F4B04469D4243
:10D34C0029DCA3F5D0039D4244DC0146FBF77CFDB0
:10D35C004FF07E51FBF776FD4FF08041054620469D
:10D36C00FBF772FD01462846FBF72AFF002704460F
:10D37C006EE700F10040BDE8F0813048BDE8F08177
:10D38C00FBF762FD2146FBF767FE01462046FBF7E3
:10D39C0059FDBDE8F0812A4B9D4214DC4FF07F51C2
:10D3AC00FBF750FD4FF07F5105462046FBF754FE2E
:10D3BC004FF07E51FBF748FD01462846FBF700FF76
:10D3CC000227044644E701461E48FBF7F9FE0327F3
:10D3DC0004463DE74FF07E51FBF734FD4FF07E5194
:10D3EC0005462046FBF730FD01462846FBF7E8FED4
:10D3FC00012704462CE700BFDB0FC93FFFFFDF3ED0
:10D40C00D769853C59DA4B3D356B883D6E2EBA3D5C
:10D41C002549123EABAAAA3E21A215BD6BF16E3D69
:10D42C0095879D3D388EE33DCDCC4C3EC0F6000833
:10D43C00D0F60008CAF24971FFFF973FDB0FC9BF56
:10D44C00FFFF1B40000080BF20F00040704700BF72
:10D45C0030F0004001D102207047A0F50003B3F179
:10D46C00FE4F01D204207047054B421E9A4201D850
:10D47C0003207047A0F1FF40B0FA80F040097047DC
:10D48C00FEFF7F00014B1868704700BFA000002012
:10D49C000000000000000000010203040607080958
:10D4AC00001001400040100200100140002010024A
:10D4BC00001001400080100228D500081CD500087F
:10D4CC001AD5000818D500080000803F000080BF66
:10D4DC000000803F000080BF0000803F000080BF44
:10D4EC00000080BF0000803F0000803F0000803FB4
:10D4FC000000803F0000803F0000803F0000803F24
:10D50C00000080BF000080BF08001402FFFFFFFF77
:10D51C00000106030D0307030C03FFFF00020102C9
:10D52C00020203020802090206030D0307030C039F
:10D53C00FFFF000000540040000C01404000800040
:10D54C001F2000000000200000580040000C01408B
:10D55C00000400082122000000004000010001022C
:10D56C000001030001040001050001060001070091
:10D57C00010800010900010A00010B00010C010364
:10D58C000D00010E00010F0001100001110001122D
:10D59C00000113000114000178E800087FE800087E
:10D5AC0084E8000895E800089FE80008AAE800084D
:10D5BC00B5E80008C0E80008C4E80008CDE8000899
:10D5CC00D3E80008DDE80008EBE80008EEE8000806
:10D5DC00FEE8000805E900080EE9000818E9000853
:10D5EC0020E900082BE9000834E9000800000000DD
:10D5FC0061687300000103030102000000000000D9
:10D60C0080250000004B00000096000000E10000A7
:10D61C0000C201000084030090D003000100000050
:10D62C00FCD6000802010000E9D600080302000045
:10D63C00E6D6000804030000E1D60008050400004B
:10D64C00DCD6000806050000D3D60008070600004B
:10D65C00D0D6000808070000CDD600080908000045
:10D66C00500700200A090000CAD600080C0A000066
:10D67C00C5D600080D0B0000C0D600080E0C00002B
:10D68C00B1D600080F0D0000500700200B0E000053
:10D69C00ADD60008100F0000A8D6000800F50A054A
:10D6AC00FF00640AFF0405040508050F05080504BE
:10D6BC00050405FF140F2305FF05050505FF0A0AE0
:10D6CC00FF1932FF3202FF05050F0505050F1EFF7E
:10D6DC001E050505FF0F050F05FF3232FF0A0A0A6A
:10D6EC000A0A28280A280A28280A0A0A0A0A46FFC7
:10D6FC00140A140A140AFF00524F4C4C3B50495464
:10D70C0043483B5941573B414C543B506F733B5042
:10D71C006F73523B4E6176523B4C4556454C3B4DDC
:10D72C0041473B56454C3B000000000064E90008B3
:10D73C00000000000100000069E900080100000081
:10D74C000200000070E90008020000000300000065
:10D75C0079E9000803000000040000007FE90008DC
:10D76C00050000000500000084E900080600000028
:10D77C00060000008EE9000807000000070000000A
:10D78C0097E900080800000008000000A0E9000864
:10D79C000900000009000000A9E900080A000000C7
:10D7AC000A000000B3E900080B0000000B000000A9
:10D7BC00BDE900080C0000000C000000C7E90008DF
:10D7CC000D0000000D000000CFE900080E00000065
:10D7DC000E000000D7E900080F0000000F00000049
:10D7EC00DFE900081000000010000000E8E9000864
:10D7FC001100000011000000EFE900081200000009
:10D80C0012000000F9E900081300000013000000EA
:10D81C0001EA000814000000140000000CEA0008E3
:10D82C00150000001500000016EA000816000000A4
:10D83C00160000001DEA0008170000001700000089
:10D84C0025EA000818000000180000002DEA000866
:10D85C00190000001900000035EA00081A00000049
:10D86C001A0000003FEA00081B0000001B0000002B
:10D87C0000000000FF0000005CE9000853E900080C
:10D88C0047E9000800000000010203040102030440
:10D89C0006070809020406089D7500084B75000868
:10D8AC000575000857760008357500085176000894
:10D8BC0083F5000886F500088EF5000897F500083A
:10D8CC0014EE0008440000000C0A002000000000C8
:10D8DC00A00F00001DEE0008410000000F0A002000
:10D8EC0000000000010000002FEE000841000000C5
:10D8FC000E0A002000000000010000003DEE0008B0
:10D90C0041000000100A002000000000010000008F
:10D91C004AEE000844000000280B0020B004000070
:10D92C00A406000051EE0008440000002A0B002061
:10D93C0000000000D00700005BEE0008440000006F
:10D94C002C0B002000000000D007000065EE000842
:10D95C0042000000240B0020000000001200000018
:10D96C0072EE000841000000250B002001000000B1
:10D97C00FF0000007DEE000842000000260B002096
:10D98C0000000000010000008DEE000842000000C5
:10D99C00660B0020000000000100000043F20008AC
:10D9AC0044000000D40A002000000000D007000052
:10D9BC00A2EE000844000000D60A0020000000007F
:10D9CC00D0070000AFEE000844000000D80A002089
:10D9DC0000000000D0070000BBEE0008440000006F
:10D9EC00DA0A002000000000D0070000CEEE00088C
:10D9FC0044000000DC0A002000000000D0070000FA
:10DA0C00DEEE000844000000DE0A002000000000EA
:10DA1C00D0070000EFEE000844000000E00A0020F0
:10DA2C0000000000D0070000FAEE000844000000DF
:10DA3C00E20A002000000000D00700000FEF0008F1
:10DA4C0044000000E40A002032000000007D0000C9
:10DA5C001EEF000844000000E60A0020320000001F
:10DA6C00F20100002DEF000841000000700B0020B7
:10DA7C0000000000010000003AEF00084100000027
:10DA8C00710B002000000000010000004DEF0008A9
:10DA9C0041000000720B0020000000003C00000060
:10DAAC005FEF000841000000730B00200000000035
:10DABC00B40000006BEF000842000000780B00205F
:10DACC00FFFFFFFF0100000081EF00084100000094
:10DADC007A0B0020300000007E00000092EF00085E
:10DAEC0041000000220B0020000000000600000096
:10DAFC00A4EF000841000000230B002000000000F0
:10DB0C000A000000B6EF0008410000008C0B00205A
:10DB1C000000000001000000C7EF000841000000F9
:10DB2C008D0B00200000000001000000DBEF00085E
:10DB3C0060000000900B0020A6FFFFFF5A000000C1
:10DB4C00F3EF000860000000940B00204CFFFFFF77
:10DB5C00B40000000BF0000841000000980B0020FE
:10DB6C00000000000100000024F00008410000004B
:10DB7C00990B002000000000010000002FF00008AD
:10DB8C00410000009A0B0020000000000100000082
:10DB9C0044F00008410000009B0B00200000000036
:10DBAC00780000005EF0000844000000180B002014
:10DBBC0000000000204E00006FF000084100000043
:10DBCC000C0B002000000000FF0000007AF00008A1
:10DBDC00410000000F0B00200A0000003200000082
:10DBEC0090F0000841000000100B00200A0000001B
:10DBFC0032000000A6F0000841000000110B0020CC
:10DC0C000A00000032000000C0F0000848000000CC
:10DC1C00120B0020F0D8FFFF10270000D4F00008F2
:10DC2C0044000000140B002000000000E40C000075
:10DC3C00E9F0000841000000170B00200000000074
:10DC4C000100000007F1000841000000160B002045
:10DC5C0000000000020000001AF100084100000062
:10DC6C00E80A0020000000000800000025F1000870
:10DC7C0041000000E90A002000000000080000003C
:10DC8C002FF1000841000000EA0A0020000000000B
:10DC9C000800000039F1000848000000EC0A0020E0
:10DCAC004CFFFFFF680100004AF10008480000002B
:10DCBC00EE0A00204CFFFFFF680100005CF1000839
:10DCCC0048000000F00A00204CFFFFFF6801000034
:10DCDC006CF1000844000000FE0A00206400000003
:10DCEC008403000082F1000844000000F40A0020C4
:10DCFC0000000000000100008BF100084100000052
:10DD0C00FA0A002000000000800000009BF10008CF
:10DD1C0044000000F60A002064000000E803000044
:10DD2C00ACF1000844000000F80A00206400000078
:10DD3C00E8030000BEF1000881000000AF0C0020D9
:10DD4C0001000000FA000000D0F100088100000082
:10DD5C00B00C00200000000001000000C7F100081A
:10DD6C0081000000AD0C002000000000200000002D
:10DD7C00E5F1000881000000AE0C0020000000005E
:10DD8C0064000000F2F1000881000000B40C0020D7
:10DD9C0000000000960000000CF200088400000057
:10DDAC00B20C0020010000008403000026F20008E1
:10DDBC0042000000F20A0020FFFFFFFF01000000FC
:10DDCC003CF2000841000000740B00200000000031
:10DDDC000100000050F2000842000000750B00200A
:10DDEC00FFFFFFFF0100000064F200084400000088
:10DDFC00760B002050000000F40100007EF20008B9
:10DE0C0081000000F00B0020000000000200000068
:10DE1C0093F2000801010000F20E00200000000047
:10DE2C00FA0000009BF2000801010000F30E002034
:10DE3C000000000064000000A3F2000801010000D3
:10DE4C00FA0E00200000000064000000AFF2000891
:10DE5C0001010000F40E002000000000640000002E
:10DE6C00B7F2000801010000F50E002000000000D0
:10DE7C0064000000C0F2000801010000F60E002052
:10DE8C000000000064000000CAF20008010100005C
:10DE9C00F70E00200000000064000000D5F200081E
:10DEAC0001010000F80E002000000000FF0000003F
:10DEBC00DEF2000801010000F90E00200000000055
:10DECC0064000000E7F2000804010000FC0E0020D2
:10DEDC00E8030000D0070000F6F200084100000043
:10DEEC00680B002000000000C800000005F30008CB
:10DEFC0041000000690B002000000000C800000079
:10DF0C0018F30008440000006A0B0020E80300002E
:10DF1C00D00700002AF30008410000006C0B002021
:10DF2C0000000000010000003FF300084400000066
:10DF3C006E0B0020000000002C0100005BF30008B9
:10DF4C00440000002E0B0020EE020000CA08000066
:10DF5C0067F3000844000000300B0020EE020000C4
:10DF6C00CA08000073F3000841000000F30A002007
:10DF7C00000000000900000080F300088100000090
:10DF8C00F80B002000000000FA0000008FF30008DE
:10DF9C0081000000000C0020000000006400000064
:10DFAC009EF3000881000000010C0020000000001E
:10DFBC0064000000ACF30008A0000000FC0B002083
:10DFCC000100000014000000BCF3000881000000F8
:10DFDC00140C00200000000001000000CBF300082E
:10DFEC0088000000F60B0020D4FEFFFF2C0100007F
:10DFFC00DAF3000888000000F40B0020D4FEFFFFC9
:10E00C002C010000E8F3000881000000040C002043
:10E01C000000000030000000F6F30008A000000033
:10E02C00080C0020000000000100000005F40008AE
:10E03C00A00000000C0C00200000000001000000FB
:10E04C0011F40008A0000000100C002000000000DB
:10E05C00010000001DF4000841000000FC0A002033
:10E06C0000000000040000002BF400084100000038
:10E07C00FB0A0020000000000300000038F4000838
:10E08C0088000000F20B0020B0B9FFFF50460000E2
:10E09C0048F40008810000009C0B002000000000E8
:10E0AC000500000057F40008810000009E0B0020C2
:10E0BC0000000000C80000005FF4000881000000B0
:10E0CC00A80B002000000000C800000054F100085C
:10E0DC0081000000B20B002000000000C80000000E
:10E0EC0067F40008810000009D0B00200000000078
:10E0FC00C80000006EF4000881000000A70B00208F
:10E10C0000000000C800000043F10008810000007E
:10E11C00B10B002000000000C800000075F40008DE
:10E12C00810000009F0B002000000000C8000000D0
:10E13C007BF4000881000000A90B00200000000007
:10E14C00C800000066F1000881000000B30B00203D
:10E15C0000000000C800000081F40008A0000000CE
:10E16C00C00B002000000000640000008AF40008CE
:10E17C00A0000000CC0B0020000000006400000098
:10E18C0093F40008A0000000D80B00200000000051
:10E19C00640000009CF40008A0000000BC0B0020F0
:10E1AC000000000064000000A4F40008A0000000BF
:10E1BC00C80B00200000000064000000ACF4000854
:10E1CC00A0000000D40B0020000000006400000040
:10E1DC00B4F40008A0000000C40B002000000000F4
:10E1EC0064000000BBF40008A0000000D00B00206D
:10E1FC000000000064000000C2F40008A000000051
:10E20C00DC0B00200000000064000000C9F40008D2
:10E21C00A0000000E40B0020000000000A00000039
:10E22C00D7F40008A0000000E00B00200000000064
:10E23C000A000000E3F4000881000000E80B002055
:10E24C0000000000FA000000F7F400088100000054
:10E25C00A00B002000000000C8000000FDF4000826
:10E26C0081000000AA0B002000000000C800000084
:10E27C0003F5000881000000B40B00200000000032
:10E28C00C800000009F5000881000000A40B002064
:10E29C0000000000C800000011F50008810000001B
:10E2AC00AE0B002000000000C800000019F50008AB
:10E2BC0081000000B80B002000000000C800000026
:10E2CC0021F5000881000000A60B002000000000D2
:10E2DC00C800000027F5000881000000B00B0020EA
:10E2EC0000000000C80000002DF5000881000000AF
:10E2FC00BA0B002000000000C800000033F5000835
:10E30C0084000000EA0B002064000000F40100000F
:10E31C003FF5000881000000EE0B0020000000001B
:10E32C00C80000004BF5000881000000ED0B002038
:10E33C0000000000C800000058F500088100000033
:10E34C00EC0B002000000000C800000065F5000880
:10E35C0048000000060B00200080FFFFFF7F00003C
:10E36C006FF5000848000000080B00200080FFFF3C
:10E37C00FF7F000079F50008480000000A0B002020
:10E38C000080FFFFFF7F0000E2EB0008EBEB0008D2
:10E39C00000000000D34000807EC00080BEC00082E
:10E3AC000000000023320008D2EB00081BEC000830
:10E3BC0000000000598D000838EC00083DEC000806
:10E3CC0050EC00087538000861EC000800000000F3
:10E3DC00000000005931000866EC00086EEC0008E3
:10E3EC0081EC00085330000894EC000898EC00080D
:10E3FC008DEC00081D890008ABEC00080000000043
:10E40C0000000000D98C0008B0EC0008B4EC000847
:10E41C00CFEC0008358C0008D7EC0008DCEC0008C9
:10E42C000000000051300008F7EC0008EFEC000889
:10E43C00FDEC0008C58600080FED00080000000088
:10E44C001AED0008018600082DED000826ED0008E5
:10E45C0035ED0008858600083FED00084BED0008FF
:10E46C0035ED0008398600085FED000867ED0008FF
:10E47C00000000002133000883ED00088AED00083D
:10E48C00000000006D350008A8ED0008ADED000897
:10E49C0000000000758D0008BDED0008C4ED0008FB
:10E4AC00000000002937000814E70008DBED000825
:10E4BC00EAED00087589000800EE0008FBED000885
:10E4CC00000000008D8800080CEE000807EE000824
:10E4DC0000000000038600080D1B5B4B000D0A2397
:10E4EC0020001B5B324A1B5B313B314800556E6B85
:10E4FC006E6F776E20636F6D6D616E642C2074721D
:10E50C0079202768656C702700082008000D0A45E3
:10E51C006E746572696E6720434C49204D6F64655B
:10E52C002C20747970652027657869742720746FA6
:10E53C002072657475726E2C206F72202768656C62
:10E54C0070270D0A00000000000000400008014088
:10E55C000100001C002800000000004000080140E1
:10E56C000200041C002800000000004000080140CC
:10E57C000400081C002800000000004000080140B6
:10E58C0008000C1C0028000000040040000801409A
:10E59C004000001D0028000000040040000801405D
:10E5AC008000041D0028000000040040000C014005
:10E5BC000100081D0028000000040040000C014070
:10E5CC0002000C1D00280000002C01400008014036
:10E5DC000001001B01280000002C01400008014034
:10E5EC0000080C1B0128000000080040000C014032
:10E5FC004000001E0028000000080040000C0140F4
:10E60C008000041E0028000000080040000C01409F
:10E61C000001081E0028000000080040000C01400A
:10E62C0000020C1E00280000456E61626C65643AA5
:10E63C002000257320006C69737400417661696C4D
:10E64C0061626C653A2000496E76616C6964206E7B
:10E65C00616D650D0A00756E617661696C61626C45
:10E66C00650D0A0044697361626C656400456E61F6
:10E67C00626C6564000D0A4C656176696E672043B7
:10E68C004C49206D6F64652C20756E7361766564E2
:10E69C00206368616E676573206C6F73742E0D0A4E
:10E6AC0000736574202573203D200061757820254A
:10E6BC00752025752025752025752025750D0A00DA
:10E6CC002573206D7573742062652062657477659F
:10E6DC00656E20256420616E642025640D0A006936
:10E6EC006E646578005061727365206572726F722A
:10E6FC000D0A00727872616E67652025752025758C
:10E70C002025750D0A0072657365740061646A7268
:10E71C00616E67652025752025752025752025756A
:10E72C002025752025752025750D0A0072786661E7
:10E73C00696C2025752025632025640D0A007278EC
:10E74C006661696C2025752025630D0A007365725E
:10E75C0069616C20256420256420256C6420256C5F
:10E76C006420256C6420256C640D0A006D61737443
:10E77C006572007261746573000D0A2320766572F0
:10E78C0073696F6E0D0A000D0A232064756D70207D
:10E79C006D61737465720D0A000D0A23206D697822
:10E7AC0065720D0A000D0A0D0A23206665617475E9
:10E7BC0072650D0A0066656174757265202D25738E
:10E7CC000D0A00666561747572652025730D0A006B
:10E7DC000D0A0D0A23206D61700D0A006D61702009
:10E7EC0025730D0A000D0A0D0A23207365726961E9
:10E7FC006C0D0A000D0A232072786661696C0D0A93
:10E80C00000D0A232064756D702070726F66696C40
:10E81C00650D0A000D0A232070726F66696C650D18
:10E82C000A000D0A23206175780D0A000D0A2320B9
:10E83C0061646A72616E67650D0A000D0A232072AD
:10E84C007872616E67650D0A000D0A232064756D80
:10E85C00702072617465730D0A000D0A23207261B9
:10E86C00746570726F66696C650D0A0052585F5062
:10E87C00504D005642415400494E464C494748546D
:10E88C005F4143435F43414C0052585F53455249EB
:10E89C00414C004D4F544F525F53544F5000534511
:10E8AC0052564F5F54494C5400534F4654534552A3
:10E8BC0049414C00475053004641494C5341464551
:10E8CC0000534F4E41520054454C454D45545259FE
:10E8DC000043555252454E545F4D455445520033FA
:10E8EC00440052585F504152414C4C454C5F50577C
:10E8FC004D0052585F4D535000525353495F4144A1
:10E90C0043004C45445F53545249500044495350C2
:10E91C004C4159004F4E4553484F5431323500420B
:10E92C004C41434B424F58004348414E4E454C5F7F
:10E93C00464F5257415244494E470053657020315F
:10E94C003620323031350032333A33363A333400F4
:10E95C00663530626563300041524D3B00414E4795
:10E96C004C453B00484F52495A4F4E3B0042415296
:10E97C004F3B004D41473B004845414446524545BD
:10E98C003B004845414441444A3B0043414D5354AC
:10E99C0041423B0043414D545249473B0047505381
:10E9AC0020484F4D453B0047505320484F4C443B6B
:10E9BC000050415353544852553B00424545504535
:10E9CC00523B004C45444D41583B004C45444C4F48
:10E9DC00573B004C4C49474854533B0043414C492E
:10E9EC00423B00474F5645524E4F523B004F53440B
:10E9FC002053573B0054454C454D455452593B0010
:10EA0C004155544F54554E453B00534F4E41523B8C
:10EA1C0000534552564F313B00534552564F323BF3
:10EA2C0000534552564F333B00424C41434B424FEF
:10EA3C00583B004641494C534146453B002E003063
:10EA4C003132333435363738394142434445464701
:10EA5C0048494A4B4C4D4E4F5051525354555657B2
:10EA6C0058595A00414552543132333435363738BF
:10EA7C0061626364656667680041455452313233A4
:10EA8C003400232042657461466C696768742F25D5
:10EA9C0073202573202573202F20257320282573A0
:10EAAC002900434A4D435500312E31302E3000722F
:10EABC0061746570726F66696C652025640D0A005F
:10EACC006D6F746F722025643A2025640D0A002046
:10EADC0025642025640053797374656D205570741A
:10EAEC00696D653A202564207365636F6E64732CC1
:10EAFC0020566F6C746167653A202564202A20309B
:10EB0C002E31562028256453206261747465727905
:10EB1C00202D202573290D0A0043505520436C6F7E
:10EB2C00636B3D25644D487A004379636C652054D2
:10EB3C00696D653A2025642C204932432045727258
:10EB4C006F72733A2025642C20636F6E66696720A0
:10EB5C0073697A653A2025640D0A004375727265F3
:10EB6C006E742073657474696E67733A200D0A00B5
:10EB7C0025732073657420746F200056616C756565
:10EB8C002061737369676E6D656E74206F75742088
:10EB9C006F662072616E67650D0A004D61703A20D8
:10EBAC0000202D202573000D0A092573000D0A5233
:10EBBC0065626F6F74696E67005265736574746912
:10EBCC006E6720746F2064656661756C7473005396
:10EBDC006176696E670061646A72616E6765006375
:10EBEC006F6E6669677572652061646A7573746DA2
:10EBFC00656E742072616E67657300617578006371
:10EC0C006F6E666967757265206D6F6465730072EF
:10EC1C006573657420746F2064656661756C7473BC
:10EC2C0020616E64207265626F6F740064756D7024
:10EC3C000064756D7020636F6E66696775726174C0
:10EC4C00696F6E005B6D61737465727C70726F6658
:10EC5C00696C655D006578697400666561747572D0
:10EC6C006500636F6E6669677572652066656174B1
:10EC7C0075726573006C6973740D0A093C2B7C2DDD
:10EC8C003E5B6E616D655D00676574006765742041
:10EC9C007661726961626C652076616C756500687D
:10ECAC00656C70006D617000636F6E66696775727C
:10ECBC0065207263206368616E6E656C206F726490
:10ECCC006572005B3C6D61703E5D006D6D69780036
:10ECDC00637573746F6D206D6F746F72206D6978CE
:10ECEC006572006765742F736574206D6F746F7235
:10ECFC00003C696E6465783E205B3C76616C7565A2
:10ED0C003E5D00706C61795F736F756E64005B3C87
:10ED1C00696E6465783E5D0D0A006368616E6765B7
:10ED2C002070726F66696C65005B3C696E64657817
:10ED3C003E5D007261746570726F66696C6500632C
:10ED4C0068616E676520726174652070726F6669A8
:10ED5C006C6500727872616E676500636F6E6669D0
:10ED6C0067757265207278206368616E6E656C20C1
:10ED7C0072616E6765730072786661696C007368A6
:10ED8C006F772F736574207278206661696C73617C
:10ED9C0066652073657474696E677300736176655C
:10EDAC00007361766520616E64207265626F6F74AA
:10EDBC000073657269616C00636F6E66696775726A
:10EDCC00652073657269616C20706F727473006377
:10EDDC0068616E67652073657474696E67005B3C6F
:10EDEC006E616D653E3D3C76616C75653E5D007394
:10EDFC00686F77207374617475730073686F772014
:10EE0C0076657273696F6E006C6F6F7074696D6587
:10EE1C000073796E635F6779726F5F746F5F6C6F8D
:10EE2C006F7000656D665F61766F6964616E6365B6
:10EE3C000072635F736D6F6F7468696E67006D69E4
:10EE4C00645F7263006D696E5F636865636B006D10
:10EE5C0061785F636865636B00727373695F636885
:10EE6C00616E6E656C00727373695F7363616C6560
:10EE7C0000727373695F70706D5F696E7665727422
:10EE8C0000696E7075745F66696C746572696E6723
:10EE9C005F6D6F6465006D61785F7468726F747418
:10EEAC006C65006D696E5F636F6D6D616E64007390
:10EEBC006572766F5F63656E7465725F70756C7387
:10EECC00650033645F6465616462616E645F6C6F7E
:10EEDC00770033645F6465616462616E645F686966
:10EEEC0067680033645F6E65757472616C003364BF
:10EEFC005F6465616462616E645F7468726F747480
:10EF0C006C65006D6F746F725F70776D5F7261749A
:10EF1C006500736572766F5F70776D5F7261746593
:10EF2C000072657461726465645F61726D0064691E
:10EF3C007361726D5F6B696C6C5F73776974636816
:10EF4C00006175746F5F64697361726D5F64656C89
:10EF5C00617900736D616C6C5F616E676C650066E6
:10EF6C006978656477696E675F616C74686F6C64EF
:10EF7C005F646972007265626F6F745F636861725F
:10EF8C0061637465720073657269616C72785F702D
:10EF9C00726F7669646572007370656B7472756DEF
:10EFAC005F7361745F62696E640074656C656D6536
:10EFBC007472795F7377697463680074656C656DDE
:10EFCC00657472795F696E76657273696F6E0066CF
:10EFDC0072736B795F64656661756C745F6C617478
:10EFEC00746974756465006672736B795F646566C9
:10EFFC0061756C745F6C6F6E6769747564650066BF
:10F00C0072736B795F636F6F7264696E6174657331
:10F01C005F666F726D6174006672736B795F756E8B
:10F02C006974006672736B795F766661735F707278
:10F03C0065636973696F6E00686F74745F616C618E
:10F04C00726D5F736F756E645F696E7465727661F5
:10F05C006C00626174746572795F6361706163697D
:10F06C00747900766261745F7363616C65007662BB
:10F07C0061745F6D61785F63656C6C5F766F6C74E7
:10F08C0061676500766261745F6D696E5F63656C64
:10F09C006C5F766F6C7461676500766261745F7724
:10F0AC0061726E696E675F63656C6C5F766F6C74B2
:10F0BC006167650063757272656E745F6D6574650A
:10F0CC00725F7363616C650063757272656E745FF9
:10F0DC006D657465725F6F6666736574006D756CD3
:10F0EC0074697769695F63757272656E745F6D655B
:10F0FC007465725F6F757470757400637572726588
:10F10C006E745F6D657465725F7479706500616CA7
:10F11C0069676E5F6779726F00616C69676E5F61BA
:10F12C00636300616C69676E5F6D616700616C6938
:10F13C00676E5F626F6172645F726F6C6C00616CA2
:10F14C0069676E5F626F6172645F70697463680097
:10F15C00616C69676E5F626F6172645F7961770081
:10F16C006D61785F616E676C655F696E636C696E0B
:10F17C006174696F6E006779726F5F6C7066006D99
:10F18C006F726F6E5F7468726573686F6C64006722
:10F19C0079726F5F636D70665F666163746F720026
:10F1AC006779726F5F636D70666D5F666163746FB4
:10F1BC007200616C745F686F6C645F64656164623B
:10F1CC00616E6400616C745F686F6C645F66617320
:10F1DC00745F6368616E6765007961775F64656110
:10F1EC006462616E64007468726F74746C655F63E2
:10F1FC006F7272656374696F6E5F76616C756500B2
:10F20C007468726F74746C655F636F72726563742B
:10F21C00696F6E5F616E676C65007961775F636FB4
:10F22C006E74726F6C5F646972656374696F6E0083
:10F23C007069645F61745F6D696E5F7468726F741E
:10F24C00746C65007961775F6D6F746F725F646960
:10F25C0072656374696F6E007961775F6A756D7042
:10F26C005F70726576656E74696F6E5F6C696D69DF
:10F27C00740064656661756C745F726174655F704F
:10F28C00726F66696C650072635F7261746500729F
:10F29C00635F6578706F0072635F7961775F657823
:10F2AC00706F007468725F6D6964007468725F657A
:10F2BC0078706F00726F6C6C5F726174650070694E
:10F2CC007463685F72617465007961775F726174F1
:10F2DC0065007470615F72617465007470615F6267
:10F2EC007265616B706F696E74006661696C7361D5
:10F2FC0066655F64656C6179006661696C736166F3
:10F30C00655F6F66665F64656C6179006661696CE8
:10F31C00736166655F7468726F74746C65006661A6
:10F32C00696C736166655F6B696C6C5F737769742C
:10F33C006368006661696C736166655F7468726F9F
:10F34C0074746C655F6C6F775F64656C6179007267
:10F35C00785F6D696E5F757365630072785F6D6160
:10F36C00785F75736563006163635F68617264776E
:10F37C00617265006163635F6C70665F6661637484
:10F38C006F720061636378795F6465616462616E5A
:10F39C0064006163637A5F6465616462616E6400DA
:10F3AC006163637A5F6C70665F6375746F66660029
:10F3BC006163635F756E61726D656463616C00613E
:10F3CC0063635F7472696D5F706974636800616315
:10F3DC00635F7472696D5F726F6C6C006261726FE7
:10F3EC005F7461625F73697A65006261726F5F6EF0
:10F3FC006F6973655F6C7066006261726F5F6366E4
:10F40C005F76656C006261726F5F63665F616C74DE
:10F41C00006261726F5F6861726477617265006D22
:10F42C0061675F6861726477617265006D61675FC7
:10F43C006465636C696E6174696F6E007069645F9A
:10F44C00636F6E74726F6C6C657200705F70697450
:10F45C00636800695F706974636800705F726F6CD9
:10F46C006C00695F726F6C6C00705F79617700691A
:10F47C005F79617700705F70697463686600695FBB
:10F48C0070697463686600645F70697463686600B1
:10F49C00705F726F6C6C6600695F726F6C6C66008B
:10F4AC00645F726F6C6C6600705F7961776600697F
:10F4BC005F7961776600645F79617766006C657669
:10F4CC00656C5F686F72697A6F6E006C6576656CDF
:10F4DC005F616E676C650073656E736974697669DC
:10F4EC0074795F686F72697A6F6E00705F616C74AB
:10F4FC0000695F616C7400645F616C7400705F6CB8
:10F50C006576656C00695F6C6576656C00645F6C34
:10F51C006576656C00705F76656C00695F76656C0E
:10F52C0000645F76656C007961775F705F6C696D04
:10F53C006974006779726F5F6375745F687A0070C5
:10F54C007465726D5F6375745F687A00647465725C
:10F55C006D5F6375745F687A006D61677A65726F51
:10F56C005F78006D61677A65726F5F79006D6167B6
:10F57C007A65726F5F7A004F4B005741524E494E7D
:10F58C004700435249544943414C004E4F5420507C
:10F59C00524553454E54000020202020202020208E
:10F5AC002028282828282020202020202020202027
:10F5BC002020202020202020881010101010101047
:10F5CC00101010101010101004040404040404048F
:10F5DC000404101010101010104141414141410120
:10F5EC0001010101010101010101010101010101FF
:10F5FC00010101101010101010424242424242020E
:10F60C0002020202020202020202020202020202CE
:10F61C000202021010101020000000000000000078
:10F62C0000000000000000000000000000000000CE
:10F63C0000000000000000000000000000000000BE
:10F64C0000000000000000000000000000000000AE
:10F65C00000000000000000000000000000000009E
:10F66C00000000000000000000000000000000008E
:10F67C00000000000000000000000000000000007E
:10F68C00000000000000000000000000000000006E
:10F69C0000000000000000000000004B000000CB48
:10F6AC0061636F7366000000000000007371727478
:10F6BC00660000006937AC3168212233B40F143373
:10F6CC006821A2333863ED3EDA0F493F5E987B3FE9
:04F6DC00DA0FC93F39
:08F6E00080A6FF7F010000007D
:10F6E8000000803F00000000000000000300000050
:10F6F8000000803F0000803F0000803F01000001C3
:10F70800B957000800127A00010000000001010149
:10F71800417F00080300000000A24A04A3F5000886
:10F7280000000000000000000000000000000000D1
:10F7380000000000000000000000000000000000C1
:10F748000CE90008000000000000000000000000B4
:10F7580000000000000000000000000000000000A1
:10F768000000000000000000000000000000000091
:10F778000000000000000000000000000000000081
:08F78800400000200100000018
:0400000508000000EF
:00000001FF
